:020000040800F2
:10000000F8FF012041840908C1840908E12F08088C
:10001000C1840908C1840908C184090800000000DE
:10002000000000000000000000000000C18409087A
:10003000C184090800000000C1840908453008088F
:10004000C1840908C1840908C1840908C184090858
:10005000C1840908C1840908715C0808B15D0808F9
:10006000715D0808315D0808F15C080859590908F4
:100070004959090839590908295909081559090818
:1000800001590908ED580908C1840908C184090803
:10009000C1840908C1840908C1840908B15C080841
:1000A000C184090829680908C18409081968090870
:1000B00009680908F9670908E96709088D570908F7
:1000C000B1570908D1560908F55609088D5909088C
:1000D00081590908813D0808753D0808693D0808EF
:1000E000315C0808C1840908000000009167090814
:1000F000A167090881670908C9670908D95809086B
:10010000C1840908E52A0908D96709087559090849
:100110005D3D0808C1840908C1840908818104087B
:10012000C5580908B15809089D580908895809088F
:1001300075580908C1840908C1840908C1840908DF
:1001400000000000000000000000000000000000AF
:10015000615809084D58090839580908513D0808DF
:10016000C1840908C1840908C1840908C184090837
:10017000C1840908C1840908C1840908000000007D
:10018000C1840908C1840908453D0808393D0808AB
:1001900069590908C1840908C1840908C18409088A
:1001A000C1840908C1840908C1840908C1840908F7
:1001B000C1840908C1840908C1840908C1840908E7
:1001C000C1840908C1840908C1840908C1840908D7
:1001D000C184090809840408C1840908C184090884
:1001E000C1840908C1840908C1840908C1840908B7
:1001F000C1840908C1840908C1840908C1840908A7
:10020000C1840908C1840908C1840908C184090896
:10021000716709086167090851670908C1840908FD
:10022000C1840908C1840908C184090800000000CC
:10023000092D0908C184090800000000C1840908CB
:10024000C1840908C1840908C1840908C184090856
:10025000C1840908C1840908C1840908C184090846
:10026000C1840908C1840908C1840908C184090836
:10027000C1840908C1840908C1840908000000007C
:10028000C184090800000000C184090800000000C2
:0802900000000000C184090810
:08029800E07E090001000000F6
:1002A0002320010010000000FC590024B85A00244B
:1002B00000000000912706080D10010070000000EA
:1002C000F8580024C85A002400000000EDE4070894
:1002D000040008008000000050580024385B00240F
:1002E0000000000000000000090201000100000001
:1002F000F8570024B85B002400000000500A0008F2
:10030000F901010004000000D4570024BC5B002464
:1003100000000000FD440808FB010100010000008E
:1003200094570024C05B0024000000009DD90808F9
:10033000FC0101000900000060560024C45B002499
:1003400000000000ADD90808F70101000600000018
:1003500054560024D05B002400000000520A00081C
:100360000A800100280000002C560024D85B0024DD
:10037000000000007D260608160215003F00000060
:1003800048440024005C0024000000002DD0080830
:10039000340001001000000058550024405C002487
:1003A000000000004D5B060811020100080000007B
:1003B00030550024505C002400000000580A00085A
:1003C000121201000400000028550024585C00248B
:1003D00000000000600A0008182001003200000040
:1003E000F45400245C5C0024000000007DDA08085E
:1003F000061001001C0000002C440024905C002426
:1004000000000000CDD9080813020100040000001C
:100410009C1E0024AC5C002400000000640A00085C
:10042000FD01010021000000E8530024B05C00241D
:1004300000000000514408081220010011000000D3
:10044000C4590024D45C002400000000680A00089D
:10045000000201000B000000B44E0024E85C002400
:100460000000000000000000020201000300000084
:10047000D4240024F45C00240000000000000000EC
:100480000C02010004000000BC240024F85C0024DD
:1004900000000000F1D80808FE010100140000006F
:1004A000444B0024FC5C0024000000009DCF0808A1
:1004B0001402010005000000745D0024D85D0024D2
:1004C000000000007A0A00080E020100020000008D
:1004D000705D0024E05D002400000000800A000838
:1004E00023120100100000000884002488880024E2
:1004F00000000000840A0008371001002E000000F0
:10050000348800249888002400000000940A000821
:10051000161001000600000000840024C888002492
:1005200000000000C20A00082F1001002200000095
:1005300064880024D088002400000000C80A000855
:100540001E000100090000002C820024F488002411
:1005500000000000EA0A0008051001000600000083
:10056000DC8300240089002400000000F40A000855
:10057000F5810100680000008881002408890024BA
:1005800000000000CD320508FD07010076000000E4
:10059000CE8000247089002400000000BD110508F1
:1005A000261001000E000000F8890024E8890024CC
:1005B00000000000311005080B3001001A00000097
:1005C000B4800024388A002400000000FA0A0008E1
:1005D0001F30010024000000C0820024548A00243F
:1005E00000000000140B00080502010004000000D8
:1005F0009C840024788A002400000000380B000846
:10060000030101000A000000448200247C8A0024C7
:1006100000000000210C0508012001000C00000072
:10062000F09200248C9C0024000000003C0B000889
:100630000EF003009E01000008900024989C002406
:1006400000000000F93B0608130001000400000050
:1006500014970024389E002400000000480B000876
:100660000101010004000000488F00243C9E00248A
:100670000000000000000000000101000400000074
:10068000408F0024409E0024000000004C0B000816
:1006900002010100030000003C8F0024449E00245E
:1006A00000000000295A0708220201001C01000076
:1006B000F4970024489E00240000000035DA080862
:1006C0000C200600CC000000CC910024649F002484
:1006D00000000000E9590708010201000B000000BA
:1006E000548F002430A0002400000000BDD0080872
:1006F0001B02010010000000F09500243CA0002423
:100700000000000041D108081B1001000C0000008F
:10071000108C00244CA000240000000031A8050823
:1007200021020100F0000000948A002458A0002457
:100730000000000005A205081A0001000E000000DC
:1007400010AF002458AF002400000000500B000838
:10075000203201000A00000000AE002468AF00242F
:1007600000000000D53B06081500100070000000D6
:10077000C0AC002474AF00240000000000000000A2
:100780002A00080060000000D0AB0024E4AF002481
:1007900000000000AD3B06082C0004001000000023
:1007A00054B0002444B00024000000008D39060835
:1007B0002B0012002400000088B0002464B0002444
:1007C00000000000613906082920140078000000AC
:1007D000B0A90024ACB0002400000000000000001C
:1007E000F62101000C000000C8A7002424B1002459
:1007F00000000000600B00081C0202001C0000004A
:1008000070A7002474B100240000000009D9080872
:1008100028200100180000008CA7002490B10024BB
:1008200000000000253C0608140001000400000040
:1008300060A70024A8B10024000000006C0B000891
:1008400003000100010000006CB30024A4B60024E2
:100850000000000000000000031201003D00000045
:1008600060B60024A8B6002400000000700B000849
:1008700025201E002C010000C4B30024E8B600248B
:100880000000000000000000101001000200000045
:10089000ACB3002414B8002400000000AE0B000824
:1008A000F8210100060000005CB3002418B8002401
:1008B00000000000B00B0008190001000500000056
:1008C0007CB2002420B8002400000000B60B000811
:1008D000020001000C000000DCBB0024ECBB002483
:1008E000000000000000000029020100400000009C
:1008F000E8BA0024F8BB002400000000BC0B00088C
:100900000A0201001400000054BB002458BC00245B
:1009100000000000AD5C07081F0208001000000086
:10092000CCC10024E0C2002400000000D1CF0808A0
:100930001A0201003C000000D0BD0024F0C20024D7
:1009400000000000F1DA0808381001000100000082
:1009500084BC00242CC3002400000000FC0B000811
:10096000FF11010006000000C8BD002430C30024B0
:10097000000000001DD00808280204000400000048
:10098000BCC300247CCA0024000000003DD108083C
:100990002702040004000000B8C3002480CA002419
:1009A0000000000031D10808260201000600000006
:1009B0009CCA002434D0002400000000FE0B000874
:1009C00007020100020000001CD000243CD00024DB
:1009D00000000000040C00080602040010000000E3
:1009E000FCCF002440D0002400000000C1D808083B
:1009F000081206001E000000DCCF002450D00024A6
:100A000000000000CDD008082502110011000000F0
:100A100084D0002470D00024000000001DD70808F6
:100A200027000100040000000CCB002498D0002413
:100A300000000000060C0008100201000100000088
:100A4000A0D000249CD00024000000000A0C000864
:100A500000001F010000C4094A4B00000101010110
:100A6000FFFFFFFF00000152000000010000054DE4
:100A700037343300000000020000000001FF0100D5
:100A80000000000000000000000000000000000066
:100A90000000000020003200C800D00796001400BB
:100AA000320028004C0440060005500014000F00DE
:100AB000080064000100010005000A000000F401C4
:100AC0009600C409000019000000000000000000AA
:100AD0000000000000000000000000000000000016
:100AE0000000000000000000000000050100000000
:100AF00000000000200002010000AE014A015E017A
:100B00002C0164010100000001000A019A01001E8D
:100B10000A000002000000000001000000050000C3
:100B200001020300000000000000000000000000BF
:100B3000000000000080070000000000E8036400DF
:100B4000040A000114001E0008044430FA000000EA
:100B50007E05EA05B4053200E803D0070000000076
:100B6000000000000100000002020000030000235A
:100B70000000000000000000000000000000000075
:100B80000000000000000000000000000000000065
:100B90000000000000000000000000000000000055
:100BA000000000000000000000000000010000053F
:100BB0000101F40114000000280100000000000001
:100BC0000000000000000000000000000000000025
:100BD0000000000000000000000000000000000015
:100BE0000000000000000000000000000000000005
:100BF00000000000000000000000000000003C4277
:0B0C000038393A3B003C2003000000A4
:100C0B0000C20100000008000A06000200000040BC
:100C1B000100000009026400030100C03209040056
:100C2B000001030000000921110100012236000719
:100C3B0005830308000A080B0102020201000904E4
:100C4B00010001020201000524001001052401002E
:100C5B000204240202052406010207058203080090
:100C6B00FF09040200020A00000007050102400010
:100C7B00000705810240000071D50408F9A404089F
:100C8B00EDD2040800000000A5990408FDD004086B
:100C9B00D1990408000000000000000000000000D3
:100CAB0085990408959904087599040865990408B1
:100CBB001A0300000000000000000000000000000C
:100CCB000000000000000000000000000403090405
:100CDB0012010002EF0201408304563200020102AE
:100CEB000301000012010002020000408304405780
:100CFB0000020102030100000090D003000002403B
:100D0B0010000240000000000000000000000B007B
:100D1B000000000000000000000000000000024086
:100D2B0028000240010000000000000006000C003B
:100D3B000000000000000000000000000000024066
:100D4B0040000240020000000000000010000D00F7
:100D5B000000000000000000000000000000024046
:100D6B0058000240030000000000000016000E00B7
:100D7B000000000000000000000000000000024026
:100D8B0070000240040000000000000020000F0073
:100D9B000000000000000000000000000000024006
:100DAB008800024005000000000000002600100033
:100DBB0000000000000000000000000000000240E6
:100DCB00A0000240060000000000000030001100EF
:100DDB0000000000000000000000000000000240C6
:100DEB00B8000240070000000000000036002F0092
:100DFB0000000000000000000000000000040240A2
:100E0B001004024000000000000000000000380049
:100E1B000000000000000000000000000004024081
:100E2B002804024001000000000000000600390009
:100E3B000000000000000000000000000004024061
:100E4B0040040240020000000000000010003A00C5
:100E5B000000000000000000000000000004024041
:100E6B0058040240030000000000000016003B0085
:100E7B000000000000000000000000000004024021
:100E8B0070040240040000000000000020003C0041
:100E9B000000000000000000000000000004024001
:100EAB0088040240050000000000000026004400FA
:100EBB0000000000000000000000000000040240E1
:100ECB00A0040240060000000000000030004500B6
:100EDB0000000000000000000000000000040240C1
:100EEB00B804024007000000000000003600460076
:100EFB000000000000000000000000007D0000006A
:100F0B00010000000000803F0A06000200000040C4
:100F1B000100000009022200010100E03209040077
:100F2B000001030102000921110100012236000713
:100F3B0005830308000A000009022200010100E0FA
:100F4B003209040000010301020009211101000113
:100F5B002236000705830308000700000902220060
:100F6B00010100E032090400000103010200092124
:100F7B00110100012236000705830308000A000057
:100F8B000A060002000000400100000009074300B0
:100F9B00020104C032090400000102020100052411
:100FAB00001001052401000104240202052406009F
:100FBB00010705820308001009040100020A000062
:100FCB0000070501024000000705810240000000F8
:100FDB0009024300020100C03209040000010202B1
:100FEB000100052400100105240100010424020264
:100FFB0005240600010705820308001009040100FF
:10100B00020A000000070501020002000705810229
:10101B000002000009024300020100C03209040073
:10102B00000102020100052400100105240100014A
:10103B0004240202052406000107058203080010A0
:10104B0009040100020A000000070501024000002C
:10105B00070581024000000005010905A101A1005F
:10106B0005010930093109320933093509340936CB
:10107B0009371581257F7508950881020509190126
:10108B00290815002501950875018102C0C00000D3
:10109B0009211101000122360000000010000000A0
:1010AB0000FF0000000000000000AA55070100002F
:1010BB000101AA55050100007EFF0000FFFFFFFFA5
:1010CB0008000000ECCA0908FF1FFF1F2D202D2D63
:1010DB00202D2D2D2D202D2D2D2D0000000000005D
:1010EB000000000000000000000000AA550B0100EA
:1010FB0000AA5505010000AA550902000000AA55D7
:10110B0003009F0001000000C0120000308A002481
:10111B0000000000088A002400000000B43D0A080B
:10112B00303D0A0800000000995A0708A08601000C
:10113B0004000000000000000000000000000000A0
:10114B000000000000000000000000000000000094
:10115B00000000000000000000000000B43D0A0881
:10116B00BC3D0A0800000000F5C60708E8030000B4
:10117B000400000000000000000000000000000060
:10118B000000000000000000000000000000000054
:10119B00000000000000000000000000C43D0A0831
:1011AB000000000000000000112F00007D00000077
:1011BB00FF00000000000000000000000000000025
:1011CB000000000000000000000000000000000014
:1011DB0000000000000000000000000074B70A08C7
:1011EB000000000000000000452500007D0000000D
:1011FB00FF000000000000000000000000000000E5
:10120B0000000000000000000000000000000000D3
:10121B00000000000000000000000000C4480A08A5
:10122B000000000000000000F10500007D00000040
:10123B00FF000000000000000000000000000000A4
:10124B000000000000000000000000000000000093
:10125B00000000000000000000000000CC3D0A0868
:10126B000000000000000000C9370808E803000078
:10127B000300000000000000000000000000000060
:10128B000000000000000000000000000000000053
:10129B00000000000000000000000000D03D0A0824
:1012AB0000000000000000008DEC06081027000075
:1012BB000300000000000000000000000000000020
:1012CB000000000000000000000000000000000013
:1012DB000000000000000000000000007CB30A08C2
:1012EB0000000000653506087D2208085F760000C7
:1012FB0005000000000000000000000000000000DE
:10130B0000000000000000000000000000000000D2
:10131B0000000000000000000000000018B70A08E1
:10132B000000000000000000254108081027000005
:10133B0001000000000000000000000000000000A1
:10134B000000000000000000000000000000000092
:10135B00000000000000000000000000DC3D0A0857
:10136B000000000000000000FDBF0708E8030000BC
:10137B00050000000000000000000000000000005D
:10138B000000000000000000000000000000000052
:10139B00000000000000000000000000E83D0A080B
:1013AB000000000000000000295F0708204E00002D
:1013BB00030000000000000000000000000000001F
:1013CB000000000000000000000000000000000012
:1013DB00000000000000000000000000F83D0A08BB
:1013EB000000000000000000E95C0708204E000030
:1013FB0003000000000000000000000000000000DF
:10140B0000000000000000000000000000000000D1
:10141B00000000000000000000000000083E0A0869
:10142B00000000000000000065340808400D0300B8
:10143B00030000000000000000000000000000009E
:10144B000000000000000000000000000000000091
:10145B00000000000000000000000000183E0A0819
:10146B000000000000000000B93108081027000040
:10147B000100000000000000000000000000000060
:10148B000000000000000000000000000000000051
:10149B000000000000000000000000005C3D0A0896
:1014AB00000000000000000061B4050810270000D8
:1014BB00030000000000000000000000000000001E
:1014CB000000000000000000000000000000000011
:1014DB00000000000000000000000000203E0A0891
:1014EB000000000000000000C9640608A08601008F
:1014FB0001000000000000000000000000000000E0
:10150B0000000000000000000000000000000000D0
:10151B00000000000000000000000000283E0A0848
:10152B00000000000000000071C5070850C3000058
:10153B00010000000000000000000000000000009F
:10154B000000000000000000000000000000000090
:10155B00000000000000000000000000303E0A0800
:10156B00000000000000000061C10708A861000036
:10157B00010000000000000000000000000000005F
:10158B000000000000000000000000000000000050
:10159B000000000000000000000000003C3E0A08B4
:1015AB00000000000000000015050608A0860100E1
:1015BB00010000000000000000000000000000001F
:1015CB000000000000000000000000000000000010
:1015DB00000000000000000000000000483E0A0868
:1015EB000000000000000000DDF20708A00F000063
:1015FB0001000000000000000000000000000000DF
:10160B0000000000000000000000000000000000CF
:10161B00000000000000000000000000543E0A081B
:10162B00000000000000000045A305081027000083
:10163B00010000000000000000000000000000009E
:10164B00000000000000000000000000000000008F
:10165B00000000000000000000000000603E0A08CF
:10166B000000000000000000F18505081A41000091
:10167B00010000000000000000000000000000005E
:10168B00000000000000000000000000000000004F
:10169B00000000000000000000000000643E0A088B
:1016AB000000000000000000590C05081027000086
:1016BB00010000000000000000000000000000001E
:1016CB00000000000000000000000000000000000F
:1016DB00000000000000000000000000443D0A086C
:1016EB000000000000000000F90E060850C30000C7
:1016FB0001000000000000000000000000000000DE
:10170B0000000000000000000000000000000000CE
:10171B00000000000000000000000000703E0A08FE
:10172B000000000000000000051C0508400D030030
:10173B00000000000000000000000000000000009E
:10174B00000000000000000000000000000000008E
:10175B00000000000000000000000000783E0A08B6
:10176B000000000000000000B9BF0708400D030097
:10177B00000000000000000000000000000000005E
:10178B00000000000000000000000000000000004E
:10179B00000000000000000000000000803E0A086E
:1017AB00000000000000000009F0050850C3000015
:1017BB00030000000000000000000000000000001B
:1017CB00000000000000000000000000000000000E
:1017DB000000000000000000000000008C3E0A0822
:1017EB0000000000000000001575070840420F00C4
:1017FB0000000000000000000000000000000000DE
:10180B0000000000000000000000000000000000CD
:10181B00000000000000000000000000983E0A08D5
:10182B00000000000000000039C1070850C3000091
:10183B00000000000000000000000000000000009D
:10184B00000000000000000000000000000000008D
:10185B00000000000000000000000000010000007C
:10186B0000000100E001010049980508000000009C
:10187B0000000000F8CC0908FF0800000000000081
:10188B000000000000000000B0E6090800000000A6
:10189B00000000000000000068E7090800000000DD
:1018AB00000000000000000014E709080000000021
:1018BB0000000000B9CF0508D99600243DE20508C9
:1018CB00000000000000000040E60908010101FFD4
:1018DB00FFFFFFFFF9FD05080000000000000000FE
:1018EB003CE8090821010608000000000000000088
:1018FB00F4E709082D202D2D202D2D2D2D202D2DFC
:10190B002D0000000000000000000000000000009F
:10191B0000000000FFFFFFFF01000000FA000000C5
:10192B000100000001000000E89200240000F40117
:10193B0001000000E69200240000F4010100000009
:10194B00E49200240000F40101000000E292002464
:10195B000000F40101000000E09200240000F401FB
:10196B0001000000DE9200240000F40101000000E1
:10197B00DC9200240000F4010100000051A00508D6
:10198B0015A005080000000004D30908CC92002420
:10199B0005320100DA9200246400F401010000001A
:1019AB00D89200246400C40901000000CA920024EC
:1019BB00E803D00701000000C8920024E803D00719
:1019CB0001000000C6920024E803D00701000000CC
:1019DB00C49200241E00B80B01000000D292002418
:1019EB0005000F0001000000D492002403000A0040
:1019FB0001000000C29200241E00F401010000004F
:101A0B00D69200240200000090D30908C092002453
:101A1B001400640001000000CE9200243200E803A1
:101A2B0001000000BE9200240000C800010000006D
:101A3B00C991002400C80100C89100240050010086
:101A4B00C7910024005A0100C59100240200000038
:101A5B009CD3090814400A081C400A085A5A00244F
:101A6B000100C40900000000585A00240100C409F9
:101A7B0000000000565A00240100C40900000000B9
:101A8B00545A00240100C40900000000505A0024DD
:101A9B000100C40900000000525A00240100C409CF
:101AAB00000000004E5A00240100C4090000000091
:101ABB004C5A00240100C40900000000738F00245D
:101ACB0000C80100728F002400C80100708F002431
:101ADB000000FFFF0A0000006E8F00240100C80009
:101AEB00010000006C8F00243200307532000000C2
:101AFB006A8F002405820500688F002405002C01E5
:101B0B0005000000678F0024055A0500648F002430
:101B1B0000FF0100668F002402000000540E002419
:101B2B00628F002403000000BCC70908638F0024E8
:101B3B0000FF0100658F002402000000540E0024FA
:101B4B00618F002403000000BCC70908A59F05088E
:101B5B00359F050800000000A8D309080093002456
:101B6B00EE02CA0801000000FE92002400C801002A
:101B7B0064000000FD92002400C801006400000016
:101B8B00FC92002402000000B4D409084E8F0024FC
:101B9B000000803E050000004C8F002480C1803E79
:101BAB0005000000468F00240083007D0500000027
:101BBB00448F002480C1803E050000003F8F00242D
:101BCB0000FF0100388F00246400F40101000000C5
:101BDB00368F002404000000C0D40908358F002480
:101BEB0002000000D4D40908F98F00240D00000076
:101BFB00E0D40908F68F002400640100F48F002460
:101C0B00320010270A000000F28F00240D000000A4
:101C1B00E0D40908F18F00240D000000E0D409087E
:101C2B00F08F00240200000018D509080693002449
:101C3B003E00000024D50908049300240100FF7F17
:101C4B0001000000039300240200000020D60908C5
:101C5B00FB8F00240300000030D60908FA8F002404
:101C6B000300000030D60908B6910024000A0100D9
:101C7B00B49100240000E80301000000B29100249D
:101C8B000000E80301000000B09100240000E8030D
:101C9B0001000000AE9100240000E80301000000E9
:101CAB00A69100240000E80301000000AC91002481
:101CBB000000E80301000000AA9100240000E803E3
:101CCB0001000000A891002400140100C49100241D
:101CDB000200000040D60908C29100240000F40164
:101CEB0001000000C09100240000F401010000007D
:101CFB00BE9100240000F40101000000BC910024FF
:101D0B000000F40101000000BA9100240000A00FB4
:101D1B0001000000B89100240000A00F010000009A
:101D2B00AB92002419640100AA9200240200000067
:101D3B004CD60908A8920024E803D0070A0000003B
:101D4B00A6920024006401000A0000009B9200246C
:101D5B00006401009A92002400640100A292002406
:101D6B00006401000A000000A1920024006401003D
:101D7B000A000000A0920024006401000A00000089
:101D8B00A592002400FF01000A000000A492002489
:101D9B0000FF01000A000000A392002400FF0100D5
:101DAB000A0000009F92002401FF01000A000000BE
:101DBB009E92002401FF01000A0000009D92002466
:101DCB0001FF01000A000000049000240000F40150
:101DDB0001000000029000240000A00F0100000091
:101DEB00009000240000A00F01000000FE8F0024D3
:101DFB000000A00F01000000FC8F00240000A00FCA
:101E0B00010000002997002400C801002897002436
:101E1B00006401002797002400640100269700242A
:101E2B00006401002597002400640100249700241E
:101E3B00FF08010023970024016401009D9E050803
:101E4B00619E05080000000058D609082C97002455
:101E5B00013201002B97002401000000C8D60908AD
:101E6B002A97002404000000D0D6090822970024EA
:101E7B0000640100209700241400E8030100000017
:101E8B001E970024E80330750A0000001C970024FD
:101E9B0000C801001B97002400C801001A970024FA
:101EAB0000C8010019970024003201002E9700246E
:101EBB00004B01002D97002404000000E4D6090814
:101ECB0018970024006401000A0000003C970024CE
:101EDB000000D007010000003797002400C8010064
:101EEB003697002400C801003597002400C8010074
:101EFB003A9700240000D00701000000349700241B
:101F0B0000C801003397002400C801003297002459
:101F1B0000C80100389700240000D0070100000022
:101F2B003197002400C801003097002400C801003D
:101F3B002F97002400C80100499C0508319C050817
:101F4B0000000000F8D60908ED8F0024005A0100AC
:101F5B00EC8F002400C80100EA8F0024E803D007AF
:101F6B00010000000000000000000000F9CF050890
:101F7B0094D709084D4154454B4837343300000082
:101F8B00608F0024000301005F8F00240003010019
:101F9B006D9B0508219B050800000000E8D7090888
:101FAB00E19A0508999A05080000000084D80908F1
:101FBB00B99B050821E205080000000004D90908B7
:101FCB00508F0024010301002DA1050801A1050874
:101FDB00000000005CDC09081D9A0508D199050872
:101FEB0000000000CCDC0908599C050879E30508C2
:101FFB000000000068DD0908A5E5050859A10508E2
:10200B000000000010DE0908B59C05080000000068
:10201B000000000090DE0908919D0508399D050818
:10202B0000000000F4DE0908259E0508E99D05085F
:10203B00000000009CDF0908A5250608D99E0508AD
:10204B000000000028E00908BD92002401060100F1
:10205B00FD9C0508C99C05080000000024E1090847
:10206B00D724060849E405080000000094E109089C
:10207B00F125060811E5050800000000E4E2090857
:10208B00BC92002401030100019C0508D19B0508AB
:10209B0000000000B8E309084D2606080000000008
:1020AB00000000001CE40908699A050809E205080C
:1020BB00000000009CE40908000000000000000084
:1020CB000000000028E509080D9F050889E50508B3
:1020DB000000000098E50908000000000000000067
:1020EB0000000000B0E70908488400249CFF2C0185
:1020FB0000000000A4990024E0150C17000000005C
:10210B006D96002402000000E8E70908308F0024D8
:10211B0088136F1701000000328F002488136F178C
:10212B00000000009E5A0024000000000000000088
:10213B009C5A002400000000000000009A5A002462
:10214B000000000000000000985A0024000000006E
:10215B0000000000965A0024000000000000000060
:10216B00945A002400000000000000000805002421
:10217B000000000000000000B88E002403000000E7
:10218B00D8E80908288F002488136F170100000076
:10219B009284002488136F17000000001199050822
:1021AB000000000000000000E8E809086E9600241B
:1021BB00010000003CE909089484002401000000A0
:1021CB0048E909088A8400240200000050E9090844
:1021DB000000000000000000000000005CE909089E
:1021EB00F99805080000000000000000F8E9090854
:1021FB000000000000000000000000004CEA09088D
:10220B00000000000000000000000000BCEA09080C
:10221B00348F002402000000F4EA09088E840024A5
:10222B00E0150C1700000000D0A2002424A300240A
:10223B0001D601FF010000000001010100000000B8
:10224B00FFFFFFFF0000803F0000000000000000C8
:10225B000000000000000000000000000000000073
:10226B000000000000000000000000000000803FA4
:10227B000000000000000000000000000000803F94
:10228B000000000000000000000000000000803F84
:10229B000000000000000000000000000100000032
:1022AB000000FA430000FA430000803FFFFFFFFFEE
:1022BB00FF000000C9330808000000000000000008
:1022CB00000000000000000048BC002408000000D3
:1022DB000000000038BC002408000000685E0C0001
:1022EB0002010000A00F0000B80B00000102FFFF6D
:1022FB00010000002D08040811080408CD0704088C
:10230B0000000000C1070408AD0704089907040882
:10231B0000000000000000000000000000000000B2
:10232B008907040800000000790704082D09040838
:10233B0021090408E9080408FD080408A108040899
:10234B008D08040879080408DD0D040875070408D6
:10235B00F1060408510D04080010000010000240A3
:10236B0000000000001100002800024000000000E7
:10237B0000120000400002400000000000130000AB
:10238B0058000240000000000014000070000240E2
:10239B000000000000150000880002400000000053
:1023AB0000160000A0000240000000000017000013
:1023BB00B8000240000000000020000010040240A2
:1023CB000000000000210000280402400000000073
:1023DB000022000040040240000000000023000027
:1023EB00580402400000000000240000700402406A
:1023FB0000000000002500008804024000000000DF
:10240B0000260000A004024000000000002700008E
:10241B00B804024000000000FFFF000070B30A0880
:10242B0000000802050306000000000078B30A084C
:10243B0001000802050406000000000070620A0893
:10244B000200FE01011003000000000074430A08A3
:10245B0003001402000300000000000080B30A0810
:10246B0004001F02020008000000000088B30A08E5
:10247B0005001F02020108000000000090B30A08CB
:10248B000600250201001100FE810300FFFFFFFF84
:10249B00FFFF0100F40100000000000019B5040863
:1024AB00A9D8040899A4040835DA0408BDB50408B2
:1024BB0005990408F1980408E998040810360A08ED
:1024CB00E0010400E001020805000000000000002C
:1024DB0090010400900102080500000000C00000FC
:1024EB0000000000000000000F06000000010000CB
:1024FB0000000030F4220030000300010100000056
:10250B00E0D10024E0E700240003000001000000FC
:10251B00010000001819002400000000000000005A
:10252B0000000000000000000000000000000000A0
:10253B000000000000000000000000000000000090
:10254B000000000000000000000000000000000080
:10255B000000000000000000000000000000000070
:10256B000000000000000000000000000000000060
:08257B00000000000000000058
:102583000100000001000000041B00200000000007
:042593002000000024
:020000040804EE
:100000002DE9F04F022389468A462DED108B99B0D9
:10001000DFEDCABA14930346169004331592179372
:100020004FEADA06169DDDF85CC04FEACA0305EB1D
:1000300046111396F0004FF0000B01EB0614370148
:100040000390A6EB86020194049706EB460E04EBA0
:10005000C202041D381D06EB86072C44C6EBC608F9
:1000600002972844029D02EB46174FEAC808ED00AC
:1000700001EBC60602954FEA0E1505954FEACE052F
:100080000695139D4FEA451E019D95ED007AD344D8
:1000900092ED005AD7ED004AD945D1ED006A50EDF6
:1000A000013A35EE241AD6ED002A1CED016A73EEF2
:1000B000875A54ED017A33EEC73A36EE264A77EE88
:1000C000A21A36EE666A77EEE27A74EE256A71EE6F
:1000D000812A77EE633A37EEC57A36EEA22A77EEBA
:1000E000E47A76EEE26A0CED012A37EE247A77EEB6
:1000F000857AD1ED018AC1ED006A74EE655A96EDFC
:10010000015AB0EE460A94ED004AA7EE2B6AD2EDF2
:10011000010AE7EEAB3A74EE456AD7ED012AA7EE85
:100120006B0A9CED007AD5ED014A34EE054A37EEB4
:10013000689A90ED005A36EEE02A76EEE26A30EEEA
:10014000A28A32EE222A76EEA06AF0EE492A75EEF5
:10015000640A37EE287A75EE249AE2EE6B2A74EE82
:10016000C54AF0EE608AB0EE40AAE6EEAB4AE6EE93
:10017000AB8AA6EEEBAAF0EE496AB0EE629A37EED1
:10018000695AE2EE2B6AB0EE432A74EE08AAA7EE93
:10019000EB9AA7EEAB2A77EE297A35EE617A75EE07
:1001A000C89A35EE415A75EEC45A37EEAABA77EEC0
:1001B000EA7A37EE011A8CED00BA36EE287AC1EDF4
:1001C000017A39EE844A76EEC27A194475EE885A7D
:1001D0009C4435EE215A00ED014A70EE8A0A70EE19
:1001E000244AC5ED005A36EE686A80ED001A72EEB8
:1001F000A33A85ED015A33EE093A04ED017A72EE25
:10020000266A87ED006A1D44C6ED000A1844C2ED57
:10021000004AC4ED007A1C44C7ED016A1F44C6EDD4
:10022000013A1E4482ED013A1A443FF62EAF139A6A
:10023000072A40F2C681039A0EF1080E169F08F1B4
:1002400008000832029E059D4FF0000894463A4689
:10025000083608357244069C0499D346109207EB81
:100260000C0208340C310F92BA190E927A190D92C1
:100270003A190C923A180B927A18099207F10C026B
:100280000A9201220892149ADDF824C09044159A2B
:100290000A9F02EBC8020B9EA8EB880E0C9D02EB96
:1002A000C80192ED00BA0D9C01EBC802D1ED00AA85
:1002B0000E9802EBC80192ED00AA01EBC802D1ED45
:1002C000009A02EBC80192ED009A01EBC802D1ED51
:1002D000008A0F9902EB0E1E92ED008A109A0EEB27
:1002E000C80ADEED017A1192CDED047A0AEBC8025C
:1002F000DAED017A02EBC80A1291CDED057AD2ED62
:10030000017A0AEBC802DDF820E0CDED017ADAEDE2
:10031000017A02EBC80ACDED067AD2ED017A0AEB3A
:10032000C802CDED027ADAED017ACDED077AD2ED91
:10033000017ADDE91121CDED037A01E0F304353FC7
:1003400017ED017ADE44D2ED007A94ED005AF145C2
:10035000D5ED006A37EE274AD0ED004A77EE677A8E
:100360001CED016A96ED007A91ED001A76EE055AC1
:1003700036EE872A97ED00DA71EE24EA76EE453AFA
:1003800074EE252A31EE641A35EE466A3EEE825A44
:1003900074EE655A31EE664A72EE854A31EE471ABE
:1003A000B0EE67CA47ED014A34EE077AD1ED014A53
:1003B00031EE261AD0ED016A72EEC52A95ED014A9A
:1003C000A7EE6BCA74EEE60A96ED010AE7EE2B7A09
:1003D00092ED017A94ED015A74EEA64A3DEE473A49
:1003E000DCED006A70EEC4CA70EEC00AB0EE43EAFB
:1003F0007CEE80CA74EE001A70EE840AACEEEBEA72
:1004000036EEC54A3DEE077AB0EE63DA36EE850A7F
:10041000ACEEAB3AF0EE4EDAA1EE2BDAA1EE2B6A9F
:10042000E1EE6BDA75EE666AB0EE441AF0EE4CCA95
:1004300037EE405AA0EEAB1AE0EEEBCAE0EEAB6A44
:1004400037EE007A74EEA10A35EEE1FA75EEE45A61
:1004500075EE6EFA37EE600A71EEA55ADDED061AFA
:1004600035EE425A7FEE244A3FEE822A22EEE1FA2E
:1004700061EE80FADDED051A3EEE855A3EEE066A23
:1004800073EEAD3A21EE82EA73EE4DDA3DEE033AB9
:1004900024EEE1DADDED071A34EE2C4A7CEE266A12
:1004A00061EE85CA25EEE1CADDED041A77EE81EA38
:1004B00077EEC17AE9EEA2FADDED032AA9EE80FA21
:1004C0009DED030AAAEEA4EADDED014AAAEE82DA66
:1004D0009DED012AE8EEA5CADDED025AA8EE85CA17
:1004E0009DED025A21EEAD1A62EE832A6EEEE11AFC
:1004F00027EEC00A64EEA34A26EEC22A65EE865AAB
:1005000024EE455AABEE2E1AEBEE2D1AE8EE272A12
:10051000A8EE030AEAEE264AAAEE232AE9EE045AD6
:10052000A9EE065A37EE207A87ED007A1F44C2ED15
:1005300000FA82ED01FA1A440CED01EA8CED00DAC2
:100540009C44C4ED00CA84ED01CA1C4481ED001A2C
:10055000C1ED011A1944C6ED002A86ED010A1E44B8
:10056000C0ED005A80ED015A1844C5ED004A85EDF2
:10057000012A1D443FF6E4AE1099089A0831013271
:1005800010910F99089208310F910E9908310E9130
:100590000D9908310D910C9908310C910B99083186
:1005A0000B910A9908310A91099908310991139917
:1005B00091427FF468AE149B8A46DB009BB2149391
:1005C0002EE519B0BDEC108BBDE8F08F124B30B4A6
:1005D0001D686B6A28B943EA01430020AB6230BC56
:1005E0007047AC6A013803EB14440BD0002303F1CD
:1005F0004002013305EB8202DBB25268834204EB16
:100600001244F4D3403044EA014405EB80004460D6
:10061000002030BC704700BF78190024037870B404
:100620002BB30246C0F10105531912F8014FDBB29A
:10063000002CF9D101335B000E4C03220B8084F8AF
:10064000083484F80924017879B1022300265A1C61
:10065000E518023354FA82F285F80814DBB282F806
:10066000086410F8011F0029F1D170BC7047022303
:10067000E2E700BF7819002430B5EFF31181802341
:1006800083F312880A4AD2F80835D2F80C45D2F81A
:100690000805D2F80C55CAB282F31188013BA84272
:1006A00094BF4FF4006000201B1B184430BD00BFF6
:1006B00078190024012380F851307047014BD3F89A
:1006C000100570477819002401207047024BC3F8C9
:1006D0001425C3F81815704778190024024BC3F885
:1006E0001C25C3F8201570477819002470477047FF
:1006F000212870B505D0222829D0202810D000202C
:1007000070BD0029FBD0072AF9D1184B18791C6855
:100710005A799B79087100200C604A718B7170BD09
:100720000029ECD0072AEAD11148104B0C680E7949
:100730004D79D0F8182589791C601E715D71997109
:10074000002ADCD02146D0F814059047D7E70029CD
:10075000D5D0022AD3D1064AD2F82035002BCED0EC
:100760000988D2F81C059847C9E700BF000000249B
:10077000781900240020704703460A2201481A8095
:10078000704700BF080000240346642201481A8015
:10079000704700BF14000024012901D000207047D9
:1007A000014BD3F89030184700000024012901D0F4
:1007B00009F0BAB8014BD3F88C3018470000002478
:1007C000014BD3F8883018470000002410B40B7890
:1007D0000A46044603F00303012B05D0022B0BD07D
:1007E00000205DF8044B70478B8843B920461146C2
:1007F0005DF8044B0CF0CEBC8B88832BF6D0034BFA
:100800005DF8044BD3F88030184700BF0000002487
:1008100038B5054B04460D46DB6F98472946204600
:1008200009F058FE002038BD0000002438B5054B03
:1008300004460D469B6F9847294620460CF080FEE3
:10084000002038BD00000024F0B4002452004E1CEB
:100850002746030FB0F1204F4FEA001003F1300597
:1008600003F1370334BF0D550B5537550234A242FF
:10087000EFD1F0BC704700BF024808B5FFF7CEFECD
:10088000014808BD70360A08801D0024024808B5DA
:10089000FFF7C4FE014808BD80360A08801D002409
:1008A0000B481A220B4B00681B680A80C01801D144
:1008B00009487047094B0822094910B51C68FFF721
:1008C000C3FF042207492046FFF7BEFF024810BDC0
:1008D00000E8F11F08E8F11FB000002404E8F11F50
:1008E000B2000024C2000024024808B5FFF796FEBB
:1008F000014808BD8C360A08801D002408B520B9BF
:100900000448FFF78BFE044808BD0448FFF786FE45
:10091000014808BD98360A08801D0024BC360A0824
:10092000042301480B807047CC000024074A084B81
:1009300010B4122492F8240503F114020C8001284B
:100940000CBF184610465DF8044B70477819002418
:10095000D0000024D8B18268104B1AB1072283F866
:100960002A25704793F828050421C3F83425032865
:10097000C3F8382583F83C250CBF80224FF48072E1
:1009800083F82A15C3F82C25C3F830257047034B8C
:10099000012283F8102783F829257047781900244D
:1009A00038B5544C00234FF4F072202104F28470C7
:1009B00084F880375AF05EFE04F664104FF4F0724B
:1009C00020215AF057FE94F8450B10B194F8463B9D
:1009D0000BB9002038BD44F0BDFDC4F8540B28B15C
:1009E00083790BB1412BF4D12323C3800D2144F033
:1009F000A3FFD4F8540B45F0C9F894F8460B01381E
:100A000040B245F055FF02231021C4F84C0B84F886
:100A1000483B4FF075FF0821D4F84C0B4FF070FFA6
:100A2000D4F8540B45F0ACF8FF218C2050F046FD73
:100A30000546D4F8540B45F0A9F80421D4F84C0B22
:100A40004FF05EFF1B2D05D0D4F8540B202144F04D
:100A500073FFBEE70122D4F8543B84F880270BB122
:100A60002322DA800821D4F84C0B4FF049FFD4F848
:100A7000540B45F085F840210A2050F01FFDFF215E
:100A80008A2050F01BFDD4F8540B45F07FF8D4F8C1
:100A90004C0B04214FF034FFD4F84C0B08214FF0DD
:100AA0002FFF0821D4F84C0B4FF02AFFD4F8540B39
:100AB00045F066F80221002050F000FDD4F8540BF8
:100AC00045F064F8D4F84C0B04214FF019FF94F86A
:100AD0005D2B94F85E3B0120C2F1200294F85C1B70
:100AE000C3F1100384F85F2B84F8603B84F8581B33
:100AF00038BD00BF781900240F4B07B5D3F8F82094
:100B00005208B2FBF1F3B3F5803F02D3012AF7D8C4
:100B1000F9E799B2019056F023F8084941F2D03331
:100B2000074A0198CA5001F59E510022103103B0C6
:100B30005DF804EB55F0BABE0000002478190024DB
:100B40008D0306082DE9F0478846002951D0461844
:100B5000451EDFF8A4908024013EDFF8A0A0EFF34B
:100B6000118184F31288D9F80825C9B2D9F80C0587
:100B7000D9F80835D9F80CC581F31188634594BFBD
:100B80004FF400630023121A1344012B1AD10120E1
:100B900042F0BAF8EFF3118184F31288D9F80825EE
:100BA000C9B2D9F80C05D9F80835D9F80C7581F314
:100BB0001188BB4294BF4FF400630023121A134400
:100BC000012BE4D0EFF3118284F31288D9F80C35AD
:100BD000D2B215F8011F534483F8E012D9F80C354E
:100BE0000133C3F30A03C9F80C3582F31188B54207
:100BF000B5D14046BDE8F08778190024702A00245A
:100C0000F8B5002390F8505080F85030CDB10F4E19
:100C100096F87C2D032A16D1D6F8B47D00F13C0459
:100C200029462046FFF78EFFD6F8B43D2D1A04441E
:100C3000DB1B322B01D8002DF2D1B5FA85F040092B
:100C4000F8BD0120FCE71846FAE700BF702A00242F
:100C5000002280F85120D3E790F85020531C024422
:100C6000DBB280F8503082F83C1090F851200AB185
:100C7000132B00D9C4E77047F8B50B4E0D46144648
:100C800096F87C3D032B0ED1D6F8B47D002C0ADDFE
:100C900021462846FFF756FFD6F8B43D241A0544EE
:100CA000DB1B322BF2D9F8BD702A00240F49D1F892
:100CB000983D10B5B3B191F8F04AD3F8042244B18D
:100CC00000244023D1F8B00D01210CF0E9FA2046B0
:100CD00010BD4FF40073D1F8B00D01210CF0E0FA13
:100CE000204610BD0224204610BD00BF702A0024FB
:100CF00010B50C4CD4F8103563B10B49013BD1F859
:100D0000B82DC4F8103512F8014BC1F8B82D047095
:100D100013B10123184610BDFFF7C8FF0123184681
:100D200010BD00BF78190024702A002413B5074CA9
:100D3000D4F8B83D03B9FEE701A8FFF7D9FF0028B2
:100D4000F6D09DF8040002B010BD00BF702A002448
:100D500010B50B68064C074AC4F81035C2F8B80D38
:100D60000BB1002010BDFFF7A1FF002010BD00BF98
:100D700078190024702A0024154BDB68C3F3022382
:100D800010B4C3F107041A1D042C28BF0424062A3A
:100D90004FF0FF328CBF033B0023A240002821EA22
:100DA000020101FA03F108DB09010A4BC9B203444D
:100DB00083F800135DF8044B704700F00F00090141
:100DC000054BC9B2034419765DF8044B704700BF68
:100DD00000ED00E000E100E0FCEC00E02A4B41F215
:100DE00087302A490022D3F8F830A1FB03132849A1
:100DF000DB0C10B5274C013B82B0C4F8C80D04F6DB
:100E0000BC50C4F8BC1DC4F8CC2DC4F8C42DC4F823
:100E1000C03D12F0A3FE204B06213720D3F8E82076
:100E200042F02002C3F8E820D3F8E83003F02003B2
:100E30000193019BFFF7A0FFD4F8BC3D4FF40000E5
:100E40001649174A4860D96841F00101D96099688C
:100E50000A40062A06D0B2F5803F03D01A6842F055
:100E600001021A600F490020D4F8983D0E4A01F69D
:100E70001C34C3F81002C2F82005C2F81805C3E9F3
:100E8000814102B010BD00BF0000002483DE1B437F
:100E900000140040702A00240044025800E100E0E1
:100EA00007000100502D002478190024014BD86060
:100EB000704700BF50400058012008B5FFF7F6FF0B
:100EC00072B655F03FFF00BF03689B0AA3F580137D
:100ED000522B00D970470D4A70B5D45C84B00D2CEC
:100EE00012D800294FF0000309494FF0010514BF43
:100EF0001E460226427901EB84106946CDE9006561
:100F0000CDE902330FF050FB04B070BDE8B809081A
:100F10006C4000240D4B4FF6FF71D3F8F82010B54C
:100F20000446520855F01CFE00212046FFF7CCFF76
:100F30000749084A41F2D4332046CA5001F59E5170
:100F400000221431BDE8104055F0B0BC0000002470
:100F5000781900249DD605084309012200F01F00DE
:100F60008AB0023B02FA00F0082B11D8DFE803F048
:100F7000665A4E42362A1E120500364BD3F8F4202C
:100F80000243C3F8F420D3F8F42010400190019BF1
:100F90000AB070472F4BD3F8E0200243C3F8E0209B
:100FA000D3F8E02010400590059BF1E7294BD3F8DA
:100FB000E4200243C3F8E420D3F8E4201040029078
:100FC000029BE5E7234BD3F8D4200243C3F8D42097
:100FD000D3F8D42010400690069BD9E71D4BD3F8D8
:100FE000DC200243C3F8DC20D3F8DC20104008905A
:100FF000089BCDE7174BD3F8D8200243C3F8D8207D
:10100000D3F8D82010400990099BC1E7114BD3F8C1
:10101000EC200243C3F8EC20D3F8EC2010400390FE
:10102000039BB5E70B4BD3F8E8200243C3F8E82055
:10103000D3F8E82010400490049BA9E7054BD3F8AF
:10104000F0200243C3F8F020D3F8F02010400790BE
:10105000079B9DE7004402582DE9F04FDFF8DC8044
:101060002A4D44462DED068B8DB0CDE90A01049240
:101070000FCD0FC40FCD0FC4254B95E8070093F893
:10108000C63884E80700042B00F2A981DFE813F0DA
:10109000D801A701A2010500E6019FED1E8ADFED40
:1010A0001E9A1E4A1E4B04981E49002818BF13465C
:1010B0001D4AC8E9062139EE887ADFED1C7AF5EE83
:1010C000006ADFF87CB04FF0000928EE278AB0EE06
:1010D000679ADA4686EE87AAC8F82430DFED148ACC
:1010E000CB46144B05930B9B5B4500F06D81059A35
:1010F0000BF1010312F8017BDEB206930592002F7B
:1011000000F0D88100230C4820E000BF3CB909085A
:10111000683B0024ACC5A737ACC5A736E144080836
:10112000D1550708D15A0708ED4408086F12833AD1
:1011300000007A4433440024484400241400002072
:10114000480000200133152B00F0B48103EB43026B
:101150004FEA4309815CB942F4D1C74B1A4492F873
:10116000E118002900F0AE8138463DF0FDFB04682F
:1011700005460390204655F075FD69793DF032FC37
:1011800002780892002A40F095813D09BA4B07F099
:101190000F02013D4B444FF00309062D83F82169EE
:1011A00083F8209900F24381B44B029303EB45038B
:1011B000B3F8800040FA02F313F0010300F03D8120
:1011C0000124AF4F04FA02F3013B184056F0C0FF70
:1011D000029BAC4A1D4495F890100144039807EB1C
:1011E000C105EE7185F8069057F83130CAF81450F1
:1011F0001A44029B007A920A079003EB4202B2F86B
:101200009800FFF7A9FEAE8857F83110002E39D0AC
:10121000089BA646CDE908BADDF81CA00EFA03F536
:101220002E4229D0DC0803F007024FF00F0C5800C3
:1012300001EB84044FF0020B9200276A0CFA02FCC7
:101240000AFA02F227EA0C0C09FA00F70BFA00F08E
:1012500042EA0C0222620A6822EA0702104308608E
:101260008A6822EA07028A604A6822EA05054D6018
:10127000CA6822EA0707CF60013336FA03F2CDD1FC
:10128000DDE908BA039B1C68049B002B00F0BD80BD
:10129000794BB3F8C43807EE903AF8EEE77AFCEEF3
:1012A000E77A17EE905A784B9C420FD003F5806393
:1012B0009C420BD0754A03F580439C4218BF944270
:1012C00004D003F580639C4240F0AA8012F07EFFB8
:1012D0006F4BD969C1F302216D4A4FF6FF73126952
:1012E000C2F3C03241EAC201029A0A44049992F858
:1012F000AC2000FB02F0B0FBF5F21A44120CB0FB7C
:10130000F2F2002970D05C49B2FBF5F591F8C618ED
:10131000ABB204296ED007EE902AF8EE676A66EE4B
:10132000887A28EEE77A544991F8C708A6EEA97A98
:101330000A990190504600910399CAED027A8AED0C
:10134000037A35F0ABFDBBF1000F65DDDAF8043050
:10135000D8F83820934261D0BBF1010F5CD0D8F8A7
:10136000502093425AD0BBF1020F55D0D8F86820D4
:10137000934253D0BBF1030F4ED0D8F88020934254
:101380004CD0BBF1040F47D0D8F89820934245D0F9
:10139000BBF1050F40D0D8F8B02093423ED0BBF14E
:1013A000060F39D0D8F8C820D31A18BF0123DDF8AA
:1013B00018B001228AF810300AF1180ABBF1080FA0
:1013C0000AF8072C7FF48FAE32480DB0BDEC068BC7
:1013D000BDE8F08F9FED308AF0EE489A61E69FED10
:1013E0002F8AF0EE489A5CE623491D4691F8C6180C
:1013F000042990D107EE905A07EE102AF8EE677A8A
:10140000F8EE476A67EE897A8BE7FAFE4A7AFCEED5
:10141000E77A17EE905A46E70123C8E70023C6E7AC
:1014200012F0ECFE1A4BD969C1F3021154E7089B84
:10143000CAF81430114B029326E7CAF8143023E798
:101440000023174A01219FED178A0A93164BF0EEED
:10145000489A0491C8E90632144B2CE60023104A3E
:1014600001219FED138A0A930F4BF0EE489A0491E5
:10147000C8E906320D4B1EE6683B0024E8B80908AF
:10148000B44400240000FEA70000014000400140D9
:101490000044025814000020282930386F12033904
:1014A000D15A07086F12833AED440808E14408084E
:1014B00000000000044A0020044BC8F81C20C8F8B3
:1014C000243082E70B68FFDEBD580708E1440808B6
:1014D000002850D0284A2DE9F84F0446274B0068D1
:1014E00003449B0A02EB4303B3F89800FFF734FD73
:1014F000B4F804C02268BCF1000F3AD000204FF0CD
:10150000010B4FF00F0A4FF0030900F007030BFA2D
:1015100000F645004FF0020EC7081CEA060F4FEA1E
:10152000830309FA05F402EB87070EFA05F500F1CB
:1015300001000AFA03FE01FA03F317D0D7F820805E
:1015400028EA0E0E43EA0E033B62136823EA040303
:101550002B431360956825EA04059560536823EAD8
:1015600006035360D36823EA0403D3603CFA00F314
:10157000CBD1BDE8F88F7047E8B809080000FEA796
:1015800000284FD0284A2DE9F84F0446274B006821
:1015900003449B0A02EB4303B3F89800FFF7DCFC1B
:1015A000B4F804C02268BCF1000F39D000204FF01D
:1015B000010B4FF00F0A4FF0030900F007030BFA7D
:1015C00000F645004FF0020EC7081CEA060F4FEA6E
:1015D000830309FA05F402EB87070EFA05F500F11B
:1015E00001000AFA03FE01FA03F316D0D7F82080AF
:1015F00028EA0E0E43EA0E033B62136823EA040353
:101600002B431360956825439560536823EA0603CE
:101610005360D36823EA0403D3603CFA00F3CCD1CF
:10162000BDE8F88F704700BFE8B809080000FEA7C2
:10163000004870471445002470B4204D06460468E5
:10164000E36931EA030323D0D5F8CC3C9B1AB3F10C
:10165000007F23681FD25807F2D5E3691B05EFD539
:101660004FF400622023002103202262226822F42A
:10167000D0722260A26822F00102A260C6F8803017
:1016800086F87C10C6F88430C6F8883070BC704785
:10169000002070BC704723F4D07320220021032067
:1016A0002360A36823F00103A360C6F8802086F8B6
:1016B0007C10C6F8842070BC704700BF683B0024D3
:1016C000F8B5044690F88000012800F0AB80B94ED0
:1016D00001272068D6F8CCCC94F8815084F880702B
:1016E000012D5FFA85FE67680BD0B7F5800F40F0DB
:1016F0008F80A568002D40F08B80BEF1040F40F074
:101700008780002B18BF002A00F08780002900F096
:10171000848094F88150042D02D0052584F88150EE
:101720004FF0000E6266A44DB7F5800FC4F884E058
:10173000A4F86A30A4F862304268A4F8683005EA78
:101740000205E165A4F8603045EA0305C4E91CEE32
:101750004560026842F00102026003D1026842F46F
:1017600000720260E2680F2A60D91A4648F2080740
:10177000416989070ED56BB1E16D51F8043B0362F5
:10178000B4F86230E165013B9BB2A4F86230B4F872
:1017900062309BB2416943EA02053942ADB211D0D1
:1017A000002A41D0056BB4F86A20616E013A41F815
:1017B000045B92B26166A4F86A20B4F86A2092B21F
:1017C00042EA0305002DD3D1D6F8CC3CA3EB0C03A1
:1017D000092B70D843691B070BD4D6F8CC3CA3EB7C
:1017E0000C03092BF6D9D4F8843043F02003C4F855
:1017F000843020460CF006FB0122002384F881206F
:10180000D4F8840084F88030C01A18BF0120F8BDD5
:101810000023022084F88030F8BD0023012084F8E2
:101820008030F8BD0220F8BD1D46CBE7072A52D80C
:10183000024619465569AD0715D5A3B1032B40F2F1
:10184000CC80E36B402B40F2DD80E56D55F8043B26
:101850001362B4F86230E565043B9BB2A4F86230D1
:10186000B4F862309BB2556915F4604F12D089B15B
:101870005169090440F18980156BB4F86A20616EE2
:10188000043A41F8045B92B26166A4F86A20B4F8A5
:101890006A1089B2D6F8CC2CA2EB0C02092A54D8D3
:1018A00043EA010292B2002A00F0C780226855691B
:1018B000AD07D8D5C1E720460CF0A4FAD4F884309F
:1018C000012284F8805043F480731046C4F88430B9
:1018D00084F88120F8BD19464269920713D593B167
:1018E000012B43D9E36B002B40D0E26D52F8043B4F
:1018F0000362B4F86230E265023B9BB2A4F8623046
:10190000B4F862309BB2426912F4604F11D081B1D9
:101910004269170452D5056BB4F86A20616E023A29
:1019200041F8045B92B26166A4F86A20B4F86A10C8
:1019300089B2D6F8CC2CA2EB0C02092A05D843EACE
:10194000010292B2002AC7D144E720460CF05AFAAD
:10195000D4F884300122002143F48073104684F8C7
:101960008010C4F8843084F88120F8BDE26D32F82C
:10197000023B0384B4F86230E265013B9BB2A4F8F9
:101980006230B4F862309BB2BDE7516901F4C041E6
:10199000B1F5005F47D9028E616E21F8022BB4F8D1
:1019A0006A206166023A92B2A4F86A20B4F86A101A
:1019B00089B26FE7683B00240000FFFF028E616E72
:1019C00021F8022BB4F86A206166013A92B2A4F8B9
:1019D0006A20B4F86A1089B2ABE7012B11D1E36D2C
:1019E0001B7882F82030B4F86230E56D013B226844
:1019F00001359BB2E565A4F86230B4F862309BB261
:101A000031E7E36B002BEAD0E56D35F8023B038448
:101A1000B4F86230E565023B9BB2A4F86230B4F8DA
:101A200062309BB21FE792F83010626E1170B4F80A
:101A30006A20616E013A013125E72068CAE600BFDD
:101A4000034690F83C00012800F0AF810220F0B579
:101A5000012483F83D0083F83C40142A54D8DFE881
:101A600012F05B005300530053009E0053005300DC
:101A700053006701530053005300DE00530053002E
:101A800053001D0153005300530015001A68D1F88C
:101A900008C0156A0F6825F480159F4E1562B24282
:101AA000106AD2F804E0546D20F4001024F4E044ED
:101AB00040EA0C5044EA07240ED0984DAA420BD0BD
:101AC00006F5804605F58045AA4218BFB24203D00C
:101AD00005F58065AA4204D12EF4003E4D694EEA18
:101AE000852E4D68C2F804E05465D5651062506DCE
:101AF0000C6940F400605065506D20F480605065C2
:101B0000516D41EA0421516500220121104683F8FC
:101B10003D1083F83C20F0BD1A688E68156A0F6886
:101B200025F001057E4C1562106A556820F0020010
:101B3000D2F818C03043784E0CEA0404B24244EAAA
:101B400007040ED006F58066B2420AD0754F06F53E
:101B50008046B24218BFBA4203D006F58066B24250
:101B60000BD1CE6820F008008F6925F44075304312
:101B70004E693E4320F0040035434E685560946141
:101B80005663106290690C6940F00800906190699A
:101B900020F004009061916921439161B4E71A68D3
:101BA0008E68156A0F6825F010055F481562146A83
:101BB000D2F804C024F02004956944EA0614564E75
:101BC0002840B24240EA072000F0F180534DAA427B
:101BD00000F0ED80534E554DAA4218BFB24203D0DB
:101BE00005F58065AA4206D14E692CF4406C8D69DA
:101BF00035434CEA850C4E68C2F804C09061966388
:101C0000146290690C6940F400609061906920F45E
:101C100080609061916941EA0421916174E71A68DA
:101C2000D1F808C0156A0F6825F480553A4E156240
:101C3000B242106AD2F804E0D46920F4005024F4CF
:101C4000E64440EA0C3044EA07240ED0334DAA4261
:101C50000BD006F5804605F58045AA4218BFB24272
:101C600003D005F58065AA4204D12EF4804E4D695B
:101C70004EEA851E4D68C2F804E0D4611564106216
:101C8000D0690C6940F40060D061D06920F48060B4
:101C9000D061D16941EA0421D16135E71A68D1F8F0
:101CA00008C0156A0F6825F480351B4E1562B242D4
:101CB000106AD2F804E0546D20F4003024F070046F
:101CC00040EA0C4044EA07040ED0144DAA420BD05F
:101CD00006F5804605F58045AA4218BFB24203D0FA
:101CE00005F58065AA4204D12EF4803E4D694EEA86
:101CF000052E4D68C2F804E0546595651062506D7C
:101D00000C6940F008005065506D20F004005065EB
:101D1000516D21435165F7E6000001400004014088
:101D20008CFFFEFF00400140FF8CFFFE004401409D
:101D30001A68D1F808C0156A0F6825F48075244E1A
:101D40001562B242146A5568D06924F4007420F018
:101D5000730044EA0C2440EA070030D006F58066A0
:101D6000B2422CD01B4F1C4EB24218BFBA4203D015
:101D700006F58066B24206D125F440574E698D695A
:101D8000354347EA05154E685560D061D663146245
:101D9000D0690C6940F00800D061D06920F00400DF
:101DA000D061D1692143D161AEE60220704724F0B1
:101DB0008004CE6844EA061424F0400414E724F4B6
:101DC0000064CE6844EA062424F48064D4E700BFAB
:101DD0000000014000400140004401402DE9F04F67
:101DE000DFF83CB28BB0482200210BF54D6059F072
:101DF00041FC0BF618504FF431727D4959F0C8FB85
:101E00009BF8DC3F1BB19BF8DD3F8BF8D03C9BF887
:101E1000DE3F1BB19BF8DF3F8BF8F43C9BF8E23FC1
:101E20001BB19BF8E33F8BF8E83C9BF8E03F1BB10C
:101E30009BF8E13F8BF8DC3C6E4B00276E4A1B8819
:101E400012881B096D4C6E49C3EB12102288CBF827
:101E5000F43F13096B4C6C4E6C4DCBF8F03F91FB8B
:101E6000F0F1CBF8F81F03E001370C34062F27D030
:101E7000042F00F08380052F00F0A5802078002833
:101E8000F2D0634A002301331E2BEDD012F80C1F51
:101E90008842F8D103EB430C5E49002205EB8C0C21
:101EA0000868EC3128B19CF881031041C00700F1AB
:101EB00031830132032AF3D101370C34062FD7D1F5
:101EC0000027554DB94655F86C3C1BB1EB6F002B04
:101ED00040F04F8109F10109EC35B9F1030FF2D15E
:101EE00000274C4DDFF83CA13E46DFF83C91DFF87F
:101EF0003C812B68002B00F03281D5F8E830002BB4
:101F000000F02D81AC68544500F031814C4500F063
:101F10002E8142488268A16849072ED495F858104E
:101F200001292AD002F01F020121092A85F8581040
:101F300000F2138240F22121D140C90740F10D8205
:101F4000A16811F0010140F08A80D4F808E0DFF8C0
:101F5000E0C01EEA0C0F3DD0EC2303FB06B6D6F81A
:101F6000743D86F8701D43F01003C6F8743DD6F832
:101F7000783D43F00103C6F8783DFEE702214FF4B7
:101F8000002CB6460A46EC2007236170012100FBB5
:101F900002B22078A372D2F8003EC4F804E043EA0B
:101FA0000C036172C2F8003E00283FF45DAF43F0BD
:101FB000D1FAFB1DDBB210B100228371C271032183
:101FC00043F0BAFC50E702214FF4802CDFF864E0C4
:101FD0000A46D8E7A16801EA080141F00101A160C1
:101FE000DBF8CCCC8168C90636D04C4534D136E01C
:101FF000A4B9090820E8F11F40E8F11F60E8F11FCB
:102000008038010038480024000084CBE8B8090873
:1020100068BC090880480024EC480024006302588A
:10202000683B00240020024000210240C0FFFF7FE7
:102030003F0000800000B8CFA168C80705D4A168A0
:1020400001EA080141F00101A160DBF8CC1CA1EB21
:102050000C01022900F247862168C907ECD5EC2063
:10206000C1494C4500FB06B0D0F874CD0CEA010123
:1020700041F48071C0F8741D00D142B9EC2202FB1A
:1020800006B2D2F8741D21F48011C2F8741DEC223E
:1020900002FB06B2D2F8741D11F4805140F0D483D3
:1020A000C2F8781D4FEA530E686D9908AF4A0EF0DA
:1020B000773E01F03331C263DA088E44AC4902F056
:1020C0001132A3EB0E0E0164AA4B1C21AEEB020EE3
:1020D000C364FF2321600EEB1E1E626800210EF018
:1020E0000F3E42F0100285F8581004F14001626082
:1020F000E268BEFBF3F322F0030C6A6BC3EB03232D
:102100004CEA0202DFF89CC2AEEB0303E2600CEB88
:1021100047020AF0FDF8AA68936803EA080343F04F
:1021200004039360002840F0B083D5F8E830924A69
:1021300059089C0801F07731D80804F0333400F0D6
:10214000113021445B1A1B1A03EB131303F00F33F6
:10215000A2FB0312D209C2EB02229B1A1F440136D2
:10216000EC35032E7FF4C5AE0BB0BDE8F08F83488D
:10217000D0E6A5F1640435F8680C0294FEF7ECFE95
:10218000EC2355F86C2CEE6F03FB09B345F8642C77
:10219000D3F8742D42F00202C3F8742D55F8643C54
:1021A00099689A6801F0040102F008020A431ED0FF
:1021B000DA68900100F18F819A68540703D59A6814
:1021C000910740F1AC859A68120703D59A68940785
:1021D00040F19D850C21DBF8CC0C05E0DBF8CC2C24
:1021E000121A052A00F23C839A680A42F6D1DA688C
:1021F000029842F40012DA600AF01EFF044600283A
:1022000000F01B8355F8643C40F2FF705C490022EB
:10221000D3F804C00CEA0101DFF88CC159601860E2
:102220009868584920F0A0409860986840F00050A5
:102230009860D86800F08020D860D86840F00040EE
:10224000D860186900EA0C0C4F48C3F810C0D3F8E6
:1022500014C00CF0404CC3F814C0D3F818C00CF0F4
:10226000784CC3F818C0D3F820C00CF07C4CC3F8ED
:1022700020C0D3F824C00CF07C4CC3F824C0D3F8A1
:10228000B0C00CF07C4CC3F8B0C0D3F8B4C00CF0B4
:102290007C4CC3F8B4C0D3F8B8C00CF07C4CC3F885
:1022A000B8C0D3F8BCC00CF07C4CC3F8BCC0D3F8A9
:1022B00030C00CEA0101DFF8F4C01963596B01402A
:1022C0005963996B014031489963D96B01EA0C0C51
:1022D0002F49C3F83CC08B42D3F860C01A66D3F8CC
:1022E00064C05A66D3F868C09A66D3F86CC0DA66E0
:1022F000D3F8A02002EA0002C3F8A020D3F8A4205B
:1023000002EA0002C3F8A420D3F8C02002EA0002C7
:10231000C3F8C020D3F8C42002F0F822C3F8C420C8
:1023200000F0CF801B4A934200F0CB801A4B9B6891
:10233000D90704D4194B9968194A0A409A60EC22CB
:10234000002302FB09B2C2F8783D45E90233C2F826
:10235000743D05F8143C5CB3FEE7EC22002302FB5D
:1023600006B686F8703D08E6FEF0FFFF959F04086C
:10237000919F04087D9F0408818080800023024093
:1023800000F8FFFF300882E0200882E00000F0FF44
:102390000020024000210240006002580063025801
:1023A000E03000FE000000301CF800FC20F8FFFFC9
:1023B00073084FF4403CB10805F8504C03F07733F4
:1023C000F00801F0333145F860CC00F011304FF0E7
:1023D000040C0B44FF2105F8484CF31A082645F875
:1023E000404C1B1A012045F83C4C03EB131305F835
:1023F0004F0C45F8440C03F00F3305F82C4C0494B3
:1024000045F854CCB3FBF1F1C1EB012145E917606C
:10241000591A03264FF4805045F84C1C45E90E60CC
:10242000D2F8743D002B00F0168255F864CCDCF82D
:1024300008309A0005D5DCF80820964B1340CCF8FC
:102440000830DCF80830DB0015D4DCF80810924ABC
:10245000924BD2F8F8200B409149B2FBF1F243F0D5
:102460008053CCF80830049202E0049B013B0493B3
:10247000049B002BF9D1DCF80830DE000ED4EC23ED
:10248000012403FB09B3D3F8742D42F01002C3F802
:10249000742DD3F8782D2243C3F8782DDCF808305A
:1024A000580744D5EC2303FB09B3D3F8743DEC2360
:1024B00003FB09B3D3F8742D42F01002C3F8742D56
:1024C000FEE7784B784A9B6892681343D8073FF53C
:1024D00036AF764B2FE735F8501C40F2011291428F
:1024E0007FF46AAE724A02E0013A00F0B9811968DD
:1024F0004906F9D540221A609A68520708D59A68A9
:10250000900705D499686B4A0A4042F010029A601D
:10251000042160E60C204FF0010C51B200FB035384
:1025200093F88803D3F884E30CFA00FC2BE5EC2342
:1025300003FB09B3D3F8742DD606B8D4D3F8742DA1
:1025400022F4817242F00202C3F8742DDCF80830E4
:10255000D90714D4534B9C4500F0AE8303F5807328
:102560009C4500F0A983544B9B68DB0707D4534973
:102570008B6855F8602C23F47C1313438B60504A0E
:1025800041F203031268B3EB124F55F85C2C02D2F0
:10259000102A00F09B8355F8343C15F84F0C134378
:1025A00015F8481C43EA403343EA0143012904D1AA
:1025B00055F8442C013A43EA424355F8402C2AB1DD
:1025C00002F4787255F83C1C0A431343DCF80C10F3
:1025D0003C4A0A401343CCF80C30DCF80820DCF805
:1025E000083002F0040203F00803134300F0BF8137
:1025F00055F8643C55F8582C012A00F0AF811A6B4D
:1026000022F00F021A63EC2606FB09B6D6F8743DD9
:1026100006F6745823F0030343F00103C6F8743D33
:10262000002C40F09A8115F8143C0594012B00F021
:1026300043810123029805F8143C0AF0FDFC0028B0
:1026400040F08281D6F8741D1F4A204B0A40204971
:1026500042F00202C6F8742D55F8642C90680340CD
:1026600043F0004393609368002BC0F21081EC228A
:102670000020DFF860E002FB09B201460190D2F8C9
:10268000743D23F0030343F00103C2F8743D05F8E1
:10269000140C29E0C0FFFF5F00000024C0FFFF6FA3
:1026A000400D0300002002400021024000230240B0
:1026B00001DC0C00C0FFFF7F00600258006302587D
:1026C0000010005C03C0F0FFFDEEFFFFC0FFFE3F07
:1026D00000F8C32538480024019B0EF10C0E01338D
:1026E000062B019300F0E9809EF80930002BF3D00F
:1026F0009EF901304B45EFD1C84B00224E1C8EF89D
:10270000087003EB810015F8143C791C0692012B2C
:10271000D0F8E844DEF80420039100F0D58155F8A4
:10272000643C0120996805F8140C4F0700F1BD8145
:10273000C2F3130CBCF1000F40F0AE81C2F384670A
:10274000910EB840D3F81CA04FEA941803F130075B
:1027500004F01F044AEA000A08F00C004FF01F08BA
:10276000C3F81CA0BA4601EA0801C75908FA04F8E0
:10277000A14027EA080848EA010140F80A109868D1
:10278000996800F0040001F00801014343D1D10D24
:10279000C2F3045A03F114044FF0070801F00401D6
:1027A000062708FA0AF8085907FA0AF7DFF888A294
:1027B00020EA080038430851DAF8001001F07041AF
:1027C000B1F1805FD96800D0D968196E900601F028
:1027D000F841B1EB826F03D1196E21F00041196607
:1027E000596E01F0F841884203D1596E21F0004141
:1027F0005966996E01F0F841884203D1996E21F033
:1028000000419966D96E01F0F841884203D1D96E32
:1028100021F00041D9669968C80708D4D3F8C010E0
:10282000002A21EA0C01C3F8C010C0F20B8100237A
:102830003146039F05F8143C4EE7EC23012203FBCD
:1028400009B3C3F8742DDDE4D2F8781D21F0060138
:10285000C2F8781D26E4C2F8784D05F8144CE4E57A
:10286000EC22012402FB09B2D2F8741D41F01001E0
:10287000C2F8741DD2F8781D41F00101C2F8781D2C
:10288000DA6842F40012DA60BCE4FFF776BB059B1D
:1028900001330593059B8B42FFF4E5AEEC23002149
:1028A00003FB09B3D3F8742D83F8701D22F01202D4
:1028B00042F01002C3F8742DFEE7594B5FFA89F617
:1028C00002204B44314693F9102043F023FB0028AB
:1028D0003FF44AAC534CD0E90123C5E9002310462C
:1028E00051F0BEFF421E731CDFF854C104EB4214CA
:1028F0000026D9B24FF48060D4F8FC304FF4006267
:1029000028616A6163450CBFA020A1204FF480724A
:102910004FF48033C5E902664FF40056C5E907233A
:10292000AE61FEF719FB019B84F81511284684F867
:10293000143109F097FE284609F0FCFF029B45F888
:10294000185CAB63FFF7C6BAD8F8003086F8704D54
:1029500043F01003C8F80030AEE7B1E5196B55F845
:102960004C2C21F00F01013A0A431A634BE6DCF8C4
:102970000C202D4915F8500C114055F8382C41EA1F
:10298000803115F82C0C0A430128CCF80C2000F0FB
:102990007E81DCF8102022F00102CCF81020DCF857
:1029A000101055F8302C21F0704120480A4384451E
:1029B000CCF8102000F063811D4A944500F05F813F
:1029C0001C4A926812F4403F14BF01220022002AE0
:1029D00000F0DF8011F02AFC55F8602C0346B2F5B8
:1029E000003F00F0D280B2F5403F00F0BD80B2F56C
:1029F000803F00F0CA80104941F203020968B2EB3F
:102A0000114FC0F0A7800D4A93426FD955F8643C2E
:102A10009A6842F480729A60ECE500BFE8B8090851
:102A2000444B002400000024FCBFFFFF00200240B4
:102A300000210240006302580010005C002D3101AB
:102A400000000240BA498B423FD001F580718B42B1
:102A50003BD0B849B8488468896804F0E077C94336
:102A600001F0010109B3B5498A4255D0B4498A42FF
:102A700043D0B4498A427FF4DAAE64023FF5D7AE60
:102A8000AC4A93427FF4D3AE836823F0E0733B43B8
:102A900043F480038360CAE692FAA2F7B7FA87F795
:102AA000910E07F01F07B8404CE6EC2303FB09B377
:102AB000D3F8742D42F02002C3F8742DEC230022C9
:102AC00003FB09B383F8702DFEE79F499F4F8C6885
:102AD0000846A1F540718968D7F808C004F0E0778E
:102AE00041EA0C01C94301F00101BBE755F8643C20
:102AF0009A6822F480729A607CE5E2013FF597AE15
:102B00008C4A93427FF493AE836823F0E0733B4397
:102B100043F0807383608AE621023FF588AE854AE0
:102B200093427FF484AE8A4A8368D2F8F8208949B8
:102B300023F0E073B2FBF1F23B43520043F4000395
:102B40008360069202E0069B013B0693069B002BE6
:102B5000F9D16CE6804A934208D855F8643C9A68EB
:102B600022F440729A6045E5830844E77B4A934229
:102B700042D97B4A934255F8643C9A6825D822F49E
:102B8000407242F400729A6034E5120CB3FBF2F327
:102B900031E774498A6D02F44032B2F5803F5ED06D
:102BA000B2F5003F4ED0002A62D055F8602CB2F545
:102BB000101F45D00DD8B2F5E01F3FD025D9B2F592
:102BC000001F7FF418AF5B0915E742F440729A606A
:102BD00010E5B2F5201F50D0B2F5301F7FF40BAFD7
:102BE000614941F203020968B2EB114FBFF47EAFB5
:102BF000594AB2EB132FB0D255F8643C9A6822F4CC
:102C0000407242F480729A60F4E4B2F5801F07D0FB
:102C10000BD9B2F5A01F03D0B2F5C01F7FF4EBAE05
:102C2000920C5200B3FBF2F3E5E6B2F5002FF7D0B9
:102C300022F40021B1F5802FF2D0DCE61B09DAE6A0
:102C40009B09D8E6CA6C12F040520FD0B2F1805FF7
:102C50000AD04649B2F1005F08BF0B46A5E707A8B6
:102C60000BF07CFB099BA0E7414B9EE7414B9CE7A7
:102C700007A80BF01FFC079B97E7DB09BBE6324A6E
:102C8000926812F4403F14BF012200229FE655E9EA
:102C9000092655F8281C324355F81C0C0139DCF87C
:102CA000106042EA01423449024331400A4342F093
:102CB0000102CCF8102072E61D4B244A9B689268F2
:102CC0001343DA073FF55BAC1F4951E415F8481C84
:102CD00015F84F0C0B0455F8342C43EA40331343DA
:102CE00043F01C0362E4EC23002203FB06B6D6F893
:102CF000743D86F8702D43F01003C6F8743DD6F885
:102D0000783D43F00103C6F8783DFFF736B999687E
:102D10001A4A0A4042F020029A60FFF75BBA9968AB
:102D2000164A0A4042F010029A60FFF74CBA00BF00
:102D3000002002400060025800630258000084CB6B
:102D4000000052C70000B8CF00230240002102401B
:102D500000000024400D030021BCBE0041787D012D
:102D600081F0FA02004402580010005C00127A0060
:102D700000093D000090D0031EF800FCC0FFFF7F5B
:102D80002DE9F041D0F800E00C46DFF8588084B01F
:102D9000DEF804501746DFF850C0194605EA08056A
:102DA000DDF82880064603932C43424644EA0C0C87
:102DB000CEF804C011F0D4FD78B931680246039B07
:102DC00030468F628021CDF8008011F0F9FD003887
:102DD00018BF012004B0BDE8F081012004B0BDE8B7
:102DE000F08100BF009800FC00200181F8B5144F6D
:102DF00004460D460BE09B69DB0602D511F070FD21
:102E0000E0B9D7F8CC3C5B1BB3F5805F09D82368E9
:102E10002A464FF4805120469E69B606EBD5002025
:102E2000F8BD636C2021002201200B4384F8402070
:102E3000636484F8411084F84220F8BD0120F8BD95
:102E4000683B00242DE9F041D0F800E00C46DFF8A3
:102E5000588084B0DEF804501746DFF850C0194699
:102E600005EA0805DDF82880064603932C43424610
:102E700044EA0C0CCEF804C011F072FD78B9316848
:102E80000246039B30468F624021CDF8008011F04E
:102E900097FD003818BF012004B0BDE8F081012083
:102EA00004B0BDE8F08100BF009800FC0020018064
:102EB000524870B490F8FC3F514D03EB43015A0067
:102EC00005EBC10111F8F81C032920D8DFE801F057
:102ED0000E220242D11805EBC10151F8F40C18B3CF
:102EE000431E002070BC41F8F43C7047454991F8FE
:102EF0002061002E69D001F59471002001E0864226
:102F000063D00C88013001F5AE71002CF7D00120A0
:102F100070BC7047D11805EBC10151F8F40C0028C2
:102F2000DED1022001F8F80C1A4405EBC20111F8B9
:102F3000EC2C013AD2B201F8EC2C42B3324B012016
:102F4000D3F8FC2202F2E733B3FBF2F370BC41F892
:102F5000F43C70471A4405EBC20252F8F41C0029F5
:102F600046D115F8982C9342D1D0013303F00304D5
:102F7000A24280F8FC4FCAD004EB44030224084666
:102F800005EBC30242F8F41C02F8F84CC0E71E4AF5
:102F9000581C032651F8F03CD2F8FC42304015F89A
:102FA000985C621E01F8F86C401B1A4418BF01209F
:102FB0009442B2FBF4F388BF002041F8F43C0028AF
:102FC000A5D0013B41F8F43CA2E70F4842F20F7153
:102FD00013440126D0F8FC4205EBC30230462144DD
:102FE00002F8F86CB1FBF4F170BC42F8F41C7047C5
:102FF0000139002042F8F41C8AE700BF683B002436
:10300000604C0024140000200000002470B5114C16
:1030100041F20D13104D41F2883254F8501C54F80F
:10302000940C0E040D218660C66835402B43C360A6
:103030000AF030FB38B154F8602C034600201343EB
:1030400044F8603C70BD54F8943C5869C0F3432088
:1030500070BD00BF604C0024C0E0FEFFF8B5374FE4
:103060000546374C082157F8940CD4F8CC6C0AF07C
:103070000BFC034608B11846F8BD57F8501C57F82A
:10308000940C09040AF0A0FB03460028F3D157F87A
:10309000940C4FF0FF31082241F2331C41628262EE
:1030A000C26A284922F0FF0242F03302C26241F2B2
:1030B00088328360C368194041EA0C0C3321C0F8A0
:1030C0000CC00AF0E7FA03460028D4D157F8941C44
:1030D0008446074640F22A5004E0D4F8CC2C921BD8
:1030E00001321FD04A6B02420AD14A6B1203F4D458
:1030F000002BF2D1D1F880700123D1F880C0ECE729
:103100004B6B1A0714D44B6B9B070ED44B6B13F00D
:10311000200310D19CFA8CF23FBA0B488863C5E9B2
:103120000027A8E74FF00043A5E702238B63A2E73F
:1031300008238B639FE720238B639CE7604C00246C
:10314000683B0024C0E0FEFF3A0F0018114B30B47A
:1031500018690025D3E9054220F01F019D6004FB9A
:103160000202521ABFF34F8FAA420DDD013A01F15C
:103170002003094822F01F021A449342C0F85C124F
:10318000194603F12003F8D1BFF34F8FBFF36F8FC0
:1031900030BC7047604C002400ED00E070B503784F
:1031A00084B004461646012B24D0022B1FD1C368DD
:1031B00041F080051BB19A88196812048A610123C5
:1031C0000DF10F020DF10E0160688DF80E504DF0FB
:1031D00063FE01233246002160684DF05DFEE36826
:1031E0008BB11A6801209B88936104B070BD0020E8
:1031F00004B070BD00920A46417990F9040051F084
:1032000085FC04B070BD0120F2E700BF2DE9F84F46
:10321000C14C0546217F606AC1F3400142F0BCFC0D
:10322000217F206AC94301F0010142F0B5FC002D65
:1032300000F0DD8005F1FF39B84E4FF01008B84FAF
:103240005FFA89F9B74D636A33B11A689B8851698F
:103250000B4218BF1B049361236A33B11A689B8821
:1032600051690B4218BF1B049361A38D002B40F0E2
:103270004C8194F82E10206B42F08EFCFA204FF413
:103280007A714FF0010C7B68C3F30803002B40F008
:103290001281EFF31183002B40F00D81D6F8B42D8D
:1032A000D5F808E0D6F8B43D9A42F7D1636D9E4553
:1032B000F4D8D4F850A001FB0AF3A3EB0E03B3FB40
:1032C000FAF301FB02327B68C3F30803002B40F0E2
:1032D000B180EFF31183002B40F0AC80D6F8B43D01
:1032E000D5F808B0D6F8B4ED7345F7D1D4F854E06A
:1032F000F345F3D8D4F850A001FB0AFEAEEB0B0E59
:10330000BEFBFAFE01FB03E39B1AB3F57A7FDAD327
:103310000138B8D1636A33B11A689B8851690B428E
:1033200018BF1B049361236A33B11A689B885169E3
:103330000B4218BF1B049361A38D002B40F0DB8070
:1033400094F82E10206B81F0010142F025FCFA2048
:103350004FF47A714FF0010C7B68C3F30803002B24
:1033600040F08980EFF31183002B40F08480D6F881
:10337000B42DD5F808E0D6F8B43D9A42F7D1636D84
:103380009E45F4D8D4F850A001FB0AF3A3EB0E033A
:10339000B3FBFAF301FB02327B68C3F3080343BBC0
:1033A000EFF311832BBBD6F8B43DD5F808B0D6F8AF
:1033B000B4ED7345F7D1D4F854E0F345F3D8D4F81D
:1033C00050A001FB0AFEAEEB0B0EBEFBFAFE01FBAA
:1033D00003E39B1AB3F57A7FDED30138BCD109F140
:1033E000FF395FFA89F9B9F1FF0F7FF42CAFBDE81F
:1033F000F88FEFF3118A88F31288D5F808B02B689C
:10340000DB0303D5C4F84CC0D5F808B0D6F8B43DFA
:103410005FFA8AFAD4F84CE08AF31188D4F850A005
:10342000734401FB0AFEAEEB0B0EBEFBFAFE01FB82
:1034300003E3CEE7EFF3118A88F31288D5F808B0DA
:103440002B68DB0303D5C4F84CC0D5F808B0D6F818
:10345000B43D5FFA8AFAD4F84CE08AF31188D4F8C4
:1034600050A0734401FB0AFEAEEB0B0EBEFBFAFE4E
:1034700001FB03E348E7EFF3118E88F31288D5F8D8
:1034800008A02B68DA0303D5C4F84CC0D5F808A00F
:10349000D6F8B43D5FFA8EFEE26C8EF31188D4F854
:1034A00050E01A4401FB0EF3A3EB0A03B3FBFEF357
:1034B00001FB023270E7EFF3118E88F31288D5F822
:1034C00008A02B68DA0303D5C4F84CC0D5F808A0CF
:1034D000D6F8B43D5FFA8EFEE26C8EF31188D4F814
:1034E00050E01A4401FB0EF3A3EB0A03B3FBFEF317
:1034F00001FB0232E7E6A36C002B3FF428AF002368
:10350000626B136084F8453021E7A36C002B3FF415
:10351000B5AE3FF0BDFDB1E6604C0024702A00243A
:1035200000ED00E010E000E02DE9F04FBE4C83B06C
:103530000523BE4E217F4FF01009606AC1F34001A0
:10354000019342F029FB217F206AC943DFF8E4821E
:10355000B74D01F0010142F01FFB636A33B11A68F5
:103560009B8851690B4218BF1B049361236A33B1D6
:103570001A689B8851690B4218BF1B049361A38D85
:10358000002B40F04A8194F82E10206B42F004FB8F
:1035900032204FF47A710127D8F80430C3F30803BE
:1035A000002B40F01181EFF31183002B40F00C81D0
:1035B000D6F8B42DD5F808E0D6F8B43D9A42F7D144
:1035C000636D9E45F4D8D4F850A001FB0AF3A3EB39
:1035D0000E03B3FBFAF301FB0232D8F80430C3F355
:1035E0000803002B40F0B180EFF31183002B40F073
:1035F000AC80D6F8B43DD5F808B0D6F8B4ED734534
:10360000F7D1D4F854E0F345F3D8D4F850A001FB37
:103610000AFEAEEB0B0EBEFBFAFE01FB03E39B1AA8
:10362000B3F57A7FD9D30138B6D1636A33B11A685A
:103630009B8851690B4218BF1B049361236A33B105
:103640001A689B8851690B4218BF1B049361A38DB4
:10365000002B40F0D88094F82E10206B81F00101EF
:1036600042F09AFA32204FF47A710127D8F80430E8
:10367000C3F30803002B40F08880EFF31183002B85
:1036800040F08380D6F8B42DD5F808E0D6F8B43DE4
:103690009A42F7D1636D9E45F4D8D4F850A001FB4F
:1036A0000AF3A3EB0E03B3FBFAF301FB0232D8F8E3
:1036B0000430C3F3080343BBEFF311832BBBD6F8ED
:1036C000B43DD5F808B0D6F8B4ED7345F7D1D4F8C9
:1036D00054E0F345F3D8D4F850A001FB0AFEAEEB5A
:1036E0000B0EBEFBFAFE01FB03E39B1AB3F57A7FD8
:1036F000DDD30138BAD1019B5F1E17F0FF030193A0
:103700007FF42BAF03B0BDE8F08FEFF3118A89F39C
:103710001288D5F808B02B68DB0302D5E764D5F82A
:1037200008B0D6F8B43D5FFA8AFAD4F84CE08AF3D0
:103730001188D4F850A0734401FB0AFEAEEB0B0EC7
:10374000BEFBFAFE01FB03E3CFE7EFF3118A89F337
:103750001288D5F808B02B68DB0302D5E764D5F8EA
:1037600008B0D6F8B43D5FFA8AFAD4F84CE08AF390
:103770001188D4F850A0734401FB0AFEAEEB0B0E87
:10378000BEFBFAFE01FB03E349E7EFF3118E89F379
:103790001288D5F808A02B68DA0302D5E764D5F8BB
:1037A00008A0D6F8B43D5FFA8EFEE26C8EF3118865
:1037B000D4F850E01A4401FB0EF3A3EB0A03B3FB69
:1037C000FEF301FB023272E7EFF3118E89F31288E8
:1037D000D5F808A02B68DA0302D5E764D5F808A06D
:1037E000D6F8B43D5FFA8EFEE26C8EF31188D4F801
:1037F00050E01A4401FB0EF3A3EB0A03B3FBFEF304
:1038000001FB0232E9E6A36C002B3FF42BAF00234F
:10381000626B136084F8453024E7A36C002B3FF4FF
:10382000B7AE3FF035FCB3E6604C0024702A0024AC
:1038300010E000E000ED00E010B4A8B10C4CA36D66
:10384000102B05D1052100205DF8044B3BF0F0BAA8
:1038500003EB4302224482F85D10012182F85C00F0
:103860000B4482F85E10A3655DF8044B704700BFFF
:10387000604C002430B5044683B00D4608480DF175
:1038800007022146FFF78AFC9DF8072035EA02036C
:1038900004D02A432146024843F052F803B030BD19
:1038A000EC4C00240378012B01D00020704790F9E4
:1038B0000420084902EB420201EB421292F8251162
:1038C000202901D018467047D2F8E4309869C0F337
:1038D000C0307047604C00242DE9F0411F4C84B08B
:1038E0000746884694F88C501646022D11D0012DBB
:1038F0000BD113460091024694F8911094F9900070
:1039000051F004F904B0BDE8F081002004B0BDE836
:10391000F081D4F898301BB19A88196812048A6132
:1039200001230DF10F020DF10E01D4F890008DF876
:103930000E704DF0B1FA334642460021D4F89000A3
:103940004DF0AAFAD4F8983033B11A6801209B8858
:10395000936104B0BDE8F0810120D3E7604C0024FE
:103960002DE9F04F037885B004460E46022B00F097
:103970008E80012B04D00025284605B0BDE8F08FCD
:1039800090F904105C4F042987F85032D4BF002509
:103990000125B1F1FF3F08BF45F00105002DEAD137
:1039A00001EB4102480007EB4212D2F8E4C0BCF13F
:1039B000000FE0D092F825E1BEF1200FDBD1DCF85A
:1039C000188018F40048D6D192F824C1BCF1010F38
:1039D000D1D04FF0400CDFF838E14FF0210BDFF889
:1039E000349194F805A0DEF8CCEC82F825B182F889
:1039F00026C107F5147CC2F82881A2F80E31C2F85E
:103A00001091B2F80E4182F82431A3B23B4CC2F8B7
:103A100008C1FF2BC2F8184169D8B2F80EC14FF0A7
:103A200000791FFA8CFC441835484FEA4A0ACDF851
:103A300000E000EB4410324607EB441451461430CA
:103A40001923A4F80CC1FFF79BF9002845D1D4F83D
:103A5000E4202C49536894F80C610B402A4DD4F8AB
:103A6000181143EA0A03A94243EA064343EA090359
:103A7000536084F8240104D0244B994218BF4FF0BE
:103A8000F2081368012543EA0803136074E7C3686A
:103A90001BB19A88196812048A6101250DF10F0281
:103AA0000DF10E0160682B468DF80E604DF0F4F9B3
:103AB0002B460DF10F020DF10E0160688DF80E50CE
:103AC0004DF0EAF9E368002B3FF456AF1A68284638
:103AD0009B88936105B0BDE8F08FB7F852320022A1
:103AE000013384F824219BB2A7F8523244E74FF007
:103AF000FF0C4FF0807996E7604C002405500508D4
:103B0000304D0024009C00FCA94D0508C14E05085D
:103B1000683B00240000FFFF036870B55E6A26B1B1
:103B200033460522BDE87040184704460D464E1D39
:103B300000E023689B68204698470028F9D0236856
:103B4000204615F8011B1B689847B542F1D170BD9E
:103B50002DE9F0470023194D84B0074695F9599295
:103B600005F518764FF0B60A00EB010805F5A065DB
:103B70001C46D6F800C0304600226946E036BCF14B
:103B8000000F14D09CF838C0BCF1140F0FD0B9F15D
:103B9000FF3F01D0CC450AD1CDE90244CDE9007800
:103BA000ADF808A08DF80E4033F058FD0346B5423D
:103BB000DFD1184604B0BDE8F08700BF604C002498
:103BC000F0B500230E680DE0BCF1050F17D9BEF16A
:103BD000050F18D80A2C16D103EB830316F8010B36
:103BE00004EB4303A0F13005A0F1610CA0F1410EFC
:103BF000A0F13704EFB2092FE6D82C46ECE7A0F18C
:103C000057040A2CE8D00E601360F0BD2DE9F7438D
:103C1000A0230124114E18255FFA84F8FF2B14DC31
:103C2000E9B2D6F800055F1CDBB2C1F11C02C1F19C
:103C30001B0180F80B808272C9B2026800930023D6
:103C4000D2F818904246C8473B46013DE6D10134C0
:103C5000052CE0D103B0BDE8F08300BF604C002428
:103C600008B5FCF79DFE38B10449054842F0BEF99D
:103C7000034819F049FC024808BD00BF10BE0908FE
:103C8000645100242DE9F04F884C16460B2287B072
:103C900094F89287054694F89DA7894640461146B8
:103CA00002951D469DF840703AF0CAFEC245834613
:103CB00040F0B0800390404641F04CFC17F0080300
:103CC0000246019300F09980BBF1000F00F0918053
:103CD0009BF80710890700F18C80C4F85CB5C4F824
:103CE0005805C4F85405002800F0DC8040F60B317C
:103CF00005F0020AC1804FF48073DFF8C881029991
:103D0000584608EB030284F81C550025C4F84415F6
:103D1000C4F830253146664AC4F82435C4F818255D
:103D2000C4F82835C4F8206584F81D75C4F8489592
:103D3000C4F82C85C4F83855C4F83455C4F8405537
:103D4000C4F83C55C4F8745784F87857A4F86C57F5
:103D500032F0DCFED4F85C0507F00101FDF7B4F8A1
:103D6000544A554BD4F85C05C4F88057C4F88427EE
:103D7000C4F87C37BAF1000F1CD0D4F86475CFB109
:103D80003A6803689A4215D001233146384684F8D0
:103D9000793732F0BBFE08F505722946D4F8640580
:103DA00052F084FD2A4608F50771D4F85C0552F0FC
:103DB0007DFD07E0414A002302F1080184F87937CC
:103DC00052F074FDD4F85C35186852F037FF019B4F
:103DD000C4F860052BB33A4832F0C0FE384807B04B
:103DE000BDE8F08F039BCDE9040113B1D8798307B7
:103DF0001FD5002007B0BDE8F08F15F00101F1D10B
:103E000005F0020C5FFA8CFABAF1000F2CD1D4F84D
:103E10005CB570E70B220C2150463AF011FE03907E
:103E200049E7274832F08EFE0121254832F0BCFEDA
:103E3000D1E7504605F0020A41F08CFB039AD446C4
:103E40000599C4F85C25049AC4F85405904202D13F
:103E5000BAF1000F1CD10028D4D040F60C3EA0F8D7
:103E600006E0BAF1000FD2D0B8F1000FC1D0C4F80B
:103E7000582591B9BBF1000FBBD0C4F85CB55FFA0F
:103E80008CFA002A3FF437AF40F60B31D18032E78D
:103E9000B8F1000FADD0C4F85825C4F864B5D4F813
:103EA0005CB5ECE705F0020A25E700BF604C002492
:103EB00060BE0908D95B0708C16B0708DC53002402
:103EC00078510024C85100242DE9F04FB648092547
:103ED000B64C0023022200F52E6665608BB0B44D0F
:103EE00094F8BD13C0F8B04DC4F804642560236392
:103EF000636123616362A261E260C4E90733C4E9DC
:103F00000A33002900F07B811F460321A84B84F867
:103F1000BD13DB6B13F48078AB6818BFD4F8108046
:103F200023F0010308BFC4F81080012AAB6040F001
:103F3000DC80AA6B9F4B22F48032616BAA6301295B
:103F4000EA6803EA0203EB60EB6823F44013EB60DA
:103F500000F09981284608F0F7FE0646B8F1010FF7
:103F600016D0FEB10222236884F8BD2394F82405FC
:103F7000012800F004818021012059625A6A42F42C
:103F800080029A62FCF722FB00200BB0BDE8F08FA4
:103F9000AB6843F00603AB60AB6843F02003AB6053
:103FA000002EDFD123683220DA6822F0C042DA60C6
:103FB000DA6842F08042DA6009F066FE606848B371
:103FC000324601273146C2EBC203551C04EB830382
:103FD00083F83C20A3F84220EAB283F83D70824285
:103FE00083F83F101965C3E91111ECD30022114683
:103FF000C2EBC203551C04EB830383F8FC21EAB235
:1040000083F8FD11824283F8FF11C3F81012C3E94F
:104010008111EDD300222368D4F80CC01546D4F8E2
:104020001080D4F82CE0D4E90671019102F140012E
:10403000013203EB81010F2A4D60F7D1BEF1000F71
:1040400040F01A81D3F8042803F5006542F002021B
:104050006A609A6B22F400129A631A6842F0400276
:104060001A601A6842F080021A600022012FC3F819
:10407000002E2A682A602A6800F0158142F00302A7
:104080002A604FF484614C4A196102E0013A00F061
:10409000128119698F06F9D41021474A196102E08B
:1040A000013A00F00A811969C906F9D40021296191
:1040B0006961E96160B303F510624FF0904A4FF017
:1040C000006B0F464FF67F399C4607E017600131C1
:1040D0001761C2F808902032884271D01368002B13
:1040E000F4DA91B1C2F800A0F1E7EB68284643F09A
:1040F0004003EB6008F028FEAB6B0646002F40F053
:10410000B78043F48033AB6328E7C2F800B0DEE742
:104110002A6900206FF0804122F480722A61986140
:104120005961B8F1000F03D19A6942F010029A6107
:104130009969224A0A439A61019A1AB19A6942F02E
:1041400008029A61BEF1010F00F0A280002E40F03B
:10415000A6800121626A84F838608A4284F8BD131F
:1041600000F0AD806B68032043F002036B6009F040
:104170008BFD94F82405236801287FF4FCAE80228F
:1041800040215A625A6A42F400129A62FCF71EFAFF
:1041900020210220FCF71AFA40210320FCF716FA2E
:1041A00000200BB0BDE8F08F702A0024781900249D
:1041B00000000840BFFFBDFF400D030000383C80F9
:1041C000002163460CF530624FF0904A4FF0006BCF
:1041D0000F464FF67F39844607E0176001311761BB
:1041E000C2F8089020328C4592D010680028F4DA8A
:1041F00011B1C2F800A0F1E7C2F800B0EEE701F09B
:10420000FF073A4B03204FF4C05584F8BC73D3F832
:10421000E01041F00101C3F8E01005A9D3F8E03047
:1042200006920A2203F00103089031480493049B8C
:1042300007970595099208F0DBFDE36A012B4BD047
:104240002A4B06216520D3F8D82042F00062C3F83B
:10425000D820D3F8D83003F000630393039BFCF716
:104260008BFD244B2021A2692568D960A76A4CE602
:1042700023F48033AB6371E69A6B03F5006542F477
:1042800000129A63F1E6EB6843F48013EB6061E699
:104290009969194A0A439A61002E3FF45AAF0222E3
:1042A00084F8BD2362E6BCF1000F3FF4E9AE42F0B2
:1042B00001022A60E5E60126EEE60126F6E684F82C
:1042C000F4639969C4F8FC2341F000610B4A9961D9
:1042D000596D0A435A6545E74FF4007305A9044830
:1042E0000593CDE9067708F083FDA9E7004402585D
:1042F0000000025800E100E004000040030000104C
:10430000094B93F8C638042B08D9053B032B08D872
:1043100001231A4600B103701046704700230122A2
:10432000F8E700231A46F5E7683B00242DE9F0473B
:104330009AB004460D4617469846DDF89090DDE9A0
:10434000226A02E0206841F09BF8206841F0A0F862
:104350000028F7D10146642201A857F08BF9264BBB
:104360008DF80450CDF85CA00293002D40D0AB1E18
:10437000012B3FD9042D14BF002303231F4A8DF8BE
:1043800005300123D2F8B42D039616448DF85B3026
:10439000CDE90594049637B14246394607A857F04F
:1043A000F7F88DF85A80164E002396F8EE9718937A
:1043B000B9F1000F19D196F8ED07642201A902FBAB
:1043C000006000F5FE6057F0E3F8012386F8ED97F2
:1043D00086F8EE37236843B143463A4629462046DD
:1043E0001AB0BDE8F0471AF0EDBD1AB0BDE8F0878D
:1043F0000523C3E70223C1E70C540024702A0024DC
:10440000604C00249FED747A07EE901A20EE070AA4
:10441000F8EE677A27EE800AFDEEC07A17EE903A42
:104420002033402B00F2C880DFED6C7AB4EEE70A4F
:10443000F0EE407AF1EE10FA0CDD9FED696ADFEDE7
:10444000696AB0EE677A77EEC67AB4EEE67AF1EE94
:1044500010FAF6DC9FED647AF4EEC77AF1EE10FA0A
:104460000CD59FED5F6ADFED616AB0EE677A77EE9B
:10447000867AB4EEE67AF1EE10FAF6D49FED5C7A25
:10448000F4EEC77AF1EE10FA40F386809FED537A8E
:1044900077EE677A67EEA75A9FED565A9FED566AF8
:1044A000B6EE007ADFED556AA5EE856A27EEA55ACD
:1044B000E5EE866AE5EE267A27EE877ADFED4C6A2E
:1044C00070EE267ABDEEE76A16EE103A2033402BE6
:1044D0006FD8B4EEE60AF1EE10FA0CDDDFED405ACB
:1044E0009FED406AF0EE676A77EEE57AF4EEC66A11
:1044F000F1EE10FAF6DCDFED3C6AF4EEE67AF1EE6E
:1045000010FA0CD5DFED365A9FED386AF0EE676A87
:1045100077EEA57AF4EEC66AF1EE10FAF6D4DFED86
:10452000346AF4EEE67AF1EE10FA48DDDFED2B6A3C
:1045300076EEE77A67EEA75ADFED2E4A9FED2E6AF8
:10454000B8EE005ADFED2D6AA5EEA46A67EEA54A23
:10455000E5EE866AE4EEA67A67EE857AC7EE206A13
:104560000023836143610362B7EE006AC36176EEA4
:10457000865A76EE666A86EE257A67EE277A80EDB1
:10458000007A66EE876A80ED027AC0ED017AC0EDAE
:10459000037AC0ED046A70479FED197AF4EEC77A8A
:1045A000F1EE10FA7FF576AF9FED0F7A77EE677A2E
:1045B00070E7DFED147AD1E79FED127A7EE7DFED49
:1045C000106AF4EEE67AF1EE10FAB3D5DFED066A82
:1045D00076EEE77AAEE700BF27D4D236DB0F49404C
:1045E000DB0FC940E4CB1641DB0F49C0E4CB16C159
:1045F000DB0FC93F92E741B99730083C15A82ABEA6
:10460000DB0FC9BF00000000F0B401282E4C2F4979
:104610004CF250372E4D08BF0421D4F8CC6C04293D
:1046200011D0D5F8102121EA020212F0040F0CBFBC
:104630000123002363B1D4F8CC3C9B1BBB42EED9D1
:104640000320F0BC70472B69C3F38003002BF2D129
:10465000012810D01E491F48D1F81021024224D150
:10466000D1F81021D20313D54FF480321846F0BC94
:10467000C1F814217047164A164C116921420AD11B
:104680001169C90304D54FF4803118465161D8E748
:104690001846F0BC7047104B104C1940D4F87038D5
:1046A0000B43C4F870385161CBE70C4C01200A4B26
:1046B0001A40D4F87038134343F00043C4F87038FC
:1046C000C1F81421F0BC7047683B0024040000804E
:1046D000002000520000EE150000EE17604C002490
:1046E000F8B5294E96F86C38012B4AD000F1784382
:1046F000012705460C46B3F5801F86F86C784FF00D
:1047000000032CD30220C6F87038FFF77DFF10BBE2
:104710001E4A0227D2F80C313B43C2F80C31214625
:10472000BFF36F8FBFF34F8F2A1B20340B688B5062
:104730000431A142FAD1BFF36F8FBFF34F8F3846D8
:10474000FFF762FF012F114A16D0D2F80C3123F087
:104750000203C2F80C31002386F86C38F8BD3846E5
:10476000C6F87038FFF750FF0028F4D1074AD36825
:1047700043F00203D360D2E7D36823F00203D3608F
:10478000E9E70220F8BD00BF604C00240020005281
:104790000C480D4BD0F88C1810B48A1E0B4C2231EB
:1047A000C0F87C38B0F8A6381B01A4FB03C3DB08B3
:1047B000A3F5B06322F8023F9142F3D15DF8044BB8
:1047C000704700BF604C00248D320608CDCCCCCCA5
:1047D00070B5084C251D2E4614F8010B34F000FD71
:1047E00028B10378B44205F8013BF5D170BDFF2331
:1047F000F8E700BF285500242DE9F0471C4F01269B
:104800004FF03C094FF0000807F10805B24617F8D1
:10481000010B40F09FFE044690B180F80690C671EF
:10482000FB7803F07F02012A17D013F0800F204697
:104830000CD185F8048041F0A3F985F805802C603F
:1048400001360835052EE2D1BDE8F08785F804A0D1
:1048500041F09CF985F805A0F1E71B0605D401217C
:10486000204641F069F8FB78DFE741F08FF9F6E781
:1048700030550024654B2DE9F04F4FF0010985B00C
:1048800003F10C0ADFF8A0B1984618F8016B002E6E
:1048900000F0B080350906F00F02013D062D00F250
:1048A000AC800BEB4503B3F8800040FA02F414F03F
:1048B000010400F0A68001235D44554C9340013B68
:1048C000184053F045FC95F890300422184404EB4E
:1048D000C004CAF8144084F80790A271002303E0D2
:1048E0000133152B00F0868003EB430249495D003C
:1048F000895CB142F4D1484B1A4492F8E11800297E
:1049000000F0828030463AF02FF80746006852F0F7
:10491000A9F979793AF066F8017800296AD13E4B15
:1049200004222B4483F8219983F82029002C44D0B9
:1049300023683A4A387A1A440290920A0BEB4202F0
:10494000B2F89800FCF708FBB4F804C02268BCF188
:10495000000F32D00397012303FA01FE1CEA0E0F69
:1049600026D0CC0801F007030F25029F02EB840438
:104970009B00266A48009D4007FA03F3022726EAB7
:10498000050603253343854007FA00F023621368C8
:1049900023EA050318431060936823EA0503936034
:1049A000536823EA0E035360D36823EA0505D560F4
:1049B00001313CFA01F3CED1039F194C09F10109F1
:1049C000184A0025B4F8FA385FFA89F9B4F8F848BB
:1049D000504639460AF1180AB2FBF3F3CDE9004517
:1049E0009BB232F05BFA0123B9F1090F0AF8073CD8
:1049F0007FF44BAF05B0BDE8F08F0024CAF8144037
:104A00006CE7CAF8144069E70B68FFDE5C550024C8
:104A1000B444002448440024683B00240000FEA75E
:104A2000604C002440420F00E8B80908974B2DE97C
:104A3000F04793F8C82982B00190002A40F0208105
:104A400093F8EC29B7EE007AB3F8F089012107EE6C
:104A5000902AB3F8EE09F0EE475A08FA01F5B8EEDD
:104A6000E76ADFED8B6A07EE900AB3F8EA09894C32
:104A70008542E6EE665AA6EE267A83F8C819F8EE65
:104A8000E77AB8BF054604F60C4104F60840AFB219
:104A900004F5416367EEA67AA4F8148CA4F8187C98
:104AA000C0ED005A81ED007AC3ED007A002A00F0D3
:104AB000E480DDED017AADB29FED770AF8EE677A1A
:104AC0006D00764E80EE270A54F056FA8246B0FB0F
:104AD000F5F5012DB8BF0125EDB2B0FBF5F39BB2A2
:104AE00084F81C5C00EE103ABBEEED0A86ED000A7D
:104AF00054F042FA6A4B06F10C01DFED6A6AA3FB3F
:104B00000A3ADFED690A9FED696A00234FEADA0A83
:104B10009FED671ADFED675A07EE90AADFED661A80
:104B20009FED662AF8EEE77ADFED652A9FED653A9C
:104B3000DFED653A86EEA77AB8FBF0F00228B8BF41
:104B4000022084F8240C86ED027A07EE903AB8EE43
:104B5000E77AF0EE467AE7EE207AFDEEE76A16EEA7
:104B6000902A2032402A00F28580B4EEC17AF1EE1C
:104B700010FA0CDDDFED556A9FED557AB0EE675AFD
:104B800077EEE67AB4EEC75AF1EE10FAF6DCF4EE00
:104B9000E57AF1EE10FA0CD5DFED4C6A9FED4D7A17
:104BA000B0EE675A77EEA67AB4EEC75AF1EE10FA75
:104BB000F6D4F4EEC67AF1EE10FA53DD73EEE77A2E
:104BC00067EEA76AB0EE424AB7EE007A67EEE64AB1
:104BD000A6EEA14A77EE677AB0EE627AB6EE005A98
:104BE000A6EE847AE4EE877A67EE857A0133E1EC0B
:104BF000017A202BA9D107EE905AB7EE006A364A07
:104C000041F2D021F8EEE76A07EE907A625002F1A5
:104C1000280702F1A80041F2CC2686EE267A41F25E
:104C2000DC2241F22D112D4BA0504FF0100CA7515A
:104C300041F2D82041F2C8272026F8EE677A41F2E7
:104C4000D4226554142124F807C0C3EDAC7AC3ED17
:104C5000AD7AC3EDAE7A2652A15283ED007A02B04E
:104C6000BDE8F087F4EEC37AF1EE10FA48BF75EEB6
:104C7000E77AA5E7F6EE007AB8E7194B1A7018E75D
:104C8000044C94F81C5CB4F8187CB4E7604C002425
:104C90000AD7233C1400002000247449340C00205F
:104CA000ABAAAAAADB0FC9413C8C4F3EDB0FC93F20
:104CB0000100F840DB0F49C092E741B99730083C4A
:104CC00015A82ABEDB0FC9BFDB0F4940DB0FC94067
:104CD000E4CB1641E4CB16C190BE09084411002074
:104CE00000000020F0B5264C83B0B4F8F859A58533
:104CF000E5B994F8F40940F02DFC94F8F529206307
:104D0000003A18BF012284F82E2048B194F8F61911
:104D10002B220029C28014BF1121012140F00CFE7A
:104D2000002003B0BDE8F0403EF0C4B994F8F47937
:104D300000222B21384639F083FE0646384640F0E3
:104D400009FC00B10EB903B0F0BD2B22A06400270E
:104D5000C280317AFCF7BCFB0A4AA4F8FA59314602
:104D600004F134000197B2FBF5F3C3F34F059BB296
:104D7000009532F093F8636B1F6084F84570E2E7AA
:104D8000604C002440420F002DE9F84F254B0026CF
:104D900093F8082A03F6FF1703F61C2483F8FC296E
:104DA0005FFA86FB4FF0010917F8010F01360BEB94
:104DB000090A49464FF000085FFA8AFA524639F06C
:104DC0003FFE054640B3387804F80E8C04F80D8C8D
:104DD00004F80FBC04F8109C44F8045C40F0BAFBE3
:104DE00018B180F8069080F807A0297AFCF770FBCC
:104DF0000D4A0021284651F0B3FE0C4B221D2146DE
:104E0000236028460A4BC4E9013851F04FFD424661
:104E10006979286831F0ACFF082E04F11C04BFD179
:104E2000BDE8F88F604C002440420F00256E070853
:104E3000AD53070870B52C4C00222C4B022194F87E
:104E4000340BC4F82C3BC4F8EC2AC4F8F02AC4F89C
:104E5000F42AC4F8282BA4F8302B39F0F1FD0028EF
:104E600040D0234B0546066803F1C0015A7C12B1BD
:104E70005A6896422BD018338B42F7D1002394F80E
:104E8000340BC4F8185A84F80C3A40F063FB08B1AC
:104E90000223C380297A0026FCF71AFB2846154A0C
:104EA000002151F05DFE144A1448154B111FC4F83F
:104EB0001C0A2846C4F8203AC4F8246A51F0F6FCCB
:104EC000324669792868BDE8704031F051BF3046FC
:104ED00051F0EEFAB36A0B4A0133B0FBF3F082F8FB
:104EE0000003CBE770BD00BF604C002400FFFF0053
:104EF0004800002040420F0080560024D553070888
:104F000071550708000000242DE9F04F644EC022BF
:104F100083B005460C4606F13400002156F0AAFB8A
:104F2000604B93F8352B8AB95F4DD5F80433002BCD
:104F300000F099800022012183F82C4083F82D1085
:104F40001A6383F82E2003B0BDE8F08F93F8363B48
:104F50006BB9564B2846544D214693F8C828003A61
:104F600018BF0122FCF778F8C5F80403DDE7DFF885
:104F700068C106F1F407DFF834A14B4D9AF8CAE88E
:104F8000BCE80F000FC7BCE80F000FC7BEF100035D
:104F900018BF01239CE8070085F808339AF8C63843
:104FA00087E80700072B424AC6F80C2148D9082B8E
:104FB00002D1404BC5F80C333F4B4FF000083F4A3D
:104FC000CDE900251D465FFA88FB44454FF00301FB
:104FD0000BF101092FDD009B5FFA89F913F8017BC2
:104FE0004A463846009339F02BFD034638461F46A3
:104FF000002B4BD040F0AEFA686120B14FF00303B4
:1050000080F8079083719AF8C7389AF8C628002B61
:1050100038D1FB795946384608F101084EF0A6FD13
:10502000002833D04FF00103B8F1080F05F118053F
:1050300005F8073CC7D1019D214BC5F8043374E73F
:10504000042BB9D99AF8C9381E4A012BC5F80C238C
:1050500006D0022B08BFBEF1000F0CBF01230023B6
:1050600085F81033A8E7184E184C0FCE0FC40FCE9A
:105070000FC496E80700A4F1200384E80700C5F8F0
:10508000043360E7FB7983F00103C3E71049002391
:10509000104A019DC6F81011C6F81821CDE700BFCF
:1050A00014000020604C00240C110020683B0024F8
:1050B0002DE308082D33000048000020334400246D
:1050C0000801002061330000E4BF0908985700245C
:1050D000E9440808E1440808B8BF090870B5694CFC
:1050E00094F8A00840F036FA94F8A16860B12D2336
:1050F00005462021C38040F01FFC0A2039F0E0FF64
:10510000284640F08BFD18B9D4F86C3BDA0100D585
:1051100070BD013E092EFBD894F89F58D5B94020A8
:1051200039F070F90028F3D090F9043094F875182C
:10513000092BC8BF143B0A29234493F8885700F071
:10514000938093F8933794F89E28002A08BF1D4651
:10515000002DDDD0284640F0FDF9054600287BD023
:105160002D230121C38040F0E7FB0121084640F0D8
:105170003BFD2B68AA889A613C203DF0C5FD0021CB
:10518000012040F031FD94F8A1387BB30026217F47
:10519000206AC94301F0010140F0FEFC217FA06AB2
:1051A00081F00401C1F3800140F0F6FC7820002D6D
:1051B00032D0AB8801362A681B04936139F080FF36
:1051C000217F206A01F0010140F0E6FC217FA06A06
:1051D000C1F3800140F0E0FC2B68AA8878209A6136
:1051E00039F06EFF94F8A1389E42D0DB94F89F38D6
:1051F00053BB94F8A038002B8AD194F8A238012B25
:1052000086D1D4F86C3B13F0807381D184F8A13837
:10521000BDE870404AF0E2BA7820013639F050FF1C
:10522000217F206A01F0010140F0B6FC217FA06AD5
:10523000C1F3800140F0B0FC782039F041FF94F8D0
:10524000A1389E42A3DBD1E732203DF05DFD284628
:10525000002140F071FBCCE7012140F06DFB012102
:10526000084640F0C1FC87E7D4F8703B5B057FF54A
:105270004FAF12F015FC00287FF44AAF002D7FF4E9
:1052800069AF45E7604C00242DE9F0411D4C002337
:105290004FF0050894F8772B04F6743704F12005D5
:1052A000227717F8010B5E1CF0B92860032E05F178
:1052B00004053346F5D1217F206AC94301F001017D
:1052C00040F06AFC217F606A81F00201C1F3400175
:1052D00040F062FC217FA06A81F00401BDE8F0414A
:1052E000C1F3800140F058BC40F034F90121F3B221
:1052F000286010B180F80680C371286840F01CFB5C
:10530000D4E700BF604C0024094BD3F8780BD3F8E6
:105310007C2BD3F8803B904202DC114602460846C3
:10532000984204DD9A42B8BF1A461046704770474B
:10533000604C00240B6810B414681B1B0360546895
:105340004B681B1B5DF8044B43608B6892689B1A8B
:10535000836070472DE9F047041E0D4612DB092CCF
:1053600026DC0B46814A82480021A0FB046059706C
:10537000C00800EB8000A4EB4000125C28461A70C5
:10538000BDE8F08764422D23092C01F8013B24D8A5
:10539000764A774B0020A3FB046348702846DB085D
:1053A00003EB8303A4EB4303D35C0B70BDE8F087EE
:1053B0006F4B632CA3FB04264FEAD60621DC0B4679
:1053C0006A4A6B49A1FB0601C90801EB8101A6EB02
:1053D0004101515C03F8011BC5E7654A632CA2FB40
:1053E00004364FEAD60637D8604A614BA3FB060362
:1053F000DB0803EB8303A6EB4303D35C01F8013B1B
:10540000C7E7A3FB0627B4F57A7F4FEAD7070DD28B
:105410000B46564A5649A1FB0701C90801EB810119
:10542000A7EB4101515C03F8011BCAE7A3FB072866
:1054300042F20F7294424FEAD80836D80B464B4AD4
:105440004B49A1FB0801C90801EB8101A8EB41010F
:10545000515C03F8011BDDE7A2FB0637B4F57A7F48
:105460004FEAD7070CD2414A414BA3FB0703DB08A5
:1054700003EB8303A7EB4303D35C01F8013BB4E7E1
:10548000A2FB073942F20F739C424FEAD90921D897
:10549000364A374BA3FB0903DB0803EB8303A9EB75
:1054A0004303D35C01F8013BDEE7A3FB0829314A43
:1054B00094424FEAD90921D80B462C4A2C49A1FB2A
:1054C0000901C90801EB8101A9EB4101515C03F815
:1054D000011BB5E7A2FB093A264B9C424FEADA0AC8
:1054E00021D8224A224BA3FB0A03DB0803EB8303E8
:1054F000AAEB4303D35C01F8013BCAE7A3FB0923F2
:105500001D4A94424FEAD30A21D80B461849174A3C
:10551000A1FB0A01C90801EB8101AAEB4101515C21
:1055200003F8011BCAE7A2FB0A38134B9C424FEA5F
:10553000D80813D80E4B0D4AA3FB0803DB0803EB76
:105540008303A8EB4303D35C01F8013BCAE70A22BB
:10555000BAFBF2F04AF004FE0346D7E70A22B8FB92
:10556000F2F04AF0FDFD0146E4E700BFE0360A082C
:10557000CDCCCCCC9F8601003F420F00344870B4A4
:1055800090F8843BA3F13001092958D800F68434FF
:1055900000F69330224612F8015FA5F13001092987
:1055A00004D88242F7D1002070BC7047141B022C33
:1055B0004BDD2848002101E010F8013B01EB81019F
:1055C000161A044603EB4103022EA3F1300303F045
:1055D000FF01F1DC204B03FB01F1A2424FF000037D
:1055E0000ED903EB830314F8016B5B00A242A3F115
:1055F0003003334403F0FF03F3D1184800FB03F3F7
:105600002E2D06D01648A0FB032370BC01EB93009F
:10561000704701320425002404EB84041078013D16
:10562000303864000928A4B2204401D8013284B281
:1056300015F0FF05F0D1642202FB0433E2E70021FC
:105640001D4600F684320B46DAE70021054CC4E71C
:10565000604C0024E55700248096980040420F00DB
:10566000ABAAAAAAE457002438B50D460446FF2188
:1056700000682A4655F0FEFF22682A44226038BDA1
:105680000C461646054683B53DF0DEFB20463DF050
:10569000DBFB0021204B0846002E08BF1E4640F0D1
:1056A000A3FA0021012040F09FFA28463FF0F0FEC7
:1056B000B0B10121002040F097FA28463FF0E0FE0B
:1056C000074620463FF0E0FE0028FAD03946204643
:1056D0003FF0E2FE3846B0470021084640F084FA29
:1056E00020463FF0D5FE0028DFD00121002040F009
:1056F0007BFA20463FF0C4FE0146284601913FF068
:10570000C3FE01990028F8D028463FF0C5FE0021CD
:10571000084640F069FAC8E7B5BF0708F0B50022AF
:1057200089B0DFF898C004AF13460A604A603E466D
:105730008A60CA600A610268C2F3855040FA03F4C5
:105740003546E40704D513F80C4005F8014B2E4606
:105750000133062BF2D1174DC2F303240023C2F309
:1057600005302C4405F5E76C33700DF1190694F8FB
:1057700030478DF8184040FA03F43546E40704D565
:1057800013F80C4005F8014B2E460133062BF2D1DD
:105790000023C2F3834506AC0846337002F00F03C2
:1057A0000549C2F303120097CDE901454AF028FFED
:1057B00009B0F0BDE8B8090808370A0810C00908A0
:1057C00070B5094C0546D4F8942B62B10026013619
:1057D0002D21D4F8940B41F0EFF8AE42F7DBBDE891
:1057E000704041F0A7BA70BD604C00242DE9F04F25
:1057F000CCB20021164685B00746084640F0F4F9C1
:105800000021012040F0F0F93FF070FE022E09D097
:10581000042E44F6C01818BF4FF49648072C06D93A
:1058200000200BE0FF2C4FF41648F7D10326C94D9A
:1058300095F8983B2BB90020C5F89C0B05B0BDE846
:10584000F08F032E15D0C44900220C44032194F894
:10585000CB0839F0F5F80028EDD0C04CC4F8A80BFF
:10586000C3799A07E7D4006851F0E8F941F2B433FC
:10587000E050BA4C41F2CB330022032195F8980B4B
:10588000E65439F0DDF8C4F8AC0F0028D3D0006836
:105890004FF0010A51F0D2F941F2B0334FF4806277
:1058A00004F6AC31E050032EAD4B04F66439C4F875
:1058B000702BC4F8643B4FF00303C4F8742B41F21F
:1058C000BC32A4F8683B4FF00003C4F8781B04F521
:1058D0007B61A35441F2B832C4F86C8B24F802A067
:1058E00041F2C432C4F8903BA35041F2C832C4F82C
:1058F000843BA35241F2CA32C4F8803BC4F87C1BFB
:10590000C4F88C3BC4F8883BA3540ED0D4F8A8BB91
:105910009BF804003FF01EFEC4F8A40B58461AF092
:105920004CFC514648461AF057FC32203DF0ECF949
:10593000002E5BD1D4F8AC0F22218A4A019051F09D
:105940000FF941F2D033884A09F66C010198E25010
:10595000324650F0ABFFD4F8A80B824A4FF6FF71E5
:10596000019051F0FDF831460198FBF7ADFA7F4AFE
:1059700041F2D43309F507610198E250324650F004
:1059800095FF4FF0060AC5F89C9B022E12D0D5F861
:105990009C0B3FF07DFD68B10121002040F024F90F
:1059A000D5F89C0B3FF074FD0146002840F09D8027
:1059B00040F01AF938463FF06BFD88B101214FF0F5
:1059C000050B4FF00008084640F00EF938463FF04E
:1059D0005FFD0146002840F09180012040F004F96D
:1059E000042ED4D005203DF08FF9CEE7012E09D149
:1059F000D4F8AC0F4146FBF77FF8D4F8A80BFBF7BF
:105A000089FABEE7022E09D1D4F8A80B1AF0C9FB17
:105A10004146D4F8AC0FFBF76FF8B2E7032E5CD128
:105A20004FF0000A41F2CC3340225148514604F86D
:105A300003A055F01FFEDFF840B18DF80FA0DFF88E
:105A40003CA19DF80F30072B09D9012149481AF0D4
:105A5000C3FB4146D4F8AC0FFBF74EF891E79DF835
:105A60000F3003EB43030BEBC30393F845306BB3E9
:105A70009DF80F3003EB43030BEBC3039B6C2BB37D
:105A80009DF80F20344B134493F8CB08F0B100225B
:105A9000032138F0D5FF0190C0B11AF082FB9DF8C8
:105AA0000F309AF8001003EB4303019A05EBC10095
:105AB0000BEBC3039B6CC0F8A03BD379DB0702D58B
:105AC000012380F8A43B01318AF800109DF80F30C3
:105AD0000133DBB28DF80F30B3E7042E7FF451AF02
:105AE000D4F8A80B1AF05DFB82E7D5F89C0B3FF0C9
:105AF000C7FC014638463FF0CFFC51E738463FF03F
:105B0000BFFC95F8EE3B01468BB9242803D14FF03A
:105B1000010385F8EE3B012E04D1384601913FF098
:105B2000BBFC0199D5F89C0B3FF0B6FC4EE7012B6E
:105B300006D14D280CBF0223002385F8EE3BEAE78F
:105B4000022B1DD13C280CBF0323002385F8EE3B1C
:105B5000E1E700BF604C0024683B00247819002472
:105B600028C0090840420F0065020608B5D505089F
:105B700000580024DC24002414000020442D0024BC
:105B8000032B10D10A2802D985F8EE8BC3E7042332
:105B900085F8E10B85F8E08B85F8E38B85F8E20B5F
:105BA00085F8EE3BB7E7042B09D195F8E23B85F881
:105BB000EF0B434085F8EEBB85F8E23BABE7052BE6
:105BC000A9D195F8E03B95F8E19B95F8E20B4B45A0
:105BD00009D25A1C48402B4485F8E20B85F8E02B8B
:105BE00083F8E41B97E78842CED195F8EF3B85F820
:105BF000EEABF42B8FD1B9F1000F8CD124213846B4
:105C000085F8EE9B3FF048FC4D2138463FF044FCC0
:105C10003E2138463FF040FC494638463FF03CFCC8
:105C2000F42138463FF038FCF42138463FF034FC8C
:105C3000032E12D0D4F8A85B284650F0F7FD494651
:105C4000284650F00DFE202128791AF099FA4A468C
:105C50004946D4F8A80B50F029FE0022D4F8AC0F26
:105C6000114650F023FE0120E8E500BF114A013043
:105C7000002302EBC000F0B4D0F874C70E4E3360BE
:105C80003361336233633364336533663367BCF146
:105C9000000F0DD090F8707757B13F0100240CEB46
:105CA0000403351910340FCBA74285E80F00F6D155
:105CB000F0BC7047E8B8090850580024F0B5154DFD
:105CC00083B00E4695F82835022B0DD1070AC4B2D1
:105CD000D5F85C070023012201A9384404F0E4FC54
:105CE000012806D003B0F0BDC0F3D41700F07F0444
:105CF000EEE795F82835022B019B04D133F81430D8
:105D0000336003B0F0BD53F8243023F070433360A8
:105D100003B0F0BD78190024D0E9011310B48B4210
:105D200090F91A2038BF0B46511C83600AD0144BDF
:105D3000FF2103EB021393F853256FF3000283F85E
:105D40005325817690F91B305A1C0FD00C49FF2443
:105D500001EB031191F85335C3F34502013A22EAEE
:105D6000E27262F3460381F85335C4760022436A37
:105D70005DF8044B114642614260036104F07ABC55
:105D80007819002438B50F4C034694F8771C04F5B5
:105D9000476084F8733C01F03F0101F10A058B1C58
:105DA000083184F8725C254484F8753C22F03CFB91
:105DB00085F86E0C94F8723C000A1C4484F86F0C51
:105DC00038BD00BF604C00242DE9F04FCD4C8DB0A4
:105DD0000027DFF83C93A4F26B2504F6A92A009073
:105DE00054F80B0C002800F0FE803FF051FB0646F3
:105DF000002800F0D281D9F8B43DE026A4F10B0BC5
:105E000044F8073C00237E4304F8033C54F80B0C91
:105E10003FF03EFB002800F0E68054F80B0C3FF00A
:105E20002FFB14F8023C80465A1E0B2A0DD8DFE8DF
:105E300012F01F003A004600530083009B00E2006E
:105E4000150134013F017101880124280CD0009A0A
:105E50003AB995F8062D824240F07981012204F882
:105E6000032C0D2BD2D186E0012304F8023CCDE7B0
:105E700000234D28C4F8C53084F8CD3084F8CE30E6
:105E800004D0582808D004F8023CBFE7022284F866
:105E9000C43004F8022CB9E7032304F8023C0223BF
:105EA00084F8C430B2E704233C2804F8023C0BD049
:105EB000B8F13E0F0CD0002304F8023CA6E70A23F9
:105EC0003C2804F8023CF3D1002304F8013C9DE790
:105ED000012304F8013C99E7D4F8C500AB19421C32
:105EE0000344C4F8C520022A83F86B8294F8CD00DD
:105EF00088EA000184F8CD1088D12378C02BDAD845
:105F00006278FF2A08D1052BD5D9012384F8C43043
:105F1000072304F8023C79E7A4F8C1200022C4F862
:105F2000C930934284F8C320C4F8C52014BF0523A8
:105F3000062304F8023C69E7D4F8C500AB19421CFB
:105F40000344C4F8C52083F86B8294F8CD00D4F8DC
:105F5000C93088EA00019A4284F8CD107FF456AF28
:105F6000062304F8023C51E794F8CD308342A2D1D5
:105F70000D2304F8023C14F801CCBCF1000F40F0F2
:105F8000ED80614B04AE0894ADF82CC0CDF80CC088
:105F90000FCB86E80F00D4F8C930324608A9D4F8F0
:105FA000D10023440993B4F8C130ADF8283094F8F7
:105FB000C3308DF82A3001238DF82E3003AB33F037
:105FC00045F948B1049B314694F8C42058460593DE
:105FD0004E4B049331F042FB0023039E04F8023C35
:105FE000002E40F0D2800137E034032F7FF4F8AE6A
:105FF0000DB0BDE8F08FD4F8C500AA194146431C86
:106000000244C4F8C53082F86B8294F8CD2094F82D
:10601000CE0088EA0202019384F8CD204AF09AF972
:10602000019B84F8CE00072B7FF4F0AEB4F8053066
:10603000C02B3FF640AFB4F80320C4F8C930A4F831
:10604000C120A27884F8C32000229342C4F8C5205E
:1060500014BF0823092304F8023CD7E6014694F84C
:10606000CE004AF077F994F8CD3084F8CE0088EA73
:106070000303D4F8C50084F8CD30AB19421C0344A7
:10608000C4F8C52083F86B82D4F8C9309A427FF4F3
:10609000BDAE092304F8023CB8E694F8CD30434085
:1060A00084F8CD3094F8CE3083427FF404AF57E7C4
:1060B000D4F8C500AA194146431C0244C4F8C530AF
:1060C00082F86B8294F8CE0001934AF043F9019B69
:1060D00084F8CE00052B7FF499AEB4F80120B4F813
:1060E0000330A4F8C1202278C4F8C93084F8C32052
:1060F00000229342C4F8C52014BF0B230C2304F8DC
:10610000023C83E6CB4E002430C10908B4D0002401
:10611000702A0024014694F8CE004AF01BF9AB190E
:1061200084F8CE00D4F8C500421C0344C4F8C5204E
:1061300083F86B82D4F8C9309A427FF467AE0C239F
:10614000A1E694F8CE3083427FF4B5AE10E7232861
:106150007FF487AE022204F8032C82E6BCF1010F23
:106160004FF0000602D004F8026C3CE7D4F8C930C6
:1061700008A8089423440993B4F8C130CDE90A660D
:10618000ADF828302FF0F0FFEDE754F80B0C3CF0A1
:106190005BFE54F80B0CB04725E714F8033C002BCA
:1061A0003FF421AFD9F8B42D54F8071C521A632AD2
:1061B0007FF619AF012B30D0022B7FF414AF54F8C7
:1061C0000B3C012285F81D0DC5F80C3DC5F8103DAE
:1061D000C5F8183D402385F8082D85F81C3D95F835
:1061E000673D0F4A003B0F48C5F8142D18BF012327
:1061F0000D4AC5F894AB82F81433C5F860AD40F091
:106200009DFD4FF4005038F0B1F9084840F08CFD86
:1062100085F8756D85F8766DE5E6FAF74DFE00BFF9
:106220008544080817370A080C1100204D370A0862
:1062300038B51E4C0968D4F87C5D0068491B1C4DBC
:10624000DFED1C6A00EE901AD4F8781DD5EDC17A06
:106250001C46F8EEE00A401A60EEA70A07EE900A24
:10626000F8EEE77A20EEA07AB1EE670AA7EEA77AF9
:10627000F1EEC77A67EEA67AFCEEE77AC2ED007A15
:106280004AF08CFA9FED0C7ADFED0C7AE0EE077A9B
:10629000FDEEE77A17EE902A002A02DBC4ED007AC1
:1062A00038BD48F6A0431344236038BD604C002439
:1062B000000000242C7D8E3FA00CB34500A00C46AE
:1062C00038B50A4C002501228021204638F086F896
:1062D00030B194F9040038F0B3F808B1006838BD63
:1062E00001350C34092DEED10020F8E7F8580024D0
:1062F00038B5041F00F1080554F8043FD81780EAA8
:1063000043001BF031FCA542F6D138BD054B0020FF
:1063100000214FF6FF72C3F8C003C3F8BC13C3F8E3
:10632000C42370470C1100202DE9F041BA4CDFED79
:10633000BB7A94EDF37A94F8AD332DED028BB8EE81
:10634000478A28EE278A002B45D094F81873002F2F
:1063500040F0B680B24E0025DFEDB28A4FF0000863
:1063600094F8D0332B41DB0712D594F8AC331BBB28
:10637000B4F8AE3307EE103A002F46D0B8EE477AA5
:10638000C8EE877A77EE887A88EE277A86ED027AE9
:1063900001352436042DE3D194F8B153B4F8B46335
:1063A000B5BB2FB994F8C83384F8D87384F8D433C4
:1063B000BDEC028BBDE8F081B4F8AE33301DD4F8EB
:1063C000CC1300EE103AB8EE400ACFB949F044FBC6
:1063D00094F81873DCE794F8AC1394F8C923B1FA75
:1063E00081F1D4F8B803B4F8AE5349092BF086FE16
:1063F00080B28542A4F8AE03A7D094F81873A9E739
:1064000055F06AFA94F81873C2E7C6F80480B5E745
:10641000854A94F8B233D2F8902D92F88320134332
:106420005ED1A5F1010194F8C923D4F8B803B1FAFB
:1064300081F149092BF062FE80B2A4F8B403002F69
:1064400061D194F8C83384F8D85384F8D433002841
:10645000AED007EE900A0123B8EE678A9D42DFEDC9
:10646000717A84F8DC33C7EE888A00F08B80022DC5
:106470009ED1D4F8CC13B0EE480A6C4849F0ECFA3F
:1064800094F8D833012B00F0C180022B90D1B0EEEC
:10649000480AD4F8CC13664849F0DEFA94F8D833A9
:1064A000012B00F0AE80022B82D1B0EE480AD4F866
:1064B000CC136048BDEC028BBDE8F04149F0CCBA8A
:1064C00094F8B153B4F8B463002D3FF471AF564A59
:1064D00094F8B233D2F8902D92F88320134304D06D
:1064E000002F7FF465AF3046ABE7A5F1010194F8CA
:1064F000C923D4F8B803B1FA81F149092BF0FEFDA4
:1065000080B2A4F8B403B0423FF452AF00283FF485
:106510004FAF94F8D833002B3FF44AAF07EE900A00
:10652000012BB8EE678ADFED3F7AC7EE888A47D045
:10653000022B7FF43DAFD4F8CC13B0EE480A3B48B1
:1065400055F0CAF994F8D833012B52D0022B7FF4BE
:106550002FAFB0EE480AD4F8CC13354855F0BCF94B
:1065600094F8D833012B47D0022B7FF421AFB0EE43
:10657000480AD4F8CC132F48BDEC028BBDE8F0419B
:1065800055F0AAB92C4A0021D2ED007A134678EED4
:10659000A76A43F8041F87EEA67A83ED017A78EEA6
:1065A000A76A0021996087EEA67A83ED037A77EED9
:1065B000A88A00221A6187EEA87A83ED057AF7E6A9
:1065C0001D4A1346F3EC017A78EEA76A87EEA67AA5
:1065D00083ED017AD2ED007A78EEA76A87EEA67A8B
:1065E00083ED037A77EEA88A87EEA87A83ED057AA1
:1065F000DEE6114A131DEDE70F4A131DD2ED007AB6
:10660000F0E70D4A131DD2ED007AD0E70A4A131DB8
:10661000D2ED007AC3E700BF0C110020BD378635EC
:106620002414002083F9223E604C0024EC14002046
:10663000101500203415002058150020012816D010
:106640002F4B93F86834012B2CD02E4BF6EE006ABA
:10665000BEEE007ADFED2C7A03EB800090ED000AAD
:1066600080FE660A80FE070A20EE270A7047274A46
:10667000F6EE006A224BBEEE007A02F6AC51DFED78
:10668000227A93F86C3491ED010A80FE660A80FE4E
:10669000070A20EE270A23B1B5EEC00AF1EE10FA80
:1066A00003DC70479FED1A0A704707EE903AB2F983
:1066B000961DB2F9AA3DDFED176AF8EEE77ACB1A1C
:1066C00007EE103AB8EEC77A27EE267AB4EEE77AEC
:1066D000F1EE10FAE6DA77EEC77AB2EE047AF4EE6B
:1066E000C77AF1EE10FADCD8B1EE047A67EEA67A3A
:1066F00030EE470AA7EE807AB0EE470A704700BF37
:106700000C1100200C5A002400004843604C002467
:1067100000000000CDCCCC3DF8B5784C40F603022B
:10672000B4F8B83D13402DED048BB0EE408A04D090
:10673000B0EE480ABDEC048BF8BD04EB4001B5EEA9
:10674000C00ADFED6F6AF7EE007AB1F9A85DBFEE1F
:10675000007AB1F9942DF1EE10FA6A4E4FEA800CEE
:10676000A2EB050206EB8001C8BF012700EE102A4C
:10677000D8BF4FF0FF37D1F87054B8EEC00A20EE02
:10678000260AB5EEC00AF1EE10FACCBF4FF0010EAA
:106790004FF0FF3E77FE877AEA1B18BF0122002DDB
:1067A00008BF0022002A48D106F58F63F0EEC06AC8
:1067B00093ED007AF4EEC76AF1EE10FA07DD774543
:1067C00008BF002D0CBF0122002200F08580002DA3
:1067D00041D0B0EE408A4C4BDFED4C8AD3ED006ADD
:1067E00097EE278A9FED4A7ADFED4A7A28EE268ACD
:1067F00088FE478A88FE278A002A61D196F8C0342D
:10680000984295D194F8BA3D262B91D1B2EE049AD4
:1068100020EE090A52F0B0FBB0EE480AA4F8BE5DC3
:10682000A4F8BC0D52F0A8FB28EE890AA4F8C00D0C
:1068300052F0A2FBA4F8C20D7AE706F58F62F0EEE3
:10684000C06AC1F8703492ED007AF4EEC76AF1EED6
:1068500010FA3FDC1A4630499FED306A01EB8001A7
:10686000D1ED077AF0EEE76AF4EEC66AF1EE10FABF
:106870002DDC9FED2B6A66EE866A2A4BF0EE408A8D
:10688000B7EE006A93ED005AFFEE005A67EE857A84
:10689000E6EEA78AF5EEC08AF0EEE87AF1EE10FA9D
:1068A000F4EE477ACCBF01214FF0FF3136FE256A66
:1068B000F1EE10FA01DD8F4215D00025002A9DD09F
:1068C0008444194B002203EB8C035A6096E7F7EEE1
:1068D000006AD2E77745BDD106EB0C03754601226D
:1068E000C3F870E473E7B0EE688A53ED017A0025CF
:1068F00097EE068A28EE278AE2E700BF604C002464
:10690000CDCCCC3D0C1100208815002000000000EB
:1069100000007A4400007AC4C00C0020FFFFF94355
:106920006F12033B8C1500209015002070B46F4C43
:106930000A7804F6AC5304EB80066D4D07EE902AFE
:1069400003EB8001D6F8C43DB8EEE76AD1ED006AEA
:10695000514207EE101A85FB0315DB17B8EEC77A14
:10696000C3EB651307EE903AF8EEE77AE6EE267A87
:10697000F4EEC77AF1EE10FA05D407EE102AF8EE1D
:10698000476A86FEE77A04EB400040F60101B4F85E
:10699000B82DB0F9943DB0F9A80D1142DFED556A5C
:1069A000A3EB000307EE903AF8EEE77AA7EEE67A5B
:1069B00006D0514B93ED000A70BC27EE000A7047D9
:1069C000B4F9943DB4F9962D002B4C484C49B8BF0E
:1069D0005B42002AD0ED017AB8BF52429BB290EDE3
:1069E000006A92B291F8C80487FE866A9342B8BFE3
:1069F000134607EE903AF8EEE77A67EEA67AE0BB28
:106A000001F2D443DFED3F5AD3ED006AF4EEE56ABC
:106A1000F1EE10FA61D5F7EE005A9FED3B4A9FED7B
:106A20003B5A01F2CC4175EEE65AD1ED004A75EEC3
:106A3000677A65EE845AE5EEA76A66EEA46ADFED32
:106A4000347AF4EEE76AF1EE10FA4BD9DFED314A11
:106A5000F7EE005A84EEA65AF0EE656AE6EE456A55
:106A6000C6FEE56AC6FEA76A2B4BD3ED007A67EE39
:106A7000277A70BCA7EEA60A704701F2CC439FEDBF
:106A8000245AD3ED005AF4EEC55AF1EE10FA21DD86
:106A900001F59A61D1ED004AF4EEC54AF1EE10FA23
:106AA00018DDDFED1E6A74EEE77AB7EE004A26EED7
:106AB000266AC7EEA46AC6EE257AC6FEC46AC6FE7A
:106AC000856A77EE847A66EEA76AC6FEC46AC6FE59
:106AD000856AC9E7F0EE456AC6E701F2CC41D1ED1F
:106AE000006AACE7F0EE676ABEE700BF604C0024C6
:106AF0001F85EB51CDCCCC3DD01500202C5A002465
:106B00000C110020AE47813F610BB63B00003443BF
:106B1000000000000000C842E41500200000C8C2C8
:106B20002DE9F04FDFF83C8098F8BA6D102E2DED6E
:106B3000048B83B000F06E85094D41F2C523002718
:106B400015F80390B9F1060F00F24E85DFE819F051
:106B5000EA05B10672050C00D5050304C60600BFA0
:106B600014000020604C0024F54C102E04F5D8626F
:106B700004F5D76304F5D96004F5DA61D2ED007A43
:106B800004F5DB6293ED007A04F2B463D2ED004ABF
:106B900004F5DD62D3ED000A04F2C463D2ED005ABD
:106BA00004F5DF6291ED004A67EE072AD2ED006A34
:106BB00004F5E162D0ED003A04F5DC61D3ED001A92
:106BC00027EEA73A04F2D463D2ED007A04F2BC6255
:106BD00091ED005A63EEA33A04F5DE6193ED002ACD
:106BE000E0EEA02A92ED001A04F2E46304F2CC6213
:106BF00091ED006A24EE044A04F5E06164EEA44AD3
:106C000093ED000AD2ED008AA1EE013AE1EEA13A3D
:106C100004F2DC6204F2047391ED007A25EE055A69
:106C200092ED008A65EEA55A04F2EC6067EEA77A51
:106C300004F2F461E2EE024A04F2FC6293ED002AEF
:106C4000A8EEA84A26EE066AD2ED001A66EEA66AFB
:106C500091ED001A27EE077AD0ED000AE2EE027AF3
:106C600004F23463B1EEE22A04F5C76204F5CA61A6
:106C700004F25C6904F5E36C04F5E26E04F5E4608B
:106C8000A8EE085AE0EE005AF1EEC32AA0EEA06A80
:106C9000B1EEE33A83ED002A04F23C63E1EE016ACF
:106CA000A1EEA17AF1EEC43AC2ED002A04F5C86261
:106CB000B1EEE44A83ED003A04F24463F1EEC54AD2
:106CC000B1EEE55AC2ED003A04F5C962F1EEC65ADA
:106CD00083ED004A04F24C63B1EEE66AC2ED004A6D
:106CE00004F25462F1EEC76A83ED005A04F5CB63F7
:106CF000B1EEE77AC1ED005A04F5E56182ED006A74
:106D000004F5E662C3ED006A04F20C7389ED007AC3
:106D1000DCED007A9EED007AD3ED004A27EEA76AFB
:106D200004F21C73D2ED007A04F2147267EE075A73
:106D3000D0ED006A67EEA77A91ED007A04F5CD6197
:106D400092ED005A04F2247293ED004A04F22C737F
:106D500066EEA66A27EE077AE4EEA45AD2ED004A60
:106D6000A5EE056A93ED005AE4EE046A04F5CC62E0
:106D7000A4EEA47A04F26463E5EE057AB1EEE55A76
:106D8000F1EEC65AB1EEE66AF1EEC76A82ED005A3C
:106D900004F26C62B1EEE77AC3ED005A04F5CE63FB
:106DA00081ED006AC2ED006A83ED007A00F0E887A9
:106DB00041F2C52315F8039009F101095FFA89F939
:106DC00005F8039095F8243C0F2B01F323800D2B3D
:106DD00004EB830103F1010C01F230800A4601F556
:106DE000C66102F23462D1ED007A92ED007AB4EE1F
:106DF000677AF1EE10FA05DDB5EEC07AF1EE10FA21
:106E000000F3B9870020DFED4F7A04EB8C0202F229
:106E10003462D2ED006AF4EE476AF1EE10FA08DD52
:106E2000F4EE676AF1EE10FA03DDF0EE667A5FFACF
:106E30008CF0D91C03F1020C0E29624600F3058187
:106E400004EB830202F23C6292ED007AB4EE667AC1
:106E5000F1EE10FA08DDB4EE677AF1EE10FA03DD18
:106E6000F0EE477A5FFA8CF004EB830202F5C86219
:106E7000D2ED006AF4EE476AF1EE10FA07DDF4EEA7
:106E8000676AF1EE10FA02DDF0EE667AC8B2591DBB
:106E900003F1040C0E29624600F3D78004EB830251
:106EA00002F2446292ED007AB4EE667AF1EE10FAE4
:106EB00008DDB4EE677AF1EE10FA03DDF0EE477A02
:106EC0005FFA8CF004EB830202F5C962D2ED006A2E
:106ED000F4EE476AF1EE10FA07DDF4EE676AF1EEC0
:106EE00010FA02DDF0EE667AC8B2D91D03F1060C85
:106EF0000E29624600F3A98004EB830202F24C6281
:106F000092ED007AB4EE667AF1EE10FA05DDB4EE99
:106F1000677AF1EE10FA00F34D8704EB830202F575
:106F2000CA62D2ED006AF4EE476AF1EE10FA0BDDA8
:106F3000F4EE676AF1EE10FA00F3378704E000BF61
:106F4000C00C00200000000003F1090103F1080C4F
:106F50000E29624679DC04EB830202F2546292ED60
:106F6000007AB4EE667AF1EE10FA05DDB4EE677AD7
:106F7000F1EE10FA00F3298704EB830202F5CB62ED
:106F8000D2ED006AF4EE476AF1EE10FA05DDF4EE98
:106F9000676AF1EE10FA00F3138703F10B0103F1B6
:106FA0000A0C0E29624650DC04EB830202F25C629A
:106FB00092ED007AB4EE667AF1EE10FA05DDB4EEE9
:106FC000677AF1EE10FA00F30B8704EB830202F507
:106FD000CC62D2ED006AF4EE476AF1EE10FA05DDFC
:106FE000F4EE676AF1EE10FA00F3F58603F10C0196
:106FF000012B0A4629DC04EB830202F2646292ED63
:10700000007AB4EE667AF1EE10FA07DDB4EE677A34
:10701000F1EE10FA02DDF0EE477AC8B204EB83021B
:1070200002F5CD62D2ED006AF4EE476AF1EE10FA95
:1070300009DDF4EE676AF1EE10FA04DD03F10D00EC
:10704000F0EE667AC0B203F10E0204F2844302F15C
:107050006C0103EB810C03EB82039CED007AD3ED12
:107060006B6AF4EE476AF1EE10FA07D5B4EE677A70
:10707000F1EE10FA02DDF0EE477AD0B20F2A02F1FB
:10708000010C00F0358404F2844303EB810103EB2F
:107090008203D1ED006A93ED6D7AF4EE476AF1EE6A
:1070A00010FA05D5B4EE677AF1EE10FA00F3CC864B
:1070B0000E2A02F1020300F01B8404F2844202EB68
:1070C000830191ED6C7AD1ED6B6AF4EE476AF1EED3
:1070D00010FA05D5B4EE677AF1EE10FA00F3BE8629
:1070E0000F2B03F1010200F0038404F2844303EB4D
:1070F000820191ED6C7AD1ED6B6AF4EE476AF1EEA4
:1071000010FA05D5B4EE677AF1EE10FA00F3AF8607
:107110000F2A02F1010300F0EB8304F2844202EB38
:10712000830191ED6C7AD1ED6B6AF4EE476AF1EE72
:1071300010FA05D5B4EE677AF1EE10FA00F3A086E6
:107140000F2B03F1010200F0D38304F2844303EB1D
:10715000820191ED6C7AD1ED6B6AF4EE476AF1EE43
:1071600010FA05D5B4EE677AF1EE10FA00F39186C5
:107170000F2A02F1010300F0BB8304F2844202EB08
:10718000830191ED6C7AD1ED6B6AF4EE476AF1EE12
:1071900010FA05D5B4EE677AF1EE10FA00F38286A4
:1071A0000F2B03F1010200F0A38304F2844303EBED
:1071B000820191ED6C7AD1ED6B6AF4EE476AF1EEE3
:1071C00010FA05D5B4EE677AF1EE10FA00F379867D
:1071D0000F2A02F1010300F08B8304F2844202EBD8
:1071E000830191ED6C7AD1ED6B6AF4EE476AF1EEB2
:1071F00010FA05D5B4EE677AF1EE10FA00F36A865C
:107200000F2B03F1010200F0738304F2844303EBBC
:10721000820191ED6C7AD1ED6B6AF4EE476AF1EE82
:1072200010FA05D5B4EE677AF1EE10FA00F35B863A
:107230000F2A02F1010300F05B8304F2844202EBA7
:10724000830191ED6C7AD1ED6B6AF4EE476AF1EE51
:1072500010FA05D5B4EE677AF1EE10FA00F34C8619
:107260000F2B03F1010200F0438304F2844303EB8C
:10727000820191ED6C7AD1ED6B6AF4EE476AF1EE22
:1072800010FA05D5B4EE677AF1EE10FA00F33D86F8
:107290000F2A02F1010100F02B8304F2844303EB77
:1072A000810292ED6C7AD2ED6B6AF4EE476AF1EEF0
:1072B00010FA05D5B4EE677AF1EE10FA00F32E86D7
:1072C0000F2901F1010300F0138304F2844202EB61
:1072D000830191ED6C7AD1ED6B6AF4EE476AF1EEC1
:1072E00010FA05D5B4EE677AF1EE10FA00F31F86B6
:1072F0000F2B03F1010200F0FB8204F2844303EB45
:10730000820191ED6C7AD1ED6B6AF4EE476AF1EE91
:1073100010FA05D5B4EE677AF1EE10FA00F3108694
:107320000E2A40F0E58204F5CE6204F26C6392ED21
:10733000007AD3ED006AB4EE667AF1EE10FA40F30B
:10734000D782B4EEE77AF1EE10FA40F3D182F0EE94
:10735000477A0F20CFE2EA4B1B78002B00F0EE8437
:1073600041F2C629E74CD5F8B01C15F8093004F2F3
:10737000844204F56A7054ED297A03EBC30C54ED92
:10738000270A02EB830300EB8C0093EDAC0AD0F8E4
:107390001CB0D0F820A020EE270AD0ED053A90EDE1
:1073A000064AFDF72FF8C0F81CB004F21443C0F8E9
:1073B00020A0C0ED053A80ED064A15F809C054ED4D
:1073C000287A02EB8C02D5F8B01C0CEBCC0092EDC5
:1073D000AC0A03EB800020EE270AD0F814B0D0F8F6
:1073E00018A0D0F81C90026AFDF70CF8102EC0F817
:1073F00014B0C0F818A0C0F81C90026200F00D850F
:1074000041F2C62CC04B41F2C52E15F80C2015F8E0
:107410000E0001320130A3FB021305F80E0003F445
:10742000FF7101EB5303D21A05F80C20DFF8EC9240
:1074300099F8003003F5937CC3F120030CEB421C58
:1074400013F0FC0FC3F385005FFA83FE04EB8C0C92
:1074500000F0D98401300CF11003A9F2045104F2B8
:1074600044624FEA001A0CEB001013ED026A10336D
:1074700011ED027A103253ED076A103153ED057A9F
:1074800026EE076A51ED074A13ED087A834211EDA3
:10749000085A66EEA46A51ED055A27EE057A02ED08
:1074A000066A67EEA57A42ED076A02ED087A42EDB8
:1074B000057ADAD19548AAF1100300F2B4629C442F
:1074C000C11813441EF003021BD0DCED007A013A10
:1074D00091ED007A67EE877AC3ED007A11D0DCED8A
:1074E000017A012A91ED017A67EE877AC3ED017A7C
:1074F00007D0DCED027A91ED027A67EE877AC3ED70
:10750000027A99F800C0BCF1000F66D041F2C623A0
:1075100000EB8E005FEA9C09EB5C04EB8E0E04EB43
:10752000C3140EF2346E04F5936435D009F10109E9
:1075300004F1100300F110010EF110024FEA091AD4
:1075400004EB091913ED026A103311ED027A1032BF
:1075500053ED076A103153ED057A26EE076A51EDB7
:10756000074A13ED087A4B4511ED085A66EEA46AF6
:1075700051ED055A27EE057A02ED066A67EEA57A07
:1075800042ED076A02ED087A42ED057ADAD1AAF1F6
:1075900010031C4418449E441CF0030C1DD0D4ED71
:1075A000007ABCF1010C90ED007A67EE877ACEED9F
:1075B000007A12D0D4ED017ABCF1010F90ED017A7E
:1075C00067EE877ACEED017A07D0D4ED027A90ED9E
:1075D000027A67EE877ACEED027A102E00F0838071
:1075E00041F2C52315F8039009F10109484B41F216
:1075F000C522A3FB0913A9EB030103EB51039B086D
:10760000C3EBC303A9EB0303AB5403B0BDEC048B82
:10761000BDE8F08F37F0F2FD3E4D98F8BA6D41F2BB
:10762000C523074615F80390102E08BFA8F8BC9D87
:10763000FFF788BA384CDFF8E8E0B0EE006AD4ED26
:10764000005A41F2C823DEED007AF6EE006AE85AED
:1076500041F2DC2377EEA77A0138E958B0EE664AAA
:107660000EF18C03B0EE677A04EBC002E5EE867A89
:107670001031083A95EE867A67EEA67A27EE267ADA
:10768000CEED1F7A8EED207AD2ED036A0138D2ED6D
:10769000027A01F1080153ED215AA2F1080253EDDB
:1076A000224A03F1080335EEE67A11ED036A37EE5C
:1076B000E45A77EEA47A76EEA56A51ED045AA6EE66
:1076C000057AE5EE857AA5EEE67AE6EE267A27EEED
:1076D000047A67EE847A03ED037A43ED047AD3D11A
:1076E000102E7FF47DAF37F089FD41F2C523C01B1A
:1076F00015F80390A8F8BE0D76E7024CFFF762BBC1
:1077000000000020C00C0020ABAAAAAA400C002058
:107710002549922414000020F41200205411002066
:10772000F812002041F2C8236F4C41F2CC22EB5AF0
:1077300004F2346AAA5859080AEB8309DB084FEAB5
:1077400081000AEB810A00F0A48003F1010C1030E3
:107750000AF1100304F244640AEB0C1A484402F1E3
:10776000100E09F1100C5CED047A103314ED041ABC
:107770000EF1100E50ED041A103453ED086A71EE3C
:10778000278A5CED032A31EE671A10ED032A36EEE4
:10779000A18A5CED013A71EEE61A13ED064A0CF18E
:1077A000100C53ED054A10305CED065A13ED075AE4
:1077B00050ED067A10ED057A35EE020A14ED063A20
:1077C00032EE455A14ED076A74EE270A54ED056A45
:1077D00077EEC47A44ED088A36EE229A36EEA32A72
:1077E00036EE626A73EE258A04ED079A74EE872AF4
:1077F00004ED052A37EE647A44ED068A73EE655A85
:1078000043ED052A76EEE36A03ED088A03ED070AE5
:1078100043ED060A53455EED074A1EED084A66EE43
:10782000242A24EE453A61EE843A24EEC12AE1EEA0
:10783000042AA6EE042AB0EE434AB0EE636AA1EE33
:10784000A44A4CED082AA5EE246A0CED072A00EDA7
:10785000084A00ED076A1EED056A1EED065A26EE7F
:10786000863A66EE653A27EE854A65EE474AE6EEC9
:10787000853AA5EE853AA7EE064AE7EE864A0CED74
:10788000063A4CED053A00ED054A40ED064A7FF414
:107890006AAF89B215480191F8F7B2FB41F2CC23E7
:1078A00001994846EA58F8F7ABFB102E7FF498AEE2
:1078B00019E741F2D42341F2D0220C4CAA58E95ADC
:1078C00020464FF071FE98F8BA6D102E00F0AE828F
:1078D00041F2C522AB5C0133AB54ACE641F2C623A6
:1078E000014CEA5CA2E500BFC00C0020F4120020AD
:1078F000002800F00582431E012B40F3DF8204F2D2
:107900008443A0F1020C03EB800191ED6B7A0A46EF
:10791000D1ED6A6AF4EEC76AF1EE10FA00F38F80D7
:10792000BCF1010F00F08B8092ED697AC11EB4EEBC
:10793000E67AF1EE10FA00F35982012900F056823E
:10794000D2ED686A011FF4EEC76AF1EE10FA76DC38
:10795000012974D092ED677A411FB4EEE67AF1EE18
:1079600010FA00F34382012900F040821346821F7F
:10797000D3ED666AF4EEC76AF1EE10FA5FDC012A15
:107980005DD004F28443C11F03EB800292ED657A5F
:10799000B4EEE67AF1EE10FA00F32882012900F045
:1079A0002582D2ED646AA0F10801F4EEC76AF1EE17
:1079B00010FA44DC012942D092ED637AA0F109016A
:1079C000B4EEE67AF1EE10FA00F31082012900F02D
:1079D0000D82D2ED626AA0F10A01F4EEC76AF1EEFF
:1079E00010FA2CDC01292AD01346A0F10B0293EDEA
:1079F000617AB4EEE67AF1EE10FA00F3F781012A2B
:107A000000F0F48104F28443A0F10C0103EB800246
:107A1000D2ED606AF4EEC76AF1EE10FA0FDC0129CC
:107A20000DD01346A0F10D0293ED5F7AB4EEE67A25
:107A3000F1EE10FA00F3DA81022A07FE267A431CDF
:107A40000E2B00F3388204F2844200F1020E02EBA6
:107A5000800CDCED6D6A61469CED6E6AB4EEE66A00
:107A6000F1EE10FA00F39280BEF10F0F00F08E805D
:107A7000D1ED6F6A00F1030CB4EEE66AF1EE10FA94
:107A800000F18280BCF10F0F7ED091ED706A00F1A1
:107A9000040CB4EEE66AF1EE10FA77DCBCF10F0FDD
:107AA00074D0D1ED716A00F1050CF4EEC66AF1EE06
:107AB00010FA69DCBCF10F0F66D00A46811D92ED09
:107AC000726AB4EEE66AF1EE10FA5FDC0F295DD05F
:107AD00004F2844200F1070C02EB8001D1ED736ADD
:107AE000F4EEC66AF1EE10FA4EDCBCF10F0F4BD08B
:107AF00091ED746A00F1080CB4EEE66AF1EE10FA4A
:107B000044DCBCF10F0F41D0D1ED756A00F1090CD6
:107B1000F4EEC66AF1EE10FA36DCBCF10F0F33D08A
:107B200091ED766A00F10A0CB4EEE66AF1EE10FA15
:107B30002CDCBCF10F0F29D00A4600F10B01D2ED6D
:107B4000776AF4EEC66AF1EE10FA1DDC0F291BD03D
:107B500004F2844200F10C0C02EB800191ED786A92
:107B6000B4EEE66AF1EE10FA10DCBCF10F0F0DD0A6
:107B70000A4600F10D01D2ED796AF4EEC66AF1EE23
:107B800010FA01DC0E2901D0F0EE466A87FE667A13
:107B9000C7EE878A41F2C62104F2844215F801A09B
:107BA0000AF1AC0BB2EE007AF7EE007A02EB8B0230
:107BB00092ED008AC8FEC78AC8FEA78A04F28442F2
:107BC00007EE900ADBB202EB8001F8EEE76A0F2BBA
:107BD00091ED6C7A27EE077A66EE876A6ED802EB33
:107BE000830207EE903A012892ED6C6AF8EEE77A8C
:107BF00026EE066AE6EE276A37EE067A5ED8B5EE1E
:107C0000C07AB5F8183CF1EE10FA70DD86EE879A6E
:107C1000CF4A92ED007A29EE077AB5F8142C07EED8
:107C2000902AF8EE677AF4EEC77AF1EE10FA05DCE6
:107C300007EE903AF8EE677AC7FEC77AC54B77EE43
:107C4000C87A04F2844493ED007A04EB8B0B28EE9F
:107C5000877AA7EE278A8BED008A2EF099FA002802
:107C6000B8BF4042C0B214280ED9BB4BB3F8DC24D5
:107C700007EE902AF8EEE77A87FE888ABCEEC88A7B
:107C800018EE102AA3F8DC24BAF1000F34D10F2E1D
:107C900000F0AF80112E7CD1B04B9FEDB10AD3ED37
:107CA000007A28EE800AFDEEE77A17EE903AA8F8FF
:107CB000BC3D51F061F9A8F8BE0D91E40138C0B2A5
:107CC00004EB800307EE900A03F23463F8EEE77AE0
:107CD00093ED006AB5F8183C26EE066A37EE067A90
:107CE000E6EE276AB5EEC07AF1EE10FA8EDCB0EE61
:107CF000487A9FED9C9A90E7102E7FF475ACF2E4E1
:107D0000F2EE008AB7EE007AC7FEE88AC8FE878ADC
:107D100041F2C62104F284438D4A15F801A092ED88
:107D2000000A0AF1AC0B03EB8B0393ED008A88EE9B
:107D3000000A51F021F9C0B2431C3FE741F2C623CB
:107D4000894CD5F8B01CEB5C04F56A7054ED270A39
:107D500003EBC30204EB830300EB820003F23473F2
:107D6000D0F814B0D0F818A0D0F81C90026A93EDA7
:107D7000000AFFF739BBF0EE477A1846FFF745B81F
:107D800037F03CFAC01B98F8BA6DA8F8C00DFFF7A1
:107D90000FB82B2EB0D1714BD3ED007AFDEEE77A00
:107DA00017EE903AA8F8BE3D1AE4F0EE667AC8B233
:107DB000FFF7CAB8F0EE477A5FFA8CF0FFF7ADB87C
:107DC000F0EE667AC8B2FFF7E8B8F0EE477A5FFAED
:107DD0008CF0FFF7D1B8F0EE667AC8B2FFF706B9BB
:107DE000F0EE477A5FFA8CF0FFF7EFB8B0EE667A04
:107DF00025E69FED5B0A29EE000A51F0BDF8A8F8D0
:107E0000C20DFFF7F1BBA9F2145009F5D07301467A
:107E1000FFF758BBF7EE008A7AE737F0EFF9C01B9F
:107E200098F8BA6DA8F8BE0DFFF7EABA37F0E6F990
:107E3000C01B98F8BA6DA8F8BE0D49E51A46002097
:107E4000DFED487AFFF701B90E2AF0EE477A5FFAC4
:107E50008CF002F102037FF430A94CE50F2BF0EE19
:107E6000477AD8B203F101027FF43FA943E50F2A14
:107E7000F0EE477AD0B202F101037FF44EA93AE561
:107E80000F2BF0EE477AD8B203F101027FF45DA91F
:107E900031E50F2AF0EE477AD0B202F101037FF408
:107EA0006CA928E50F2BF0EE477AD8B203F1010256
:107EB0007FF47BA91FE5F7EE006A67E6B7EE007A6C
:107EC000BDE50F2AF0EE477AD0B202F101037FF44C
:107ED00084A910E50F2BF0EE477AD8B203F1010226
:107EE0007FF493A907E50F2AF0EE477AD0B202F1AA
:107EF00001037FF4A2A9FEE40F2BF0EE477AD8B27B
:107F000003F101027FF4B1A9F5E40F2AF0EE477AFC
:107F1000D0B202F101017FF4C0A9ECE40F29F0EE28
:107F2000477AC8B201F101037FF4CFA9E3E40F2B34
:107F3000F0EE477AD8B203F101027FF4DEA9DAE469
:107F40000E2AF0EE477AD0B23FF4EDA9D3E400BF99
:107F5000340C00203C0C00200C110020F4130020F5
:107F60000000C84200000000C00C0020F8B5214C01
:107F70001D270E46054684F8D87D20F079FB0020A9
:107F800020F01AFB082020F017FB0E2020F014FB35
:107F9000384620F011FB042020F00EFB042020F0D6
:107FA0000BFB002020F008FB302020F005FB002018
:107FB00020F002FB304620F0FFFA002020F0FCFA0F
:107FC00020F042FB04F6D95020F04BFA234670B162
:107FD00094F8D92D62B994F8DA2D302A00D03AB944
:107FE00093F8DB2D22B993F8DC3D01202B70F8BD0E
:107FF0000120FCE7604C0024104B034410B50446FC
:1080000093F8580817F03EFB0D480A2300EB440490
:108010000920B4F9EC1DB1F5FA6FA8BF4FF4FA616D
:10802000B1F57A7FB8BF4FF47A71A1F57A71B1FBDF
:10803000F3F1BDE81040C9B217F052BBE8B8090827
:10804000604C00241C4991F8842B9AB3F0B40026AC
:1080500005463346304637461BB991F8844B2D2CE4
:1080600022D02E2A18D0CA1800EB800092F8844B38
:108070004000A4F13002092A02D8A0F13002A01871
:108080000E2B14D80133CA1892F8842B002AE3D19E
:1080900006B14042F0BC70470133002DF8D0CA1839
:1080A0002A4482F8847BDEE701231E46EBE70020AA
:1080B000F0BC704700207047604C00241FB503AC33
:1080C0008DF80C30002300948DF80D3010F03CF842
:1080D00004B010BDF8B50546262028F0A9FB134CC6
:1080E0000146F8B9D4F8100E90F838301E3B012B39
:1080F00001D93DF0D1F90E4F0026AE420ADBB4F8AB
:10810000343E0133A4F8343E0A4BD3F8B43DC4F8EE
:10811000443EF8BD17F8011B0136D4F8100E3DF0AF
:10812000BBF9EAE7002384F8423EEDE7604C002407
:10813000745A0024702A002410B5F9F779FA04461D
:1081400011213DF0F9FB20463DF01AFDC8203AF020
:10815000DBFD2046BDE810403DF018BD08B55220BB
:108160003DF0F8F9054BC3F8480E08B12A23C38047
:108170004021BDE808403DF0DFBB00BF604C00245B
:10818000F8B5694CD4F8BC1D0B699E0702D5CB68C5
:108190009D074BD40B69580702D5CB685A073DD4CD
:1081A0000B691B0702D5CB681F072FD40B69DE06AE
:1081B00002D5CB68DD0621D40B69D80702D5CB6880
:1081C000DA073FD40B691B0603D5CB681F0600F105
:1081D0008F800B69DE0503D5CB681D0600F18C800E
:1081E0000B695C0603D5CB68580600F189800B69E2
:1081F0009A0602D5CB689B0620D4F8BD6FF010021A
:1082000000230A61CA6984F8D83DD5E76FF00802F7
:1082100000230A61CA6984F8D83DC7E76FF00402F9
:1082200000230A618A6984F8D83DB9E76FF0020239
:1082300000230A618A6984F8D83DABE76FF0200318
:108240000B61F8BD394B6FF0010299420A61B9D157
:10825000D4F8980DD0F81432002BB3D1344E354AEF
:10826000D6F84C5E95B1D2F808C505F03F076544D5
:10827000C2F80855D2F80855B5F5006F01D1C2F81B
:1082800008350023C6F84C3E002F43D0D2F80855DD
:10829000D2F80C359D4295D0D2F80855D2F80C355D
:1082A0009D4231D9D2F80855C5F50065D2F8087558
:1082B000B5F5007F204A28BF4FF40075D0F814327E
:1082C0003A44C0F81052C0F80822002B7FF47AAF6D
:1082D000012781212B46C4F8105BC0F81472D4F832
:1082E000B00D04F0E7FED4F8BC1DC6F84C5E69E79B
:1082F0006FF080030B616CE76FF480730B616FE7C5
:108300006FF040030B6172E7D2F80C55D2F80835D4
:10831000ED1ACBE7D2F80825074BC0F810721344CA
:10832000C0F808324EE700BF702A00240014004055
:10833000604C002478190024502D002438B5D0F862
:10834000D04201F00F03626893422BD80A062BD467
:108350001C25C1EBC102002005FB014104EB820298
:1083600001F5FE7182F8FD0101220B708A7094F80C
:10837000BC03904216D084F8BC234A782068012AB6
:1083800009781DD000F5306202EB41121568002D0E
:1083900000DBF1B9116841F4001111601BB3002337
:1083A00084F8BC33002038BD1C21C3EBC30201207C
:1083B00001FB034104EB82023C3182F83D00D3E72C
:1083C00000F5106202EB411215680029E2D0002D81
:1083D000E0DB116821F080411160116841F4001167
:1083E0001160002BDBD104F57172217C04F0C6FC16
:1083F000D5E700BF10B504468021FFF79FFF00219D
:108400002046BDE8104099E72DE9F04F9A4D89B01C
:108410002B685C6914F0010402D009B0BDE8F08F4C
:1084200059699A691142F8D05A6999690A409007C6
:1084300003D55A6902F002025A615A699969019397
:108440000A40D10612D59A6922F010029A611A6A7E
:10845000C2F3434102F00F07022900F09D83062971
:1084600000F0FC829A6942F010029A615A69996997
:108470000A40120300F119825A6999690A405103AE
:1084800000F14E8159699A69114252D45A69996929
:108490000A4012050AD5019A02F500629268D707D0
:1084A00000F1B2835A6902F400625A615A6999690B
:1084B0000A40160110D55A6902F000625A6195F817
:1084C000F423002A40F03782012285F8F4235A6D04
:1084D000C2F38302C5F8F8235A6999690A40D004A7
:1084E00000F1BC805A6999690A40920458D45A69CB
:1084F00099690A40170747D45A6999690A40D60210
:108500003DD45A6999690A40940233D45A699969E9
:108510000A40500029D45A6999690A4051077FF5E9
:108520007CAF5C68620700F163835A6814435C6047
:1085300073E7019A02F50061D2F8042822F00102E3
:108540004A6095F8F423012A00F00F82D5F804243C
:1085500092F89C12042903D192F89D1282F89C1281
:108560005A6902F000425A6190E75A6902F080426B
:108570005A61D0E75A6902F400125A61C6E75A6993
:1085800002F480125A61BCE7D5F8040490F89C22EA
:10859000032A00F031825A6902F008025A61ABE7FF
:1085A000D3F8000935490140C3F80019D3F804187D
:1085B00041F48071C3F80418D3F8082812F00601BA
:1085C00040F0C3810193E9600BF030FEEA68019B43
:1085D000D1B2022900F0CD81D968B2F1000821F4AE
:1085E000705118BF4FF00108D960DA6842F4105298
:1085F000DA60D5F804444027002301263A46D4F82F
:10860000D002194604F022FF3A460023D4F8D002E3
:108610008021C4F85861C4F8647104F017FF002386
:10862000D4F8C822A661676284F89C62C4F89432C8
:108630006360C4F8A432002A00F01383D4F8B43283
:10864000204600215B689847D5F804242B6882F8FF
:1086500010805A6902F400525A6148E7019A4FF4B7
:108660008460D2F8041802F50066054A21F0010181
:108670007160186108E000BF7819002400F8FFFF5E
:10868000400D0300013A02D019698906FAD46F68D7
:1086900017B3019A4FF67F3002F5106290600134F3
:1086A00011682032BC4221F4001142F8201C52F81B
:1086B000201C41F0006142F8201CC2F8E801D2F809
:1086C000E01121F40011C2F8E011D2F8E01141F0FC
:1086D0000061C2F8E011E1D1F269296B42F00112A8
:1086E000F261002900F03781D6F8842042F00B02B5
:1086F000C6F88420726C42F00B027264019C18462A
:10870000C24AD4F8001821F4FE63297CC4F800386A
:1087100004F034FB2B685A6902F480525A61E1E696
:10872000D3F81828D3F81C1802EA01081FFA88F8B1
:10873000B8F1000F3FF4A6AE019A4FF0000AB44E14
:1087400002F51067029407E05FEA58080AF1010A8F
:1087500006F11C0600F0988118F0010FF4D05FFAC2
:108760008AF9D3F81018D3F8344803F5106209F0E9
:108770000F0002EB4912C4409268E401E4B20C43DA
:108780001440E20727D54FF0010E019A0AF00F0CB2
:1087900007EB4A10D2F834180EFA0CFC21EA0C014F
:1087A000D5F810C0F445C2F83418C0F808E000F05D
:1087B0003582D5F804B4B9F1000F00F05082DBF82F
:1087C000B42252693AB19BF89C12032903D158464E
:1087D000494690472B68200703D507EB4A1208212A
:1087E0009160E10603D507EB4A1210219160620601
:1087F00003D507EB4A1240219160A00703D507EB90
:108800004A120221916021069ED5D6E914048442C1
:108810009AD8011B726C03EB4A1C8A420CF5106C4F
:1088200028BF0A46DCF81810033289B2B1EB920F68
:108830002CD309F101099E4603EB093928B3844280
:1088400023D2011B726C2B7C914228BF1146B26C63
:1088500001F1030B4FEA9B0B73B98BB203339B08F7
:108860000AD002EB830352F8040B9A42C9F80000C5
:10887000F9D1B26CD6E91404DCF818300A440C447F
:108880009BB2B26474659B45D8D973468442FFF4A9
:108890005BAF0AF00F000124D3F8341804FA00F09B
:1088A00021EA0001C3F834184EE7D3F81828D3F8AA
:1088B0001C180A405FEA124A3FF4DEADDFF850B1FF
:1088C0004FF00009DDF80480029407E05FEA5A0ADD
:1088D00009F101090BF11C0B00F0D4801AF0010F13
:1088E000F4D05FFA89F603F5306101EB4610846835
:1088F000D3F814281440E70700F12981270700F175
:10890000C580E70605D508F53062102102EB491253
:108910009160A60605D508F53062202102EB4912C8
:108920009160A004D2D508F530624FF4005102EBFB
:1089300049129160CAE7D5F80424042092F89C12E9
:1089400082F89C0282F89D12C6E512F0020F14BF55
:1089500002210F2136E6716942F22B020A4372614D
:10896000326942F00B023261C8E6002285F8F42336
:10897000F6E5284A284902448A4240F22083274AE1
:10898000274902448A4240F23383264A2649024458
:108990008A4240F2A083254A254902448A42C0F017
:1089A000B583244A244902448A4240F20F84234A70
:1089B000234902448A42C0F01984224A22490244CF
:1089C0008A42C0F07684214A214902448A42C0F09A
:1089D0006C84204A204902448A4234BF4FF4E0505C
:1089E0004FF4C050D9684FF0010821F47051D9609C
:1089F000DA680243DA60FCE5D0F8B422D269002AD2
:108A00003FF4C9AD90472B68C5E500BF3C1D00246D
:108A100078190024405327FFFF340C00401E1BFF31
:108A20003F420F0000DC0BFF7F4F1200808CF9FEED
:108A300020D6130060B6E5FE5FE3160000D3CEFE3D
:108A400040771B00C05BB3FEC091210000CA91FEBD
:108A500020753800E05459FEE09C4100C7EBC70187
:108A600003F58050C2F30A1205EB81010768D1F8C3
:108A70001462C5F8C47332440068C1F81422C5F802
:108A8000C803EFE4029CF7E4029CFBE408F53062C3
:108A9000082003EB491102EB491201F530619060A7
:108AA0001B6CD0481A4603938B68824204D91E047B
:108AB00002D54FF400438B60D5F8046495F8C4C325
:108AC00006F52A7386F8A8C20CF01F07059395F8DF
:108AD000C533012F86F8A93295F8C70395F8C62348
:108AE00002EB002291B2A6F8AA1295F8C92395F8D4
:108AF000C80300EB022080B2A6F8AC0295F8CA23A6
:108B000095F8CBE304924FF00102C6F89422049A40
:108B100002EB0E2292B2A6F8AE22C6F8982200F01E
:108B2000F580022F00F0DE80002F00F010810CF0A5
:108B300080013046FFF702FC039B1A46A94B9A427C
:108B400003D92969012900F04E822B68D9E62869EA
:108B500008F53062012701EB491102EB49120128A7
:108B600097601F6C8A6800F087809F48874200F0FA
:108B70001D82D5F8102259EA020100F07882C6EB76
:108B8000C6033146D5F8040405EB8303D3F8082265
:108B900004F01EFC2B68B1E647F6F0710A423FF480
:108BA00061ACC2F30A10C7EBC7014FEAC70E024619
:108BB000033005EB81018008D1F808820AD008EB68
:108BC000800603F5805C4146DCF8000041F8040BA8
:108BD0008E42F9D1AEEB070108EB020605EB8101ED
:108BE000D1F81402C1F808620244C1F8142239E431
:108BF000D5F804040122D0F8B43280F89C2201791F
:108C00005B6898472B6890E4D5F80424042092F818
:108C10009C1282F89C0282F89D1243E4D6E911125C
:108C20000A44B264BAF1000F7FF4C3AD2A6D002A82
:108C300000F0E181D5F804B4AA6CDBF89432022B81
:108C400028D033F0040300F0C9819BF8A032012B37
:108C50007FF4C0AD00222B688BF8A022BBE5AA6C84
:108C6000EBE7D4F8B832002B7FF4E8ACD4F8C0328C
:108C7000002B7FF4E3ACE7E4100740F1A3815948EF
:108C800087427FF63BAE16047FF538AE4FF40042C4
:108C90008A6033E6DBE90813994200F2B281DBF81F
:108CA0001C10B1FBF3F203FB121212B98B4240F21B
:108CB0001582DBF8B432DB682BB19BF89C22032AC7
:108CC00001D15846984780215846FFF737FB0023CB
:108CD0000522DBF8D0021946CBF894221A4604F09C
:108CE000DFFAB2E70CF06007202F00F07081402F10
:108CF00000F06D81002F00F0BF8180213046FFF72A
:108D00001DFB30460021FFF719FB15E70CF060034F
:108D1000402B02D01CF0400FEFD196F89C32013B63
:108D2000022BEAD8C0B20328E7D8D6F8B4323046CE
:108D300005999B689847B6F8AE32002B7FF4FCAEDD
:108D400000287FF4F9AE304604F004FAF4E60CF0A3
:108D5000600CBCF1200F00F03A81BCF1400F00F034
:108D60003681BCF1000F08D080213046FFF7E6FACB
:108D700039463046FFF7E2FADEE6092BBDD801A7F7
:108D800057F823F0E18E0408498E0408FB8C040890
:108D9000CF8E0408FB8C0408698E0408158E040825
:108DA000FB8C0408F18D0408AD8D0408CFB20F4A86
:108DB000012F82F8507EA0D896F89C32022B00F04A
:108DC0004982032B00F0318280213046FFF7B6FA4A
:108DD00000213046FFF7B2FA3946304602F004FD72
:108DE000AAE600BF0A30544F0A31544F604C0024A9
:108DF000012A82D196F89C32022B00F20E82002BBF
:108E00003FF47BAF00233146304641F8083F04F081
:108E1000B1F991E60B0A0022013BADF81E20062BAA
:108E20003FF66BAF01A252F823F000BF9D8F0408FC
:108E3000838F04086B8F0408FB8C0408FB8C0408E8
:108E4000558F04080F8F040896F89C32013B022BC3
:108E50003FF653AF01297FF46FAE00233046C6F8CA
:108E6000A43204F077F967E650EA02037FF445AFD5
:108E70007F293FF642AF96F89C32032B3FF43DAF7B
:108E8000CFB2D6F8D03286F89E7293F8BC23012A6E
:108E900011D01A68002083F83870D2F8007827F4CF
:108EA000FE67C2F80078D2F8007847EA0117C2F8E6
:108EB000007883F8BC033046049104F04BF9049920
:108EC000002900F00482022386F89C3234E601294E
:108ED0007FF432AE3046C6F8A41204F03BF92BE61C
:108EE00096F89C32013B022B3FF607AF022A7FF433
:108EF00004AF0122D6F8A432F2600BB10323F36071
:108F0000022206F10C01304604F034F914E6337CF9
:108F1000002B7FF4F2AED6F8B4320DF11E001B6BBD
:108F2000984707234370BDF81E206AB1B6F8AE32E9
:108F3000002B3FF408AF9A420146304628BF1A463C
:108F4000ADF81E2004F016F9B6F8AE32002B7FF40F
:108F5000F3ADF8E6337C002B7FF4CFAED6F8B43215
:108F60000DF11E005B6B9847DDE7CBB2052B3FF69A
:108F7000C4AEDFE813F0F301ED01E701E101D50133
:108F8000CA01337C002B40F0AF81D6F8B4320DF12A
:108F90001E009B6A984702234370C4E7D6F8B0329C
:108FA0000DF11E01307C1B689847BCE710043FF5AB
:108FB0006DAE93067FF5E3AD20238B60DFE54FF4C4
:108FC00070500FE590062FD520228A6096E4D6F8DF
:108FD000B432304605999B689847ADE580215846E4
:108FE000FFF7ACF931E6D14A286803F0C7FEACE5DB
:108FF0004FF46050F6E461461846CC4A03F0BEFEDA
:1090000018E6A1EB030CDBF8D00200211FFA8CF369
:10901000CBE9073C04F04EF80023DBF8D0021A46F7
:10902000194604F03DF910E612F0280F7FF466AC03
:10903000BF48874202D917043FF528AE0A69DBF81A
:109040000402C2F31202DBF80812821A0144CBF8C0
:109050001422D5F81022CBF8081259EA02027FF444
:109060008EAD1846B14A012103F088FE87E5184607
:10907000AE4A03F083FE82E5012B5FFA80FC5CD0F0
:10908000032B46D0002B7FF46FAE96F89C32022B58
:1090900000F0B080032B7FF430AE030600F1E980CE
:1090A0000CF00F02142303FB0262D2F85871002F58
:1090B0003FF45AAE0CF07F0003FB006303F5AA7285
:1090C000002840F01A810023136011463046022226
:1090D00004F050F830E54FF4505083E4DBF8983258
:1090E0009942BFF4E6AD0023DBF8D0021A461946D8
:1090F000CBF81C3003F0DEFF0023DBF8D0021A4669
:109100001946CBF8983204F0CBF89EE54FF4405066
:1091100068E496F89C32022B5BD0032B7FF424AEDC
:1091200051EA02037FF40FAE1CF07F0F3FF40BAE49
:1091300061463046FFF702F905E696F89C32022BAD
:1091400047D0032B7FF410AE00297FF4F5AC1CF060
:109150007F0F3FF4F8ADD6F8D0220CF00F01536822
:1091600099423FF6F0AD00064FF01C0300F1A580D8
:1091700003FB01200027034600F5FE7083F8FD7114
:1091800000230170837092F8BC33012B3FF4DBADF8
:109190000121136882F8BC1347780178012F0CBFB6
:1091A00003F5106303F5306303EB4113196821F4F1
:1091B00000111960C1780239012903D8196841F0FA
:1091C00080511960002382F8BC33BCE54FF4305065
:1091D00008E41CF07F073FF4C7AD61463046FFF757
:1091E000ADF830468021FFF7A9F8A5E44FF42050F0
:1091F000FFF7F8BB1CF07F0F7FF47FAD02064FF046
:10920000000330464FF002024CBF06F1140106F590
:10921000AA710B6003F0AEFF8EE4032B7FF46DADFB
:10922000311D304603F0A6FF86E4002F53D071684D
:1092300001293FF488ADC9B2304602F0D5FA3D4A63
:10924000304692F8501E716002F0D6FA02287FF480
:109250007AAD52E5002F3FF476AD0121032330466D
:10926000716086F89C3202F0C7FA02287FF46BAD79
:1092700043E50CF00F03142202FB03639F69002FE8
:109280003FF472AD0CF07F0303FB02223244002B4B
:109290003FF419AFD6F8D0121C2000FB031393F84B
:1092A0003E3093B1012313600FE74FF40050FFF7F6
:1092B00099BB4FF41050FFF795BB03FB012001272A
:1092C00003463C3083F83D705AE71360FDE6012306
:1092D00086F89C3230E4022339463046776086F8BF
:1092E0009C3202F081FA2EE5D6F8B4320DF11E0060
:1092F000DB6A98470223437015E6D6F8D0321C206B
:1093000000FB0C3393F8FE31CBE7D6F8B0329F69FF
:10931000002F3FF429AD0DF11E01307CB84702E665
:10932000D6F8B0325F69002FF5D11DE53C1D002451
:109330000A30544F604C0024D6F8B0321F69002F19
:10934000E9D111E5D6F8B032DF68002FE3D10BE5A3
:10935000D6F8B0329F68002FDDD105E5D6F8B032DF
:109360005F68002FD7D1FFE470B5114C4422002173
:10937000032604F21475284652F07CF994F8283537
:109380004FF6FF72D4F87817022B2846A4F82E2740
:109390004FF0100218BF334684F82C67C4F8381712
:1093A00084F8143784F82D27FCF7B6FC012070BD33
:1093B000781900242DE9F041344A4FF0FF3500239D
:1093C000A2F5A5602C4603E0013310320B2B14D01C
:1093D00092F82A100429F7D100EB031191F85315E4
:1093E000CF07F1D4661C116A01D0A942ECD21C4609
:1093F00001330D4610320B2BEAD1631C02D1012040
:10940000BDE8F081224DA71C05EB0713B3F830151A
:10941000F1B92601DFF88080AA19D5F84015D8F8EF
:10942000546E0023D2F8440501EB44213669194AF1
:10943000B047E0B1022817D1D5F8F83505EB07178A
:1094400001220020013B87F83225C5F8F835D7E71F
:10945000DFF8448005EB04122601D8F8543ED2F818
:109460004405DB689847D7E70020BDE8F081D5F8D0
:10947000F83505EB071703210122013B87F8321568
:10948000C5F8F83585F8FC25BAE700BFA01E002412
:109490007819002405A40408604C0024054B93F8B7
:1094A000102712B9012283F81027012283F82925F9
:1094B000704700BF7819002443682DE9F04F164625
:1094C00083B0C3F30808002A00F0DE800546894611
:1094D0004FF0000BDFF8B8A1C8F5007495F91A70C9
:1094E0002846B44228BF3446791C30D001F0C4FC71
:1094F0000AEB0713D3F84435984205D0FFF7CEFFA7
:10950000584603B0BDE8F08FDAF8400500EB47207D
:109510000028F5D0224649464044A34452F038F88A
:1095200000222146284601F0A5F80028E8D02B7E2D
:109530001B0706D52A69DAF8F0369A4201D3FFF7FD
:10954000ADFF361BA1444FF00008C5D1D8E700F0AD
:10955000F9FF002845D1284601F08EFC6968C1F367
:10956000080313BB494AAB680A4002F500729A42ED
:109570002CBF062207222B7E03F00C030C2B1AD0E3
:10958000002301A901F090F80128B9D10198DAF877
:109590004035C31A48BF03F2FF13B3F5B05F4FEA7B
:1095A00063224AD257B2AF76B2E72B7E072203F08E
:1095B0000C030C2BE4D19AF828C5DAF86C37BCF10F
:1095C000030F0CBF4FF0800C4FF4807C03FB0CF3B7
:1095D0004FEA432C0CF1FF3C0CEA0101A3EB5123B1
:1095E000CFE72B7E1A072DD59AF82825DAF86C37A5
:1095F000032A95F828200CBF80214FF48071062A99
:1096000003FB01F34FEA43233FF47AAFDAF8D416B1
:109610008B4232D89AF81137002B7FF471AF002AB1
:109620007FF46EAF06216B69284685F8382085F8EF
:109630002810EB6201F016FA1BE0FFF72FFF0198EC
:10964000AF7665E795F82830002B7FF459AF9AF88C
:109650001137002B7FF454AF08216A6985F8343044
:10966000284685F82810DAF87037EA622B6301F093
:1096700093FB01283FF46FAF42E7012358468AF875
:10968000113703B0BDE8F08F934639E700FEFFFFC6
:109690007819002408B50B46114602070FD50A4A6F
:1096A000581CD2F8F036834204D305D100230120A0
:1096B0000B6008BDFFF7F2FE0860012008BD1846E8
:1096C000BDE80840FCF7FABA7819002410B5037811
:1096D0000446023B012B037E02D913F0060F58D13A
:1096E000980638D494F91A20511C0AD02C4BFF212B
:1096F00003EB021393F853256FF3000283F853250D
:10970000A17694F91B305A1C0FD02549FF2001EB9C
:10971000031191F85335C3F34502013A22EAE2728C
:1097200062F3460381F85335E076237E1B0709D5A3
:109730001B4991F8F436072B01D0FFF7AFFE002349
:1097400081F8F4360023E26A237084F82830FAB1F5
:10975000BDE810401047134B0022E069D96910336F
:10976000884206D001320B2ABCD0D9691033884216
:10977000F8D10B4B03EB021292F85335C3F34501BA
:10978000013921EAE17161F3460382F85335A9E713
:1097900010BD012101F086F80128F9D1237E9FE751
:1097A00078190024A01E0024B8B138B5027822B17F
:1097B00090F828201AB1002038BD012038BD8268F9
:1097C00003244568C162AA4280F8284038BF2A466F
:1097D0008260FFF77BFF012038BD0120704700BF8A
:1097E0002DE9F04190F8283084B00446013B082B65
:1097F0003FD8DFE803F046054B5056633E68410012
:10980000384B4168D3F87477056B0F40D3F86C3749
:10981000EA194FEA4328B2EB432F16D258E02169E8
:10982000207EFFF737FF012823D1256B6168A5EB68
:10983000080522694144039B3D446261C91B2361C1
:10984000A84537466160256342D8204600F07AFE7D
:1098500003AA06460028E2D06168A3680020E26AF5
:10986000994284F8280038BF1946A1600AB1204601
:10987000904704B0BDE8F08101F01CFB04B0BDE8E6
:10988000F08101F02FFC04B0BDE8F081FFF71EFF6E
:1098900004B0BDE8F081002101F0E8F904B0BDE8B2
:1098A000F081012101F0E2F90128E2D10023216CCD
:1098B000204684F82830FFF777FFDAE701F0D2F886
:1098C00004B0BDE8F08101F067FA04B0BDE8F081B2
:1098D0002046019100F036FE01990028BDD12944AF
:1098E0006160BAE77819002400487047385D0024A9
:1098F000034B93F82400032894BF002001207047F5
:10990000105D0024034B93F82400003818BF012099
:10991000704700BF105D002403460A2201481A80E8
:10992000704700BF080300240023D0F8C022184667
:10993000137370470346222201481A80704700BF04
:10994000140300240346222201481A80704700BFF6
:10995000380300240346222201481A80704700BFC2
:109960005C03002403460A2201481A80704700BFA6
:10997000800300240346432201481A80704700BF39
:109980008C0300240346432201481A80704700BF1D
:10999000D00300240346432201481A80704700BFC9
:1099A00014040024D0F8BC3283B110B5D0F8B8420A
:1099B00094F80002FF2807D09B68214694F8012202
:1099C0009847FF2384F80032002010BD0020704724
:1099D00001F00F01D0F8D022C1EBC10102EB8102EE
:1099E00038B5D0F8B832D0F8BC52D2F8144203F5EA
:1099F0000371EA68D3F80402C3F80C4290470020D0
:109A000038BD00BF70B40479611E072930D80268E0
:109A10001B4B1C4E1C4DB24218BF9A4206F1280641
:109A20000CBF01230023AA4208BF43F001032835DD
:109A3000B24208BF43F001032836AA4208BF43F0F0
:109A400001032835B24208BF43F00103AA4208BF10
:109A500043F0010313B90D4B9A420BD10C4B0D4D42
:109A600023449B00012202FA01F1C0E91B35416742
:109A700070BC7047084B094D23449B00F2E700BFC0
:109A8000085402581C540258305402589454025836
:109A90003F960016405902583F820010400902408C
:109AA0000368294A294930B4294D2A4CAB4218BFD2
:109AB000934205F13C050CBF01220022A34208BFDE
:109AC00042F001023C348B4208BF42F001023C31BB
:109AD000AB4208BF42F00102A34208BF42F00102BC
:109AE0008B4208BF42F0010212B91B4A934213D1C4
:109AF000DBB21A4D1A4A0121083B1A4CA5FB03534D
:109B0000446602EB1312C3F30413920001FA03F349
:109B10000266836630BC7047DAB21349134C1944AD
:109B2000103AA829A4FB02234FEA131300D80833E4
:109B30000F4A03F01F0501210E4C1A44A940446648
:109B4000920081660266E5E70854025844540258C0
:109B50001C5402583054025894540258CDCCCCCCEA
:109B60000096001680580258F0FBFDBFABAAAAAAC7
:109B700000820010800802400268354B354930B43D
:109B8000354C364DA24218BF9A4204F148040CBF2E
:109B9000012300238A4208BF43F001034831AA424F
:109BA00008BF43F001034835A24208BF43F0010358
:109BB00048348A4208BF43F0010301F56271AA42AA
:109BC00008BF43F0010305F56275A24208BF43F0E8
:109BD000010304F562748A4208BF43F0010348316F
:109BE000AA4208BF43F001034835A24208BF43F030
:109BF000010348348A4208BF43F001034831AA42B6
:109C000008BF43F00103A24208BF43F001038A42A8
:109C100008BF43F0010313B9114B9A4213D1D3B2D9
:109C20001049114C103BA1FB03515F2B0F4BC1F3AB
:109C3000021103EA0203615C88BF0433C1658365D6
:109C4000184630BC704722F0FF038365F8E700BF79
:109C5000100002404000024028000240580002402C
:109C6000B8040240ABAAAAAA70C6090800FCFFFF0C
:109C7000F0B54B780D78012B26D000F530603B4CC9
:109C80003B4B00EB45104D690669344004610469A3
:109C9000234003618B6805B14B610469C3F3120370
:109CA000012A44F400240461046943EA04030361C3
:109CB00005D0036843F0044303600020F0BDCB6887
:109CC000002BF6D04361F4E74C6900F510638CB3C8
:109CD00003EB4513254FD1F808C0D3F810E0244E0C
:109CE00064450EEA07071F611F6906EA07061E6141
:109CF00002D96446C1F814C01E69C4F31204012AD3
:109D000046F400261E611E6944EA06041C6124D044
:109D10001A68496942F004421A600029CDD005F062
:109D20000F020125D0F8343895401D43C0F834584F
:109D30000020F0BD03EB45130D4EA4F50024012ACD
:109D40001F6906EA07061E611E6946F400261E61A9
:109D50001E6904EA06041C61DAD10A6902B15A617B
:109D60001A68002042F004421A60F0BD0000F8FFBB
:109D7000FFFF07E02DE9F0434D780F78012D4DD01E
:109D800000F530637A4E4C6903EB4713794D1F6938
:109D90003E401E611E6935401D616CB38D68012A0D
:109DA000754E2C441F6904F1FF34B4FBF5F41FFA1F
:109DB00084FC06EAC44405FB0CF544EA0704C5F339
:109DC00012051C611C6945EA04051D6121D0CA7891
:109DD000012A0AD1D0F8082812F4807F1A680CBF33
:109DE00042F0005242F080521A601A6842F0044277
:109DF0001A600020BDE8F0838C68012A1D69C4F355
:109E0000120444EA05041C611C6944F400241C612A
:109E1000DDD1CA68002ADAD05A61D8E74B6900F56B
:109E20001064002B3CD004EB4714D1F808E0DFF8B5
:109E30004091C3F31206D4F8108003EB0E0C08EA2D
:109E400009090CF1FF3CDFF82C81C4F81090D4F81C
:109E50001090BCFBFEFE09EA0808DFF81CC1C4F83C
:109E600010800CEACE4CD4F810E04CEA0E0CC4F88A
:109E700010C0D4F810C046EA0C062661CE78012E38
:109E800047D0012A5FD0226807F00F0342F0044256
:109E90009D402260D0F834783D43C0F83458A8E79C
:109EA00004EB4714334E324D012AD4F810C00CEAAB
:109EB00006062661266946F400262661266905EA1B
:109EC00006052561CE7833D02568012E45F004457E
:109ED00025608ED1D0F8085815F4807F25680CBF16
:109EE00045F0005545F080552560002A81D19BB290
:109EF00003339C083FF47DAFCA6800F5805302EB42
:109F0000840403EB073352F8041B94421960FAD11E
:109F10006FE72569012A25F0C0452561256945F0CF
:109F20000055256114D0256845F004452560D1E72A
:109F30000B695BB9012E0ED02368002043F0044367
:109F40002360BDE8F0830B69002BF5D06361F1E776
:109F50000B69002BFAD1D0F8083813F4807F2368FE
:109F60000CBF43F0005343F080532360E4E700BF8D
:109F70000000F8FFFFFF07E00000F81F836B5A6D39
:109F800042F040025A659A6D42F004029A657047A9
:109F9000704700BF836B5A6D12F0500F5A6D1AD183
:109FA000196842F400725A650A6812F0080FCA680C
:109FB00016D012F4406F15D1CA68920412D45A6DAB
:109FC00022F480725A655A6DD1040BD45A6D42F056
:109FD00001025A657047D20604D4DB6CDB6C18476B
:109FE0009007ECD0704700BF11F0800F4FF01C03BA
:109FF00001F00F0170B432D103FB0103C1EBC102C8
:10A00000002400EB820203F5FE7382F8FD41197013
:10A0100090F8BC23012A31D00121026880F8BC13DA
:10A020005C781D7802F500638C422AD005F00F049D
:10A03000DE6B02F53062A1401C4C02EB451226EAB1
:10A040000146DE63DD6925EA0141D96113681C40E0
:10A050001460002380F8BC33184670BC704703FBC3
:10A060000103C1EBC102012400EB82023C3382F800
:10A070003D40197090F8BC23012ACDD1022070BC5C
:10A08000704705F00F01DE6B02F510628C40084945
:10A0900002EB451226EA0406DE63DD6925EA0404C4
:10A0A000DC61136819401160D3E700BF0078F3EF5B
:10A0B000007833EC0022836BA3F85E20A3F85620CF
:10A0C000704700BF836B1A6830B4D3F88040D3F870
:10A0D000840091680D0601D5212C1CD09168490699
:10A0E00001D5222807D0D3F8882042F0100230BCD6
:10A0F000C3F88820704700240E492025A3F85E404D
:10A10000106820F490701060906801409160DC66E7
:10A11000C3F88450E7E700212024A3F85610116803
:10A1200021F0C0011160916821F400019160C3F831
:10A130008040D3E7FEFFFFEF704700BF704700BFCE
:10A14000C369B3F5807F13D0826B00212020136890
:10A15000A2F85E10196821F480711960996821F0E5
:10A1600001019960996821F040019960C2F884006A
:10A17000704700BFC369B3F5807F0CD0826B0021AC
:10A180001368A2F856109A6822F080029A601A6842
:10A1900042F040021A607047836B00220121A3F84D
:10A1A0006A20A3F8622083F881107047F0B43A4D1A
:10A1B000AB6A03F00303032B66D02B682A46374CA7
:10A1C00023F080532B60256803E023685B1B022B80
:10A1D00057D813689E00F8D4936A056823F07C73FF
:10A1E0002F4E43EA05539362D0E902356F1E013BBF
:10A1F00045685B0205F1FF3C3F0405699BB207F42B
:10A20000FE07CCF3080C013D3B432D0643EA0C034B
:10A2100005F0FE452B431364D36A456923F440637C
:10A220002B43D362D36A856923F400732B43D36233
:10A23000D36A23F48073D362556CC3692E4046EA17
:10A24000C3065664D36A43F48073D362D36AF1B110
:10A2500001290CBF43F4000343F08073D3620E4B1B
:10A2600019681A4641F080511960216803E023689B
:10A270005B1A022B05D813689B00F8D50020F0BCB0
:10A2800070470320F0BC70470120F0BC704743F4D6
:10A290008003D362E3E700BF00440258344800243F
:10A2A0000700FFFFF0B43A4DAB6A03F00303032B42
:10A2B00066D02B682A46374C23F080632B602568D4
:10A2C00003E023685B1B022B57D813681E01F8D4E8
:10A2D000936A056823F47C332F4E43EA0533936277
:10A2E000D0E902356F1E013B45685B0205F1FF3C7A
:10A2F0003F0405699BB207F4FE07CCF3080C013D4F
:10A300003B432D0643EA0C0305F0FE452B439363C4
:10A31000D36A456923F0C0032B43D362D36A8569AE
:10A3200023F020032B43D362D36A23F01003D362BC
:10A33000D56BC3692E4046EAC306D663D36A43F0A1
:10A340001003D362D36AF1B101290CBF43F4801327
:10A3500043F40013D3620E4B19681A4641F0806132
:10A360001960216803E023685B1A022B05D8136883
:10A370001B01F8D50020F0BC70470320F0BC7047EB
:10A380000120F0BC704743F40023D362E3E700BF31
:10A3900000440258344800240700FFFF836B01216A
:10A3A000002283F83D101A77704700BF0122836BAB
:10A3B00083F83D20704700BF70B5114E002433462E
:10A3C00093F82A0010B1DD698D4204D001341033B6
:10A3D0000B2CF5D170BD72B1B36903EB44239A42E3
:10A3E00001D1022801D0FFF759F806EB041401232C
:10A3F00084F82A3070BD06EB041484F82A2070BD5E
:10A40000A01E002438B50020144B04461D4683F8D6
:10A41000D40003E0013410330B2C13D0D8698842E8
:10A42000F8D193F82A000328F4D162B1AB6903EBA9
:10A4300044239A4201D0FFF731F805EB04140123BD
:10A4400084F82A3038BDD5F8D03005EB0414042246
:10A45000013384F82A20C5F8D03038BDA01E00246E
:10A4600010B50B4C002394F85920236202B1E36528
:10A4700049F00AFB20B10423022084F8243010BDE7
:10A48000044A0923126884F82430626110BD00BFB9
:10A49000105D00242438002470B50D4D04460E468E
:10A4A00095F82430042B0AD0082B06D1EB6983429F
:10A4B0000CD0FFF7D5FF022801D0012070BD082382
:10A4C0000220C5E9074685F8243070BD022070BD22
:10A4D000105D002438B504468321D0F8D002002551
:10A4E000FFF782FDD4F8C002656518B151F092F80B
:10A4F000C4F8C052002038BD38B50446002581217B
:10A50000D0F8D002FFF770FD0121D4F8D002E56247
:10A51000FFF76AFDD4F8D0028221C4F86C51FFF72E
:10A5200063FDD4F8B83225644BB1D4F8BC325B6813
:10A530009847D4F8B80251F06DF8C4F8B85200202A
:10A5400038BD00BF0378022B0FD0006908B9012085
:10A5500070470E4B1B78032B11D080B24FF6F77368
:10A56000984294BF002001207047084A4368D2F8FF
:10A570005422B3EB422F2CBF012000207047044B24
:10A58000984294BF00200120704700BFA01E002405
:10A59000F7FFFF0F2DE9F0410D46416882B00446F8
:10A5A000C1F308032B44B3F5007F53D390F91A305D
:10A5B000591C09D02E4A0233FF2102EB0313DA7A29
:10A5C0006FF30002DA72817694F91B305A1C0ED0B8
:10A5D000274A0233FF2002EB0313DA7AC2F3450164
:10A5E000013921EAE17161F34602DA72E0762378FB
:10A5F000022B35D01E4AD2F84432B5EB432F4FEA36
:10A60000432823DCD2F84C6267683E407342AB4279
:10A610001CDCAB19434511D301AA2169207EFFF749
:10A6200039F8012812D16768A5EB0805226947446B
:10A63000019B35446261BF1B236167602046FFF7C1
:10A6400081FF20B93D440120656000E0002002B098
:10A65000BDE8F08129440120616002B0BDE8F081CD
:10A66000616801202944616002B0BDE8F08100BF4B
:10A67000A01E002470B5154604460E46FFF78AFF5B
:10A6800050B994F8280028B90223C4E90B5684F87D
:10A69000283070BD022070BD1DB12046A8470120A2
:10A6A00070BD012070BD00BF2DE9F84F02F0020C13
:10A6B0009B4610B9BCF1000F53D1774DD5F83C72D1
:10A6C000002F54D14FF0FF36734F0024B146B046EF
:10A6D000B246FB69984200F0A88097F82AE0BEF1E4
:10A6E000000F50D0BEF1010F13D105EB041E9EF8F0
:10A6F0002BE01EF0010F0CD11EF07E0F09D15FEA96
:10A70000DE1340F09A80D7F824E0F24501D9F246F2
:10A71000A146013410370B2CDBD1741C04D1B8F1E5
:10A72000FF3F00F091804646D5F8CC40B71C05EBC2
:10A73000061E4FF00009013405EB0718CEF81C0087
:10A74000C5F8CC40CEF82040C8E9014905EB071414
:10A75000A47A042C00F29B80DFE804F01B3511354D
:10A760004C000224FEF79AFE2046BDE8F88FD5E99A
:10A77000904606FB0744A042A4D3FEF78FFE0024B8
:10A780002046BDE8F88F2646013410370B2CA0D1A7
:10A79000C3E712F0010E67D105EB0710BBF1030F01
:10A7A0004FEAE20490F80B8064F3C71880F80B803E
:10A7B00058D94FF6FF705B46834528BF03469BB2CE
:10A7C00005EB07100381BCF1000F13D005EB061356
:10A7D00093F82A001C3304280CD0D5F8CC000424AC
:10A7E0000130C5F8CC0058609C73D5F8D0300133E7
:10A7F000C5F8D030500705D505EB0710C37A43F0F4
:10A800000103C372D30608D505EB0717FB7AC3F320
:10A810004502013262F34603FB72AB69012403EB8C
:10A82000462620460E60BDE8F88FA71C05EB071EE4
:10A830009EF80A606EB9264676E7A04601341037C6
:10A840000B2C7FF446AF68E7B9F1FF3F97D04E4637
:10A850006AE7D5F8CC3026465C1CC5F8CC40CEF86B
:10A86000044073E77346ABE70C4A0023A969D2F8AA
:10A8700000C001EB46210A4ADCF80860B047002816
:10A880003FF47DAF05EB07150223AB726CE70224A2
:10A89000FEF704FE68E700BFA01E0024B45A00249F
:10A8A000B9A3040830B50446C06983B010B90120CB
:10A8B00003B030BD0D460023032201A9FFF7F4FECB
:10A8C0000128F5D1B4F92030002B03DAFEF7E6FDBC
:10A8D0000220EDE7019A012D4FEA431102EB4313E9
:10A8E00003D0022D12D1E5255554A268DA612278F1
:10A8F000032A04D100221A775A779A77DA77626AA4
:10A90000C2F30F415A83998203B030BDE268DA6125
:10A91000EDE700BF2DE9F04FDFF84491174683B013
:10A920008A4699F800300A68022B79D1D6B2D9F854
:10A9300034524FF48074A6EB020805EB1225B8449C
:10A94000A044BA4208F1FF38B8FBF4F864D200F032
:10A95000010BA844032B06EB0704A8EB05030CBF6F
:10A9600080214FF48071A41A8C4228BF0C460EB986
:10A970008C4235D20B2201A92846FFF795FE01280B
:10A9800002D003B0BDE8F08F99F80010DAF800208B
:10A99000022902F1010325D0A64210D2019A6FF0DC
:10A9A0004040111F304401EB840102EB800242F869
:10A9B000043F914203F10103F9D1DAF80020A61B0C
:10A9C0003244BA42CAF8002002D1BBF1000F37D19D
:10A9D000BA4205F101051FD299F800300026B9E707
:10A9E0000A22C8E7A642EAD201996FF0004C881EFD
:10A9F000B44400EB440001EB4C0121F8023F8842D3
:10AA000003F10103F9D1DAE76FF00043019A4FF641
:10AA1000FF71234422F81310012003B0BDE8F08F2A
:10AA200002F07F06032BC2F3D415D9F83412A6EB3B
:10AA3000020814BF4FF4807480240D44B8447FE7AB
:10AA400099F80030022BDFD06FF04043019A4FF0AD
:10AA5000FF31234442F82310DAF80020B8E700BFA2
:10AA6000A01E0024F8B590F838300446032B49D8CE
:10AA7000DFE803F0022B343F284BC0681A78D3F884
:10AA80004412032AD3F8AC51D3F8C8210CBF802656
:10AA90004FF48076226101FB06F1971900EB41200B
:10AAA000A5EB4125E060D3F8B001C3F8AC51A0EBB1
:10AAB0004121E06AC3F8C871C3F8B011C4E90C279A
:10AAC00048BB6262012384F8383000211448FFF744
:10AAD000E9FE012811D1022384F83830626B04F1B9
:10AAE00030010120FFF716FF012806D1032384F867
:10AAF000383000212046FFF7D5FE431EDBB2012B84
:10AB000001D9F8BD022094F82830062BF9D1002392
:10AB100084F82830F8BD921B2263D3E7A01E0024DE
:10AB2000442000242DE9F04F3D4D012883B00C4610
:10AB30002F788CBF4FF0000B4FF0010B1646032F00
:10AB40000B682ED0022F51D14FEA13284FF4807991
:10AB5000DFB20138012819D84FF0010A9E425CD9B2
:10AB6000D5F8AC211AB1D5F8C811994241D0D5F821
:10AB700034020023092201A94044FFF795FD012872
:10AB800018D0022809D028B12368E7E787B1FEF77B
:10AB900085FC022003B0BDE8F08F022003B0BDE8C1
:10ABA000F08F4FF08009C3F3D41803F07F07D0E78C
:10ABB000CA46D3E7019A2B78022B14D0032BECD191
:10ABC00052F8273023F07043B3FA83F357445B09FC
:10ABD0005B4523681FD053444F452360EBD308F1F6
:10ABE00001080027BAE732F81730EDE74FF4807913
:10ABF000D9E7D5F84412013A02EB41224902B2FBEF
:10AC0000F1F21344B3FBFAF20AFB12320AB15344D5
:10AC10009B1A2360A2E7B342BCD303202660B9E7A6
:10AC2000A01E0024F0B5104D83B00E462B78022BE9
:10AC300015D1070AC4B2D5F834020023032201A9B2
:10AC40003844FFF731FD012807D12B78022B019BF7
:10AC50000CBF23F8146043F8246003B0F0BDC0F3C8
:10AC6000D41700F07F04E6E7A01E00242DE9F04190
:10AC7000002990F83C3082B0044614BF0221002124
:10AC8000042B72D8DFE803F0030C38436000FFF7B1
:10AC900009FE012867D1626B002A6CD184F83C0060
:10ACA000DFF8F0804FF6F776394F1AE0B54294BFDF
:10ACB0000025012501A9002D43D1FAF7FFFF012846
:10ACC00029464DD1206BFFF7ADFF012848D1019AED
:10ACD000D8F84832511E22638B4228BF0B46C8F871
:10ACE000483298F80030206B032B85B2DED1B84291
:10ACF00094BF00250125DDE7426B04F130010020FF
:10AD0000FFF708FE01282ED1032384F83C30214BA5
:10AD10000021E56AD3F8C82103F5D270C3F8C85101
:10AD2000551BD3F8442202FB05F2D3E96B6506EB11
:10AD3000422605EB4222C3E96B62FFF7B3FD01280F
:10AD400011D1042384F83C3094F82830042B02D12C
:10AD5000002384F82830A36B8BB12046984701204C
:10AD600002B0BDE8F0810228FAD194F82830042B13
:10AD700009D00220F4E7022384F83C30BDE701202B
:10AD800002B0BDE8F0810023022084F82830E7E714
:10AD9000F7FFFF0FA01E002438B590F834300446AA
:10ADA000052B40D8DFE803F01E03390F1863006B52
:10ADB0004FF0FF31FFF736FF012834D1E06AA0BB26
:10ADC000032384F8343000212046FFF76BFD01286F
:10ADD00029D1042384F8343094F82830082B28D063
:10ADE000012038BD234D00F130010120D5F83C226F
:10ADF0000232FFF797FE012828D00238C0B201289E
:10AE000011D8052384F8343094F82830082B15D055
:10AE10000123022085F8E93138BDC06A216BFFF7B4
:10AE200001FF0128CCD0002038BD022384F8343043
:10AE3000F4E70023012084F8283038BD00230220E5
:10AE400084F82830012385F8E931E5E7D5F8442274
:10AE5000E368206B03EB4223E26AC5F84802C4E9C9
:10AE6000033002B96062012384F83430A0E7014D59
:10AE7000CAE700BFA01E00240378022B0FD00C4AA3
:10AE80004368D2F84C1200690B40D2F844120238E1
:10AE9000D2F840225B0A01FB003010447047044B9B
:10AEA0004268D3E98D0100EB410000EB522070476E
:10AEB000A01E00242DE9F04790F8384082B00546E6
:10AEC000032C00F29A80DFE804F00218610BFFF710
:10AED00063FF01280FD0022809D1032385F83830F9
:10AEE00000202B6C022485F8280003B198472046E7
:10AEF00002B0BDE8F08785F838002B78022B51D0DE
:10AF00003F4A6B68D2F84C2203EA0208C8F34F2884
:10AF10002846DFF8EC90FFF7AFFF0646A8EB0008E5
:10AF2000022201A930460023FFF7BEFB08EB06070B
:10AF300001284FF40072BFB24FF00001044606F141
:10AF40000106D4D1019850F095FBEB694FF40071E4
:10AF500028460BB16B685BB3D9F844325A1E97424E
:10AF600006D2FFF717FB0028DAD1FEF797FAD7E7EA
:10AF7000C3EBC3532846590201F50071FFF70AFBE2
:10AF800008B9FEF78BFA022385F8383000222B6CC3
:10AF900085F8282053B1012428469847204602B05E
:10AFA000BDE8F0876B68C3F34F28B1E701249EE743
:10AFB000019B4FF020322E244FF0100C1A605A6083
:10AFC0001C70C3F80720D5F824E01A625A62CEF349
:10AFD0000F4A83F8204083F82140C3F8272083F8E4
:10AFE0000BC0EA6BA3F81AE0C2F30F44A3F814A055
:10AFF0005A879C8683F82BC0AEE7002477E700BF12
:10B00000A01E0024B1F904300F2B2DE9F0410C46AD
:10B0100082B01646054633D02846FFF72DFF95F936
:10B020001B800746B8F1FF3F34D02D4B03EB0812CD
:10B03000D26990420BD0FEF731FA2846FFF782FA28
:10B04000D0B100230120336002B0BDE8F0819969DE
:10B0500001EB48210029F0D0A388284601331BB218
:10B0600001EB4311A3803160FFF706FF0346012087
:10B07000236002B0BDE8F081002002B0BDE8F0819D
:10B080004FF40071FFF786FA0028F5D04FF6FF73F2
:10B09000A380C1E72846FFF755FA0028CDD10FB9A4
:10B0A000FEF7FCF938460023112201A9FFF7FCFA4C
:10B0B0000128C2D10A4B01999B69CB1A48BF03F200
:10B0C000FF13B3F5B05F4FEA632204D24FFA82F860
:10B0D00085F81B80BEE7FEF7E1F90199F8E700BFAC
:10B0E000A01E00242DE9F04390F8303089B00446CA
:10B0F000042B00F2A280DFE813F0A300AC000500EF
:10B100008400E000C54D95F81432002B40F0958086
:10B1100004F11C0901AEC24F4FF0090832464946FE
:10B120003846FFF76FFF012840F03A810198002868
:10B1300000F01A8103780BB1E52BEFD1AA69821ACE
:10B1400048BF02F2FF12B2F5B05F4FEA622380F00F
:10B150005F811B01B34A13449A7B042A0CD0D5F8B3
:10B16000CC2004210132C5F8CC205A609973D5F85F
:10B17000D0300133C5F8D03095F906325E1C09D0C5
:10B180000233FF2205EB031385F80622DA7A6FF308
:10B190000002DA7295F907325A1C0ED00233FF21F1
:10B1A00005EB0313DA7A85F80712C2F3450101397A
:10B1B00021EAE17161F34602DA722022002150F0A7
:10B1C00059FA2346019A05A853F8315F596815606A
:10B1D000516019899B7A11819372019B627EDA72A8
:10B1E00044F0F8FFBDF81430002B40F04D8144F2DC
:10B1F0008172019903200A82CB810A83CB8284F871
:10B200003000237E980600F1CE802046FAF784FDB8
:10B210002369002B00F0D380237E03F0F70213F0A4
:10B220000403227640F0D980122A00F0DF80002249
:10B23000E36A204684F82820984709B0BDE8F083E7
:10B240007748FAF769FD4FF6FF720123228484F8EC
:10B25000303004F11C0701AE714D04F13109324662
:10B2600039462846FFF7CEFE01282DD00228E4D12A
:10B270006A4D95F906325A1C09D00233FF2205EBBC
:10B28000031385F80622DA7A6FF30002DA7295F971
:10B2900007325F1C0ED00233FF2105EB0313DA7A6D
:10B2A00085F80712C2F34501013921EAE17161F322
:10B2B0004602DA72042384F830300020E36A2070FA
:10B2C000984709B0BDE8F083DDF804800B224946B9
:10B2D0004046B8F1000F00F0A78098F80030002B2E
:10B2E00000F0A28050F0ACFA0028B8D1B8F81430C1
:10B2F000B8F81A20494D42EA0342D5F84432626256
:10B300005A02D8F81C30B3FBF2F102FB1131A360F2
:10B3100009B113445B1AE36098F80B30637695F932
:10B320000632581C09D00233FF2205EB031385F8BF
:10B330000622DA7A6FF30002DA7295F90732591CA5
:10B340000ED00233FF2105EB0313DA7A85F80712DA
:10B35000C2F34501013921EAE17161F34602DA7273
:10B36000032384F830304CE795F8EC313846022B53
:10B37000A0D095F8141200299CD1D5F80022D5F858
:10B38000483285F8148285F8241285F82012C5E920
:10B390008A11C5E98623FFF78DFD01283FF4BEAE73
:10B3A000022887D049E70023112205A9E069FFF7A9
:10B3B0007BF901283FF429AF09B0BDE8F083237E73
:10B3C00019077FF534AF154B93F8CC21002A7FF491
:10B3D00034AF072283F8CC2129E70023E26AA16871
:10B3E000204684F82830FFF745F926E7E56A04216E
:10B3F000626A204684F83C306363A56384F82810B1
:10B400006362C4E90233C4E90B22FAF785FC14E74E
:10B41000FEF744F801986FF00F039BE6A01E00248E
:10B420008C200024BC1E0024284D95F906325A1C9D
:10B4300009D00233FF2205EB031385F80622DA7ADE
:10B440006FF30002DA7295F907325F1C0ED00233F7
:10B45000FF2105EB0313DA7A85F80712C2F34501E1
:10B46000013921EAE17161F34602DA72237EDE06D8
:10B470007FF520AF1648FAF74FFC4FF6FF72022314
:10B48000228484F830303EE6124B05A902A8B3F9B5
:10B49000602044F0F5FE9DF80C309DF80D00DB02B5
:10B4A0009DF80A509DF80B20BDF8081043EA4013A0
:10B4B00042EA45129DF80E00A1F2BC7143EA500326
:10B4C00042EA41229BB292B293E600BFA01E002442
:10B4D0008C200024105D0024014B1B681B6A184758
:10B4E000B45A0024024B186808B1836918477047A2
:10B4F000B45A002410B5074C606D40B13AF08EFB91
:10B5000094F8513013B180F00100C0B210BD012099
:10B5100010BD00BF105D002410B54379164C002B00
:10B5200014BF0122002284F8502019D094F865300D
:10B53000003B18BF012384F85930FFF7DBFF28B91F
:10B54000237E84F824000133237610BD47F040FDAC
:10B5500048B1237E0022013384F82420237610BDD5
:10B5600084F8243010BD054B012220761B6884F836
:10B570002420636110BD00BF105D00242438002426
:10B5800010B547F025FD48B10A4C237E0133DBB2EC
:10B59000072B237603D9002384F8243010BDFFF74E
:10B5A000A9FF0028F7D0044B01221B6884F824204F
:10B5B000636110BD105D0024243800242DE9F84F8C
:10B5C000864C94F85050002D00F0ED8094F8242023
:10B5D000834E844F531E082B37D8DFE803F02C2FFF
:10B5E00094365A421436050048F04EFA002840F0CE
:10B5F000EC8063693268FA33934223D2FFF7C0FFCD
:10B6000094F82420E6E748F03FFA0028F1D0236AB6
:10B610000022012B227640F2DC80E169013B94F8A4
:10B6200059500131C4E9071305B1E2650823054605
:10B6300084F8243012E0022384F8243048F024FAFD
:10B64000002845D194F82420531EDBB2022B35D9B3
:10B65000082A18BF042A0CBF012500252846BDE88A
:10B66000F88F604B5B6A002B2ED15D4B0722E5689B
:10B670001B6884F824206361002DEFD0236901202A
:10B68000D4E90021A847DDE7636932686433934257
:10B690001AD2D7F82080B8F1000FF5D148F0F4F9AC
:10B6A0000028ADD00423E56884F8188084F824309D
:10B6B000002D00F0888040462369E1E7484B62692D
:10B6C0001B689B1AC82B73D800252846BDE8F88F45
:10B6D00047F01CFB0028B5D194F86930002BA3F18A
:10B6E0000203B3FA83F314BF022201225B096276DC
:10B6F000A37647F00BFB002880D1D4F8B8200323B1
:10B70000A26284F8243047F001FB8246002899D1D8
:10B7100094F89C104FF0040EB4F89EB00323D4F8B4
:10B72000A020C4F820A0D4F8A0704FEA126CD4F87E
:10B73000A06084F82E103F0CD4F8A090360A94F83C
:10B74000A48094F8A55094F8A520D4F8A80025FA70
:10B750000EF5B4F8AEA002F00F02B4F8AE1084F803
:10B760003160C1F30B11B4F8AE6084F8385041EA8F
:10B770001A2106F00F0584F83920724601F00F01F6
:10B78000A4F82CB084F82FC001F5FA6184F8307069
:10B7900084F8329084F833806063618784F83C5089
:10B7A00084F824E051E7284684F82450BDE8F88F57
:10B7B000FFF7E6FE94F82450082D18BF042D0CBFA7
:10B7C000012500254AE7054648E7042384F824308C
:10B7D00044E7FAD1FEF744FE34E700BF105D0024D1
:10B7E00024380024484C002408B5D0F8B4325B68F3
:10B7F0009847002008BD00BF08B5D0F8B4321BB18F
:10B800001B68984700B908BD022008BDF0B5D2E911
:10B810000236156933435669224C2B439569645CA3
:10B820003343D669204F2B43956A334306592B4344
:10B830003740D66A05193B430351AEB16F69D2F860
:10B8400038C027F00707D2E90C3E1E433E436E6125
:10B85000065926F0C07646EA0E060651035923F42F
:10B86000C00343EA0C030351176A566AD2E9003455
:10B870000E4AEC60AB6090426B684FF001000C4CDC
:10B8800004EA03040B4B0B4444EA07044FEA830326
:10B890006C6018BF20331A6822F0FF0232431A602E
:10B8A000F0BD00BFB4C609081F80FCFF00000240C5
:10B8B0000000FFFF0082001070B46A4C0D1E6A4A3F
:10B8C0000346645C18BF0125821A005918BF012283
:10B8D00020F00100185132BB2DBB6448644A00249B
:10B8E00021250A440460446092008460C4600461BD
:10B8F0004561106820F0FF00106021B93F2201204F
:10B900009A6070BC7047012932D002292BD00329DC
:10B9100044D0042947D0052934D006294BD0072923
:10B9200055D00020EDE75348181A18BF01209DB9E3
:10B9300090B951488D00514A002421262A440460C0
:10B9400044608460C46004614661106820F0FF00B8
:10B9500010600029D7D1D1E74C1E18BF01246AB965
:10B9600064B94748BAE74FF47C1201209A60C8E7EF
:10B970004FF47462084670BC9A60704738B934B9A5
:10B980004048D7E74FF474620120DA60B9E78C1EB3
:10B9900018BF01245AB954B93B489FE74FF074626D
:10B9A00001209A60ADE73F220120DA60A9E738B9AB
:10B9B00034B93648BEE74FF47C120120DA60A0E7C4
:10B9C000CC1E18BF01243AB934B9314886E74FF08C
:10B9D00074620120DA6094E710B90CB92D48A9E728
:10B9E0000C1F18BF012412B90CB92B4876E710B907
:10B9F0000CB92A489EE74C1F18BF012412B90CB994
:10BA000027486BE710B90CB9264893E78C1F18BF7D
:10BA1000012412B90CB9244860E710B90CB92348C5
:10BA200088E7114A934203D1072901D1204855E7FD
:10BA30000F4A00240C4D21260A441E48AB424FEA0F
:10BA400082020460446018BF20328460C4600461D4
:10BA50004661106820F0FF00106000297FF453AFAA
:10BA60004CE700BFB4C609080000024010000240C5
:10BA7000008200100004024010040240200802402E
:10BA800028000240280402404000024040040240D6
:10BA90005800024058040240700002407004024006
:10BAA0008800024088040240A0000240A004024036
:10BAB000B8000240B80402402DE9F0479F4A002533
:10BAC0009F4E82B0036882469E49846D934218BFA0
:10BAD000B342019508BF01260D68276818BF0026EC
:10BAE00021684AD03032DFF86CE29748734518BFBE
:10BAF00093420EF1480E0CBF01220022834208BF80
:10BB000042F001023030734508BF42F001020EF1ED
:10BB1000300E834208BF42F0010200F55C707345AD
:10BB200008BF42F001020EF55C7E834208BF42F07E
:10BB300001023030734508BF42F001020EF1300EB1
:10BB4000834208BF42F001023030734508BF42F023
:10BB500001020EF1300E834208BF42F00102303084
:10BB6000734508BF42F00102834208BF42F0010260
:10BB70001AB9764A934240F00B82DAF85C10082238
:10BB800001F01F0C02FA0CF2174240F08D8127FAE7
:10BB90000CF2D2070CD55A69100609D5012202FA17
:10BBA0000CF2A260DAF8542042F00202CAF85420E3
:10BBB0004FF0040E0EFA0CF038425BD0002E4FD13D
:10BBC000634ADFF89091DFF880814B4518BF9342BC
:10BBD00009F148090CBF01220022434508BF42F089
:10BBE000010208F130084B4508BF42F0010209F19B
:10BBF0003009434508BF42F0010208F55C784B4527
:10BC000008BF42F0010209F55C79434508BF42F0E4
:10BC1000010208F130084B4508BF42F0010209F16A
:10BC20003009434508BF42F0010208F130084B4596
:10BC300008BF42F0010209F13009434508BF42F054
:10BC4000010208F130084B4508BF42F001024345AC
:10BC500008BF42F001021AB93C4A934240F02F82D9
:10BC60001A68920706D5A060DAF8542042F0040260
:10BC7000CAF85420102202FA0CFC1CEA070F6FD0FD
:10BC8000002E46D1324A33482F4E834218BF93428A
:10BC900000F148000CBF01220022B34208BF42F06D
:10BCA00001023036834208BF42F001023030B34215
:10BCB00008BF42F0010206F55C76834208BF42F0FD
:10BCC000010200F55C70B34208BF42F00102303659
:10BCD000834208BF42F001023030B34208BF42F055
:10BCE00001023036834208BF42F001023030B342D5
:10BCF00008BF42F001023036834208BF42F0010221
:10BD0000B34208BF42F001021AB9104A934240F010
:10BD1000DE811A68C2F3C00212B3C4F808C01A6800
:10BD2000520300F18B811A68D60503D41A6822F0F9
:10BD300008021A60DAF8403093B10DE028000240A2
:10BD400010000240F800002470000240B8040240D5
:10BD5000580002404000024050469847DAF85C1014
:10BD600001F01F0120268E403E426AD0DAF8002002
:10BD7000A74BA848A84F824218BF9A4200F1300052
:10BD80000CBF01230023BA4208BF43F00103303740
:10BD9000824208BF43F001033030BA4208BF43F08B
:10BDA00001033037824208BF43F001033030BA420A
:10BDB00008BF43F0010307F55C77824208BF43F0F8
:10BDC000010300F55C70BA4208BF43F0010330374D
:10BDD000824208BF43F001033030BA4208BF43F04B
:10BDE00001033037824208BF43F001033030BA42CA
:10BDF00008BF43F001033037824208BF43F001031C
:10BE0000BA4208BF43F001031BB9844B9A4240F089
:10BE100073811368C3F300139BB1A6609AF83530A1
:10BE2000042B136800F0148113F4802F136800F0C2
:10BE30002D811C0340F13881DAF83C300BB15046BB
:10BE40009847DAF85430002B00F0DF80DAF85430ED
:10BE5000D8071FD5DAF8002004248AF83540136883
:10BE600023F0010313606E4BA3FB0535AD0A02E01E
:10BE70001368D90704D5019B0133AB420193F7D96D
:10BE800000238AF834301368DB074CBF03230123F7
:10BE90008AF83530DAF84C30002B00F0B680504686
:10BEA00002B0BDE8F0471847186840070AD518687F
:10BEB00020F004001860A260DAF8542042F0010279
:10BEC000CAF8542027FA0CF2D2077FF571AE554A12
:10BED0005148DFF86481834218BF934200F1480063
:10BEE0000CBF01220022434508BF42F0010208F1C5
:10BEF0003008834208BF42F001023030434508BF9A
:10BF000042F0010208F55C78834208BF42F001026A
:10BF100000F55C70434508BF42F0010208F13008AB
:10BF2000834208BF42F001023030434508BF42F06F
:10BF3000010208F13008834208BF42F001023030AC
:10BF4000434508BF42F0010208F13008834208BFB0
:10BF500042F001023030434508BF42F00102834203
:10BF600008BF42F00102002A7FF415AE002E7FF4D4
:10BF700012AE04221E6802FA0CF23A4240F09F8090
:10BF8000102202FA0CFC17EA0C0F3FF4E9AE79E636
:10BF9000254A264E264DB34218BF934206F1280685
:10BFA0000CBF01220022AB4208BF42F0010228353B
:10BFB000B34208BF42F001022836AB4208BF42F04C
:10BFC00001022835B34208BF42F00102AB4208BF6C
:10BFD00042F0010212B9174A934216D1DAF85C50C6
:10BFE00004261A6805F01F05AE400E4273D05707AD
:10BFF00071D51004666040F19F80D10300F1A280EA
:10C00000DAF84830002B7FF44AAF02B0BDE8F08781
:10C01000100002402800024040000240B8040240E4
:10C02000B5814E1B58000240085402581C54025857
:10C030003054025894540258700002401B681B038D
:10C040007FF578AEDAF84830002B7FF485AE87E6CE
:10C0500023F01603DAF840501360536923F080038D
:10C0600053613DB3136823F0080313603F23002599
:10C07000012203FA01F1DAF85030A1608AF8345055
:10C080008AF83520002B7FF40AAFBEE713F48073E3
:10C090007FF4D2AE1168012421F0100111608AF8FA
:10C0A00034308AF83540C7E6DAF84430002B7FF4A4
:10C0B000C6AEC6E6DAF84830002BD3D1D6E7102258
:10C0C0001E6802FA0CFC17EA0C0F3FF449AE1A681E
:10C0D000C2F3800220E60226AE400E4210D097073F
:10C0E0000ED56660140433D5D0033DD4DAF844305D
:10C0F000002B7FF4D4AE88E71368C3F340038BE6CC
:10C100000826AE400E4280D011077FF57EAF196839
:10C110000122002621F00E0102FA05F51960DAF875
:10C120004C306560CAF854208AF834608AF83520AB
:10C13000002B7FF4B4AE68E7920603D41A6822F0AD
:10C1400004021A60DAF84030002B7FF4A8AE5CE7F6
:10C1500012F0200208D11968012421F00A011960A7
:10C160008AF834208AF83540DAF83C30002B7FF426
:10C1700096AE4AE7002860D038B590F835200346DF
:10C18000022A56D10168594A914249D01832914247
:10C1900046D030325648574C814218BF914200F188
:10C1A0004800554D0CBF01220022A14208BF42F0B9
:10C1B00001024834814208BF42F0010200F562707A
:10C1C000A94208BF42F0010205F56275A14208BF0D
:10C1D00042F0010204F56274814208BF42F001029C
:10C1E0004830A94208BF42F001024835A14208BFC9
:10C1F00042F001024834814208BF42F00102483057
:10C20000A94208BF42F00102A14208BF42F0010268
:10C21000814208BF42F0010212B9384A91420ED160
:10C220000422002083F835200B6823F001030B6003
:10C2300038BD802201205A6538BD0120704704F1C5
:10C24000C0542F4A2F4804F59F442F4DA14218BFD8
:10C25000914204F150040CBF01220022814208BF28
:10C2600042F001020868A94208BF42F0010220F032
:10C270000E002835A14208BF42F0010208602834B0
:10C280000868A94208BF42F0010220F00100A14263
:10C2900008BF42F00102086012B91C4A914217D14E
:10C2A0001C6E0121D86D226800F01F009D6D22F4E4
:10C2B00080728140586E2260D3E91A4269604460FE
:10C2C00032B11168186F5C6F21F4807111604460A5
:10C2D000002401211A6D83F8344083F835101AB117
:10C2E00018469047204638BD104638BD1000024021
:10C2F0004000024070000240A0000240B80402402A
:10C300001C54025830540258445402589454025851
:10C31000002800F08A812DE9F047044690F83400A7
:10C32000012800F08481012094F83550854284F87A
:10C33000340007D000224FF4006384F83420636592
:10C34000BDE8F08725684FF0020C58480027584E8A
:10C3500084F835C0B54218BF8542DFF85CC106F1EC
:10C36000300667650CBF01200020524F654508BFAD
:10C3700040F001000CF1300CB54208BF40F0010064
:10C3800006F56276654508BF40F001000CF5627C59
:10C39000BD4208BF40F0010007F56277B54208BF13
:10C3A00040F001004836654508BF40F001000CF13F
:10C3B000480CBD4208BF40F001004837B54208BFF5
:10C3C00040F001004836654508BF40F001000CF11F
:10C3D000480CBD4208BF40F00100A7F58F67B54289
:10C3E00008BF40F00100A6F58F66654514BF824680
:10C3F00040F0010AB54218BFBD420CBF012600261D
:10C4000002D0BAF1000F59D02F68D4F858C027F0E5
:10C4100001072F60002E00F08480676ED4E91A0EA9
:10C420007860BEF1000F02D0D4E91C707860E76D2F
:10C430004FF03F09D4F8088007F01F07B8F1400F0C
:10C4400009FA07F7CCF808702F6827F480272F60C7
:10C450006B6000F0EF80A960EA601EB9BAF1000FCE
:10C4600000F0EE802B68226C23F01E0343F01603CD
:10C470002B601AB12B6843F008032B60236E1A68F7
:10C48000D20303D51A6842F480721A60BEF1000F1D
:10C4900005D0DEF8003043F48073CEF800302B680E
:10C4A000002043F001032B60BDE8F087400002400C
:10C4B00058000240B800024070000240654FDFF8AB
:10C4C0009CE1DFF89CC1754518BFBD420EF13C0EE2
:10C4D0000CBF01270027654508BF47F001070CF195
:10C4E000280C754508BF47F001070EF1280E654579
:10C4F00008BF47F001070CF1280C754508BF47F04D
:10C500000107D5F800E0654508BF47F001072EF0A8
:10C51000010ED4F858C0C5F800E017B94E4FBD421F
:10C520000DD1676ED4E91A0E7860BEF1000F02D00B
:10C53000D4E91C707860BAF1000F7FF478AF474FF0
:10C54000DFF81081DFF818E1454518BFBD4208F15A
:10C5500028080CBF01270027754508BF47F00107D1
:10C560000EF1280E454508BF47F0010708F12808DD
:10C57000754508BF47F001070EF1280E454508BF75
:10C5800047F00107754508BF47F0010717B9324F5B
:10C59000BD4255D1E76D4FF0010ED4F8088007F089
:10C5A0001F07B8F1400F0EFA07F7CCF804706B6064
:10C5B00043D0A960EA602B68226C23F00E0343F09D
:10C5C0000A032B60002A2DD02B6843F004032B6054
:10C5D000204B224A2249954218BF9D4202F13C025B
:10C5E0000CBF012300238D4208BF43F00103283113
:10C5F000954208BF43F0010328328D4208BF43F043
:10C6000001032831954208BF43F0010328328D42CF
:10C6100008BF43F00103954208BF43F00103002B1C
:10C620003FF43DAFD4F86CE028E7012070470220CA
:10C63000BDE8F087AA60E9600FE7AA60E960BAE7A1
:10C640002B68226C23F00E0343F00A032B60002AB0
:10C65000BAD1BDE71C5402589454025808540258E9
:10C660003054025838B50446864B87492268874DB6
:10C670008A4218BF9A42864801F160010CBF01232B
:10C680000023AA4208BF43F001034835824208BF95
:10C6900043F0010300F562708A4208BF43F00103D2
:10C6A00001F56271AA4208BF43F0010305F5627506
:10C6B000824208BF43F0010348308A4208BF43F07A
:10C6C00001034831AA4208BF43F0010348358242C2
:10C6D00008BF43F0010348308A4208BF43F001031A
:10C6E0004831AA4208BF43F00103824208BF43F029
:10C6F00001038A4208BF43F001033BB9A1F59561EC
:10C70000644B9A4218BF8A4240F0CE8011680023E1
:10C710002125204621F001011160136053609360D0
:10C72000D36013615561FDF727FAE26D3F2302F0F4
:10C730001F02934083602268574B5649524D8A42EC
:10C7400018BF9A424F4801F148010CBF0123002352
:10C75000AA4208BF43F001034835824208BF43F0B4
:10C76000010348308A4208BF43F001034831AA421E
:10C7700008BF43F0010305F56275824208BF43F02C
:10C78000010300F562708A4208BF43F0010301F51E
:10C790006271AA4208BF43F001034835824208BFD4
:10C7A00043F0010348308A4208BF43F00103483197
:10C7B000AA4208BF43F001034835824208BF43F054
:10C7C000010348308A4208BF43F0010301F1C05120
:10C7D000AA4208BF43F0010301F59F412F4D824259
:10C7E00008BF43F001032E488A4208BF43F001030B
:10C7F0003C31AA4208BF43F001033C35824208BFE6
:10C8000043F001033C308A4208BF43F001033C314E
:10C81000AA4208BF43F00103824208BF43F001036C
:10C820008A4208BF43F0010313B91E4B9A4211D14B
:10C830002046FDF735F9236E23B10020D4E91921F4
:10C84000186051606368013B072B11D90023C4E9CC
:10C850001B33636700236365184684F8353084F81A
:10C860003430C4E90F33C4E91133C4E9133338BD9C
:10C870002046FDF7C7F8E16E0020D4E91C320860BD
:10C880005A60E3E758000240400002407000024056
:10C890008800024028000240100002401C54025848
:10C8A00030540258945402581D4B1E491E4D8A4262
:10C8B00018BF9A421D4801F13C010CBF012300231F
:10C8C000AA4208BF43F001033C35824208BF43F04F
:10C8D00001033C308A4208BF43F001031168AA42B9
:10C8E00008BF43F0010321F00101824208BF43F079
:10C8F0000103116013B90E4B9A420FD10023204659
:10C90000136053609360D3601361FDF735F9E26DF6
:10C91000012302F01F02934043600CE7012038BD61
:10C92000085402581C5402583054025844540258B7
:10C9300094540258A549F8B504460868002C00F044
:10C9400065812268A24B9A4249D018339A4246D058
:10C950003033A04EA04DB24218BF9A4206F14806AD
:10C960000CBF01230023AA4208BF43F00103303566
:10C97000B24208BF43F001033036AA4208BF43F079
:10C98000010305F55C75B24208BF43F0010306F5EB
:10C990005C76AA4208BF43F001033035B24208BFBB
:10C9A00043F001033036AA4208BF43F0010330359B
:10C9B000B24208BF43F001033036AA4208BF43F039
:10C9C00001033035B24208BF43F00103AA4208BF59
:10C9D00043F001031BB9814B9A4240F03C81022392
:10C9E000002584F8353084F83450136823F00103AF
:10C9F000136004E00B681B1A052B00F2BF8013685C
:10CA0000DD07F7D4D4E9023120690B431768D4E974
:10CA1000051603430B437249D4E9070533433940F4
:10CA20000343606A2B43042841EA030100F0AD8010
:10CA30001160536923F00703184350612046FDF746
:10CA40009BF8E26D3F2302F01F029340836022684F
:10CA50005F4B64495F4D8A4218BF9A42624801F1B8
:10CA600048010CBF01230023AA4208BF43F0010381
:10CA70004835824208BF43F0010348308A4208BF6C
:10CA800043F001034831AA4208BF43F0010305F512
:10CA90006275824208BF43F0010300F562708A426A
:10CAA00008BF43F0010301F56271AA4208BF43F0D9
:10CAB00001034835824208BF43F0010348308A42EF
:10CAC00008BF43F001034831AA4208BF43F0010305
:10CAD0004835824208BF43F0010348308A4208BF0C
:10CAE00043F0010301F1C051AA4208BF43F0010322
:10CAF00001F59F413D4D824208BF43F001033C4890
:10CB00008A4208BF43F001033C31AA4208BF43F008
:10CB100001033C35824208BF43F001033C308A42A6
:10CB200008BF43F001033C31AA4208BF43F00103B0
:10CB3000824208BF43F001038A4208BF43F0010369
:10CB400013B92C4B9A4213D12046FCF7A9FFA368D6
:10CB5000802B5DD06368206EDDB2013BD4E91921E2
:10CB6000072B0560516047D90023C4E91B33636775
:10CB700000200123606584F83530F8BD20220323AE
:10CB80000120626584F83530F8BDD4E90B50A36A02
:10CB9000284301431160506920F00700184340F01A
:10CBA0000400002D3FF449AF002E39D1012B4DD0A8
:10CBB00033F002037FF441AFEB017FF53EAF012379
:10CBC00040221846626584F83530F8BD34480024A8
:10CBD000100002404000024070000240B8040240D1
:10CBE0003F8010FE28000240580002401C540258AA
:10CBF00030540258945402582046FCF703FFE16E6B
:10CC00000020D4E91C3208605A60B1E70120F8BD69
:10CC10000023A16ED4E91802636003605160A3E7AA
:10CC2000B6F5005F04D0022BC9D9032BC4D004E7AA
:10CC3000032B3FF602AF01A151F823F0BFCB04084C
:10CC4000B9CB0408BFCB04084DCC0408B5F1C07FB4
:10CC50007FF4F3AEB3E7344B344935488A4218BF0A
:10CC60009A4201F12801334D0CBF01230023824277
:10CC700008BF43F001033C308A4208BF43F0010380
:10CC80003C31AA4208BF43F00103824208BF43F08F
:10CC900001038A4208BF43F0010313B9264B9A42AD
:10CCA0003AD102230021254F84F83530A36884F857
:10CCB0003410402B116807EA01072BD0802B0CBFE2
:10CCC0004FF48041002123692046E668DB0865694E
:10CCD000DFF870C043EAD603A66943EAD503E569E5
:10CCE00043EAD603164E43EAD5031644256A43EABF
:10CCF0001513ACFB06653B432D091943AD001160CC
:10CD0000E565FCF739FFE26D012302F01F02934055
:10CD100043609CE61021D6E7402203230120626590
:10CD200084F83530F8BD00BF085402581C5402582E
:10CD30003054025858540258945402580F00FEFFC1
:10CD4000F8ABFDA7CDCCCCCC0B4B01E0013B10D018
:10CD50000269002AFADA0369074A43F00103036112
:10CD600001E0013A05D0036913F00103F9D1184637
:10CD700070470320704700BF400D0300144B10B4F0
:10CD8000046C9C421AD800F530600023012903612D
:10CD9000036943F400230361036943F0180303614B
:10CDA000036943F0C043036104D14261036843F067
:10CDB0008023036000205DF8044B7047D0F8003BEF
:10CDC00000F53060002BE0DA00205DF8044B70477E
:10CDD0000A30544F002807DB00F01F0101234009EF
:10CDE000024A8B4042F82030704700BF00E100E06B
:10CDF0002DE9F04F0D6883B0002D00F0C4800023B2
:10CE0000DFF82C82DFF82CE201229A4012EA050CAE
:10CE100000F0B4804C6824F01007022F40F0B68078
:10CE2000DF0803F0070A4FF00F0B0E6900EB8707CE
:10CE30004FEA8A0AD7F820900BFA0AFB06FA0AF69C
:10CE40004FEA430A29EA0B094FF0030B46EA0909A6
:10CE50000BFA0AF604EA0B0BC7F820906FEA0609F2
:10CE600007680BFA0AFB27EA06064BEA0606066085
:10CE70008768C4F3001607EA090BCF689E4007FADB
:10CE80000AF747EA0B078760476827EA020216435A
:10CE90004660C668E7008A6806EA090902FA0AF2EB
:10CEA00042EA0902C26069D5D8F8F47023F0030998
:10CEB00003F003020F2647F0020709F1B049920080
:10CEC000C8F8F47009F58069D8F8F47006FA02FA27
:10CED00007F0020701974D4F019EB842D9F808604C
:10CEE00026EA0A0620D007F58067B8426BD0484F83
:10CEF000B8426DD0474FB84260D0474FB84271D06A
:10CF0000464FB84273D0464FB84266D0454FB842FC
:10CF100072D0454FB84274D0444FB8420CBF092775
:10CF20000A2707FA02F21643C9F808606FEA0C07ED
:10CF3000DEF80020E60354BF3A404CEA0202CEF885
:10CF40000020A203DEF804604FF0B04254BF3E4020
:10CF50004CEA0606CEF804601668E2024FF0B042D2
:10CF600054BF3E404CEA0606A4024FF0B04416609F
:10CF7000526854BF3A404CEA02026260013335FA0B
:10CF800003F27FF441AF03B0BDE8F08F4FEA430AEC
:10CF90004FF00309D0F800B0013F04EA090609FA8E
:10CFA0000AF9012F2BEA090B06FA0AF66FEA0909BA
:10CFB00046EA0B0606603FF66CAF59E7032707FA0F
:10CFC00002F21643B0E7012707FA02F21643ABE775
:10CFD000022707FA02F21643A6E7062707FA02F22B
:10CFE0001643A1E7042707FA02F216439CE7052738
:10CFF00007FA02F2164397E7072707FA02F21643E9
:10D0000092E7082707FA02F216438DE7000002585C
:10D0100000080258000C0258001002580014025870
:10D0200000180258001C0258002002580024025820
:10D03000004402588000005802689168890702D5B0
:10D040009368002070479168CB070ED5916803461E
:10D0500001F00D0101290AD0426D012042F01002B9
:10D060005A659A6D02439A6570470020704730B444
:10D070000E49032495680E48294041F00201916051
:10D080001460046803E00168091B022905D891684F
:10D09000C907F8D4002030BC70475A6D012042F017
:10D0A00010025A659A6D02439A65F4E7C0FFFF7F4C
:10D0B00034480024F8B501F00F05012600271C2193
:10D0C000C5EBC50401FB050100EB84043C31A264FF
:10D0D000236584F83C50676584F83D600369B3427A
:10D0E00008BFE264DAB200681DB9FCF7C1FD002098
:10D0F000F8BDFCF73FFE0020F8BD00BFF8B5D0F842
:10D10000B8322BB301EB8107064600EB8707FA69BB
:10D110005AB1D0F8D0C2C1EBC1040CEB8404606CEE
:10D12000B2FBF0F400FB14241CB10020C3F814027D
:10D13000F8BD01F07F05FC616046234605EB8505DF
:10D14000224606EB8505EC61FFF7B4FF2046F8BDEB
:10D150000220F8BD10B504210024C0F89412234623
:10D16000C46122462146D0F8D002FFF7A3FF204633
:10D1700010BD00BF10B5134602240A460021C0F8B6
:10D180009442C0E90733D0F8D002FFF793FF0020A4
:10D1900010BD00BF10B50C7882B00023D0F8C022BB
:10D1A00014F06004ADF8063016D0202C0ED14B7868
:10D1B000023B092B0AD8DFE803F0333909090909D2
:10D1C00009093F2F90F89C32032B5AD00224FBF719
:10D1D00011F9204602B010BD4B780B2BF6D80FF298
:10D1E000080C5CF823F000BF6DD20408CDD1040810
:10D1F000CDD10408CDD10408CDD10408CDD1040887
:10D2000043D20408CDD10408CDD10408CDD10408FF
:10D21000C5D104085FD204088B7800241360D8E7D6
:10D22000111D01220024FFF7A5FFD2E711460122BC
:10D230000024FFF79FFFCCE74B8800241B0A5360B4
:10D24000C7E74B881B0A222B1FD0212BBED1CA88CF
:10D250001149092A28BF0922FFF78CFFB9E790F886
:10D260009C32032BB2D18B789360B2E790F89C226A
:10D27000032AABD102220DF106011C46FFF77AFF0B
:10D28000A7E702F108010122E6E7CA880349362A26
:10D2900028BF3622E0E700BF900400245804002491
:10D2A00070B5C1EBC1040D4600261C2100EB8404BF
:10D2B00001FB0501C4F80822C4F8103201F5FE7123
:10D2C00084F8FC51C4F8146284F8FD610369012BF1
:10D2D00008BFC4F80C22DAB200681DB9FCF7C8FC1C
:10D2E000002070BDFCF746FD002070BD2DE9F04127
:10D2F0000A7882B000270D4612F060060446D0F886
:10D30000B8828DF80570ADF8067013D0202E17D1B5
:10D31000CB88EBB1120641D5D0F8BC621A46414623
:10D320006878B3683E469847EA8841462046FFF74A
:10D3300021FF09E04B780A2B21D00B2B29D093B188
:10D3400020460226FBF756F8304602B0BDE8F081D1
:10D35000D0F8BC421E461A464878A3689847304623
:10D3600002B0BDE8F08190F89C32032B2AD002264F
:10D370002046FBF73FF8304602B0BDE8F08190F858
:10D380009C32032BF3D101220DF10501FFF7F2FED0
:10D39000DAE790F89C32032BD6D0E8E74A780325E9
:10D3A00088F80132394688F800224246C0F85C31DC
:10D3B0003E46C0F86031D0F8D002C4F89452FFF76E
:10D3C0006FFFC1E702220DF10601FFF7D3FEBBE7B5
:10D3D00070B5054641B9D0F894320C46032B10D0F5
:10D3E000052B1FD0002070BDD0F8B4329B6933B13B
:10D3F00090F89C22032A02D19847002070BD022099
:10D4000070BDD0E958639E4212D8D0F8B4321B697F
:10D4100023B190F89C22032A00D198472846FFF7B1
:10D4200099FEDFE7C5F89412FAF788FF204670BD31
:10D43000F61AD0F8D002B342C5F8606128BF33466F
:10D440009BB2FFF72DFF204670BD00BF11F0800F8B
:10D4500001F00F01F0B44FF01C0442D1C1EBC10543
:10D4600004FB0104002600EB850504F5FE7485F835
:10D47000FD6165782170A260E37005B1E180022B47
:10D4800001D10023237190F8BC33012B53D001222A
:10D49000036880F8BC236178257891422CD003F58D
:10D4A000006605F00F0103F530638A40F16903EB74
:10D4B000451341EA0242F2611A68120405D50023BD
:10D4C00080F8BC331846F0BC7047A2681D68C2F3F0
:10D4D0000A02E47819492A4342EA84421143196056
:10D4E000EDE7C1EBC105012604FB010400EB850556
:10D4F0003C3485F83D60BCE705F00F06D3F81CC846
:10D5000003F5106203F50067B14002EB451241EAF2
:10D510000C01F96113681904D1D4A3681668C3F328
:10D520000A03E4780549334343EA844343EA8553D5
:10D5300019431160C3E70220F0BC7047008000105F
:10D5400010B50323044608228321D0F8D002FFF748
:10D550007DFF0123102063654EF054F8C4F8C0022B
:10D5600018B100230373184610BD022010BD00BF80
:10D570002DE9F041037C04460125002B3CD1022318
:10D580004FF400728121D0F8D002FFF75FFF2946E7
:10D5900002234FF40072D4F8D002E562FFF756FF81
:10D5A000C4F86C514FF00108032308228221D4F8FB
:10D5B000D002FFF74BFF4FF40770C4F840804EF0E5
:10D5C00021F80546C4F8B80278B3D4F8BC32002775
:10D5D0001B689847267CC5F814724146D5F804228A
:10D5E000D4F8D002C5F81872C6B140233E46FFF702
:10D5F00057FE3046BDE8F081022340228121D0F859
:10D60000D002FFF723FF294602234022D4F8D0029C
:10D61000E562FFF71BFFC4F86C51C3E74FF40073DA
:10D62000FFF73EFE3046BDE8F0814646E1E700BF29
:10D63000154B014641F288321B6810B4134CA4FB11
:10D6400003035B0A02FB03F24AB1531E4A6B013B20
:10D6500012F0450F01D0920406D5581CF6D14FF0B8
:10D6600000405DF8044B70474B6B5B0709D4486B77
:10D670005DF8044B10F0010014BF0123044B8B63D1
:10D68000704704208863ECE7F8000024D34D621053
:10D69000C5002000474B10B41B68474CA4FB034354
:10D6A0005B0A02FB03F24AB1531E444C426B013B3E
:10D6B000224201D0920407D55A1CF7D14FF0004303
:10D6C00018465DF8044B7047436B5C073DD4436BD1
:10D6D00013F0010334D13A4B83630369DBB29942FF
:10D6E00031D14269374B1340002BE9D0002A2FDBA0
:10D6F000510030D4940030D4D00030D4110131D452
:10D70000540132D4D00133D4110234D4540235D46C
:10D7100090023FD4D1023AD4540335D4900330D48C
:10D72000D10343D414043ED4500439D4910434D4E6
:10D7300012F0080F14BF4FF400034FF48033BFE71B
:10D7400001228263BCE70123BAE704238363B7E7BE
:10D750004FF00073B4E74023B2E78023B0E74FF403
:10D760008073ADE74FF40073AAE74FF48063A7E737
:10D770004FF40063A4E74FF48053A1E74FF4005344
:10D780009EE74FF480239BE74FF4003398E74FF474
:10D79000004395E74FF4804392E74FF480038FE70F
:10D7A0004FF400138CE74FF4801389E74FF4002304
:10D7B00086E700BFF8000024D34D6210450020002A
:10D7C000C500200008E0FFFD70B4816041F237140D
:10D7D000C66841F28832034D372135402C43C4607E
:10D7E00070BC57E7C0E0FEFF114B0146114A1868B4
:10D7F00041F2883330B4104C0025A4FB00408D600A
:10D80000CC68400A224003FB00F342F48052CA6015
:10D8100002E04A6B120605D4013BFAD24FF00040F9
:10D8200030BC7047054B002030BC8B63704700BF95
:10D83000F8000024C0E0FEFFD34D6210C5002000B8
:10D84000C16841F20C130E4A41F0800170B5C1600D
:10D850000026C16804460B4D21F04001C1600C2137
:10D860008660C66835402B43C360FFF713FFE3684B
:10D87000B0F1007F08BF002023F08003E36070BD9B
:10D8800000E1F505C0E0FEFF70B4816041F21014C4
:10D89000C66841F28832034D102135402C43C460E4
:10D8A00070BCF7E6C0E0FEFF2DE9F04F5A4D83B0A3
:10D8B00006460C4695F8247091469A46042F09D0E6
:10D8C000082F03D0002003B0BDE8F08FFCF7C8FD9F
:10D8D0000228F7D10122514B51484FF400719A6050
:10D8E0000262C3E90041002C40D0DFF83C8198F887
:10D8F0003030012B28D1731CD8F8502000279342D8
:10D90000C8F834702BD80323D8F8000088F83030DA
:10D91000D8F83830C762012BC8E909414FF40071CB
:10D9200014BF4FEA462BB346FFF7AEFF034618B3CA
:10D93000D8F8002001213B489063D8F834201343E5
:10D94000C8F8343088F83010FDF71AFEEC68002C67
:10D95000B8D000222B6969681046A047B2E7D8F812
:10D96000343043F00073C8F83430EDE72E4A536B7F
:10D9700043F000635363E7E74FF0FF314FF4007269
:10D9800001904FF0810ED8F80000012741F2111CE0
:10D9900041628262C26A254922F0FF0242F092028D
:10D9A000C262C26842F04002C26084650765C8F87E
:10D9B0002CE0C0F808B0C268114041F2883241EA58
:10D9C0000C0C1121C0F80CC0FFF764FED8F8002041
:10D9D00060B11449019B9163D8F834201043C8F812
:10D9E000340088F83070C8F82C30ADE7D36B0521CF
:10D9F000DFF83CC0384643F495732C606E60D36307
:10DA0000DCF80030C5F80C9085F82410C5E904A3B3
:10DA100003B0BDE8F08F00BF105D0024704C0024FF
:10DA2000484C0024FF0FE01FCC4B0024C0E0FEFF59
:10DA3000243800242DE9F047064682B00D46914671
:10DA40009A468A4C94F8241004290CD0082906D14F
:10DA5000E369B34207D0FCF703FD0228F2D00120AE
:10DA600002B0BDE8F087D4F85C802560C8F34F278A
:10DA70004FEA582266600F2F03D8236A0193002BC8
:10DA800068D101204FF4007807460123DFF8F0C188
:10DA9000062225F01F012372CCF8243005EB080381
:10DAA000C4F80C905B1AC4F810A084F82420BFF3CB
:10DAB0004F8F002B0EDD013B01F12002DFF8C4C1C6
:10DAC00023F01F0313449A42CCF86812114602F166
:10DAD0002002F8D1BFF34F8FBFF36F8F002D6BD0B3
:10DAE000DFF8949199F83030012B26D13044D9F8E1
:10DAF000503000229842C9F834204ED8D9F8383036
:10DB00000321D9F80000012B89F830104FF400717F
:10DB1000C26218BF7602C9E90758FFF7B5FE0028B0
:10DB200050D0D9F80020012351499163D9F834200D
:10DB30001043C9F8340089F83030FDF721FDE5685D
:10DB4000002D00F090800120236900226168A84721
:10DB5000032085E794F85910002992D0B8F5005FAA
:10DB600022D044484FF40072294608F5007740441B
:10DB70004DF00EFD019B7A0AE765012BC7F34F2795
:10DB800012D0102F10D0E269013B04210220013293
:10DB9000236284F82410E26162E7D9F8343043F05C
:10DBA0000073C9F83430C8E792B238464FEA4728C4
:10DBB000304D013AB61A68E72F4A536B43F00063C1
:10DBC0005363BAE7D9F800004FF0FF3301224362F4
:10DBD000C0F828809742C36A23F0FF0343F0900304
:10DBE000C362C36843F04003C3608565026520D902
:10DBF000A0232249C9F82C3041F219138660C2686B
:10DC0000114041F288320B431921C360FFF742FDF6
:10DC100000B3D9F800100122154D00238D63D9F807
:10DC200034100843C9F8340089F83020C9F82C3082
:10DC300083E790231149C9F82C3041F2181386600C
:10DC4000C268114041F288320B431821C360FFF7CC
:10DC500021FDDDE7D9F80020D36B43F48D73D36346
:10DC600002B0BDE8F0870320FAE600BF105D002493
:10DC7000FF0FE01FE45D0024CC4B0024C0E0FEFF5A
:10DC8000484C002400ED00E0034A0130116813689D
:10DC90005B1A8342FBD370473448002438B5114BDC
:10DCA000114A1B68A2FB03239B09013BB3F1807F50
:10DCB0000CD20E4A05460E49F0205360002407237B
:10DCC0000F2D81F823009460136001D9012038BD25
:10DCD00029464FF0FF30F3F74FF8064B2046C3F8C4
:10DCE000945138BDF8000024D34D621010E000E0DC
:10DCF00000ED00E00803002438B50021144A036851
:10DD00000446C0F88810156819680A070CD41B6807
:10DD10005B0713D420220023C4F880201846C4F8DF
:10DD2000842084F87C3038BD2A464FF40011F3F784
:10DD300083FC58B923681B685B07EBD52A464FF470
:10DD400080012046F3F778FC0028E3D0032038BD9B
:10DD500034480024836ADA0710B406D50168C46A1F
:10DD60004A6822F4003222434A609C0706D50168C3
:10DD7000046B4A6822F4803222434A60590706D570
:10DD80000168446B4A6822F4802222434A601A07E1
:10DD900006D50168846B4A6822F4004222434A6037
:10DDA000DC0606D50168C46B8A6822F480522243DF
:10DDB0008A60990606D50168046C8A6822F40052CC
:10DDC00022438A605A060AD50168446C4A68B4F551
:10DDD000801F22F4801242EA04024A600BD01B0624
:10DDE00006D50268C16C536823F400230B435360CB
:10DDF0005DF8044B70474A68846C22F4C0022243E9
:10DE00004A60ECE7036834495A6910B49C6944F0ED
:10DE100008049C619C6944F010049C611C6824F017
:10DE200001041C601C6921401961996821F440417A
:10DE3000996090F88110042901D0940633D490F8A9
:10DE4000811003290FD0510609D5D0F8841041F074
:10DE50000401C0F88410996941F040019961816A18
:10DE6000B1F5800F2AD0910509D5D0F8841041F082
:10DE70000101C0F88410996941F400719961D205DB
:10DE800009D5D0F8842042F00802C0F884209A69AD
:10DE900042F480729A6100235DF8044BA0F862306E
:10DEA000A0F86A307047D0F8841041F08001C0F8C3
:10DEB0008410996941F020019961C0E71406D2D518
:10DEC000D0F8841041F00201C0F88410996941F043
:10DED00080019961C7E700BF90FCFFFF03681969E3
:10DEE0005A69D3F808C02DE9F04101EA0205044659
:10DEF00090F8817005F06406042E4AD005F04500C4
:10DF000001284FD005F02600022800F0C88028071D
:10DF10005BD59A691CF4404F42F008029A619A69F5
:10DF200042F010029A619A6942F400629A611A6999
:10DF300022F008021A6108D0FFB2042F00F0BF805F
:10DF4000A26FD269002A40F0B7809A6812F4404F5D
:10DF500031D1B4F86A2092B26AB3616E0EE02268E1
:10DF6000126B41F8042B6166B4F86A20013A92B250
:10DF7000A4F86A20B4F86A2092B2E2B1E2680F2AEB
:10DF8000EDD8072A40F290801A8E21F8022B6166A4
:10DF9000EAE7436F9847236F2046984705F045030B
:10DFA000012B02D1236F2046984705F02605022D4C
:10DFB00075D0BDE8F0812046FFF724FF012384F8E7
:10DFC0008130D4F88430BDE8F081120501D50F0707
:10DFD0007BD415F4587FECD06E0609D5D4F8842094
:10DFE00042F00402C4F884209A6942F040029A6127
:10DFF000A80509D5D4F8842042F00102C4F8842091
:10E000009A6942F400729A61E90509D5D4F884202E
:10E0100042F00802C4F884209A6942F480729A613E
:10E02000AA0609D5D4F8842042F08002C4F88420DE
:10E030009A6942F020029A61D4F88420002AB8D06C
:10E0400019680CF4404C254A21F00101BCF5404F01
:10E050001960196902EA01021A613BD19A68E06FFE
:10E0600022F440429A6050B11D4B0365FEF782F8DE
:10E0700028B1D4F8843043F04003C4F88430A06F52
:10E08000002896D0164B0365FEF774F8002890D050
:10E09000D4F8843043F04003C4F8843089E7636FD8
:10E0A0002046BDE8F0411847226892F830200A70F7
:10E0B000616E0131616657E7032F3FF47AAFE26F7B
:10E0C000D269002A3FF441AF73E79A6942F40062D3
:10E0D0009A616EE7012384F881306AE794FCFFFFC0
:10E0E00099A1040803460221002210B41C681046BE
:10E0F00083F88110216821F001012160C3F8842098
:10E1000083F8802083F881205DF8044B704700BFBE
:10E110008449034602682DE9F04F834CA24218BFA0
:10E120008A42C46814BF0121002129D07F4882425D
:10E1300026D00F2C21D8D3F83CC004F108004FEAB8
:10E140005C15C00805FB0000082816D89D6A4FF032
:10E15000000BB5F5800F33D1744ED3F83080B24246
:10E1600003D011B1B8F5702F07D8B8F1000F01D165
:10E170004FEA0448B4EB184F24D90120BDE8F08FD2
:10E18000694804F10805674ED3F83CC0ED08B24277
:10E1900018BF8242654F4FEA5C160CBF0120002079
:10E1A00006FB0555BA4214BF834640F0010BBBF194
:10E1B000000F01D0102DE0D89D6AB5F5800FCBD0AF
:10E1C0004FF0000893F8816006F0FF07002E00F082
:10E1D000A08002269F69D3F804E083F88160B7F13C
:10E1E000806F1668D3F8389026F00106166000F0AC
:10E1F00083805E6BB5F5800F986847EA060A5F6A10
:10E200001E694AEA070746EA07065F6946EA070603
:10E210001F6A46EA0706DF6C46EA07069F6C46EA75
:10E220000006D86947EA060745EA000A9E6D4AEAF1
:10E230000C0C46EA07064CEA040446EA090644EADE
:10E24000080446EA0E069460D66029D0BEF1000F9D
:10E2500014D0116D1EF4800F21F00101116505D05D
:10E26000D168586D21F000410143D16000200122A6
:10E27000C3F8840083F88120BDE8F08F2DB9916840
:10E2800021F4C05141F400619160916821F4C061B2
:10E2900041F480619160116D21F001011165E5E7A4
:10E2A0001C6C012C14680CBF44F4004424F400449A
:10E2B00014605C6C012C14680CBF44F4804424F49A
:10E2C00080441460194CA2420CBF002101F00101EE
:10E2D00011B1B8F5702F1FD0BBF1000F02D0B8F507
:10E2E000F81F19D0116821F400511160D96A116426
:10E2F000BEF1000FC9D0ACE7BEF5800F7FF479AF57
:10E30000B9F1000F7FF475AF166846F480561660B9
:10E310006FE783F880705CE7116841F40051116089
:10E32000E4E700BF0038004000300140003C0040FE
:10E3300008B505F08DFF064B06499B69064AC3F3F5
:10E340000323CB5C03F01F03D840106008BD00BF5F
:10E350000044025860C60908F80000244F4B70B40E
:10E36000996A9D6ADC6A15F07C7FC5F305525E6C84
:10E370005CD0C6F3CC06C4F3002401F0030104FB17
:10E3800006F4012907EE904AB8EEE77A03D0022995
:10E3900075D000294FD007EE902ADFED416AF8EEE4
:10E3A000E77A1B6C86EEA76ADFED3E5AC3F30803DB
:10E3B00006EE903AB7EE005AF8EEE66A76EE856A17
:10E3C000E7EE256A66EE266A344AB7EE006A136CF9
:10E3D000C3F3462307EE103AB8EEC77A70BC37EEA7
:10E3E000067AC6EE877AFCEEE77AC0ED007A136C07
:10E3F000C3F3064307EE103AB8EEC77A37EE067A53
:10E40000C6EE877AFCEEE77AC0ED017A136CC3F3AF
:10E41000066307EE903AF8EEE77A77EE867A86EEB4
:10E42000A77ABCEEC77A80ED027A704770BCC0E96B
:10E430000022826070471968890627D5196807EE9F
:10E44000902A194AF7EE004AC1F3C101F8EEE77AC3
:10E450001B6CCA409FED135AC3F3080306EE102A43
:10E4600006EE903AF8EEC65AF8EEE66A85EEA76A2E
:10E4700076EEA46AE7EE056A66EE266AA4E707EE82
:10E48000902ADFED0A6AF8EEE77A8AE707EE902A2B
:10E49000DFED076AF8EEE77A83E700BF0044025831
:10E4A0000024744A000000390090D0030024F44A8C
:10E4B0000024744C4F4B70B4996A9D6ADC6A15F461
:10E4C0007C3FC5F30532DE6B5CD0C6F3CC06C4F3EB
:10E4D000001401F0030104FB06F4012907EE904A41
:10E4E000B8EEE77A03D0022975D000294FD007EEA5
:10E4F000902ADFED416AF8EEE77A9B6B86EEA76A19
:10E50000DFED3E5AC3F3080306EE903AB7EE005A29
:10E51000F8EEE66A76EE856AE7EE256A66EE266A2A
:10E52000344AB7EE006A936BC3F3462307EE103A02
:10E53000B8EEC77A70BC37EE067AC6EE877AFCEE84
:10E54000E77AC0ED007A936BC3F3064307EE103A07
:10E55000B8EEC77A37EE067AC6EE877AFCEEE77A2F
:10E56000C0ED017A936BC3F3066307EE903AF8EEC1
:10E57000E77A77EE867A86EEA77ABCEEC77A80EDE8
:10E58000027A704770BCC0E9002282607047196847
:10E59000890627D5196807EE902A194AF7EE004A2E
:10E5A000C1F3C101F8EEE77A9B6BCA409FED135AA5
:10E5B000C3F3080306EE102A06EE903AF8EEC65AA8
:10E5C000F8EEE66A85EEA76A76EEA46AE7EE056ADB
:10E5D00066EE266AA4E707EE902ADFED0A6AF8EEF7
:10E5E000E77A8AE707EE902ADFED076AF8EEE77A26
:10E5F00083E700BF004402580024744A0000003939
:10E600000090D0030024F44A0024744C08B505F0AF
:10E610000DFE054B054A1B6AC3F30213D35C03F0DE
:10E620001F03D84008BD00BF0044025860C6090857
:10E630002DE9F04383680446B04D87B0E169B04EE0
:10E64000D0E904201A43236802431F68606EB34276
:10E6500042EA010205EA0705A76942EA0002E0680A
:10E6600042EA05021A605A6822F4405242EA000265
:10E670005A6000F0A680986806F16846226AA14DAB
:10E6800006F582363A430540606AB34242EA050223
:10E690009A60DA6A22F00F0242EA0002DA6225D0BA
:10E6A000994A934257D0994A934200F02D82984A52
:10E6B000934200F09982974A934200F0F181964A82
:10E6C000934200F09B82954A934200F0D785944A8A
:10E6D000934200F0B385012500234FF00112284634
:10E6E0002367C4E91A2307B0BDE8F0838D4B5B6D47
:10E6F00003F03803282BEED88B4A13441D7AB1F56A
:10E70000004F35D0202D00F2D581202D00F2BA80A7
:10E71000DFE815F09A016D01B800B8006401B80097
:10E72000B800B8003B01B800B800B800B800B800A5
:10E73000B800B8000E01B800B800B800B800B800C2
:10E74000B800B800B800B800B800B800B800B80009
:10E75000B800B800C400734B5B6D03F00703052BD2
:10E76000B9D8714AB1F5004F134493F83450C9D168
:10E77000202D00F20E82202D00F2FA81DFE815F044
:10E780001204D403F801F801A403F801F801F80118
:10E790000204F801F801F801F801F801F801F801A4
:10E7A0006E03F801F801F801F801F801F801F80129
:10E7B000F801F801F801F801F801F801F801F80191
:10E7C0003F0399684F4A57480A403A439A60DA6AC9
:10E7D000616A22F00F020A43DA62836D03F00703D5
:10E7E000052B3FF678AF504A134493F83C60202E37
:10E7F00000F29481012E7FF66EAFB31E1E2B3FF602
:10E800006AAF01A252F823F0EBED0408D7E6040842
:10E810007FED0408D7E60408D7E60408D7E6040825
:10E82000D5ED0408D7E60408D7E60408D7E60408BF
:10E83000D7E60408D7E60408D7E60408D7E60408B4
:10E8400021ED0408D7E60408D7E60408D7E6040853
:10E85000D7E60408D7E60408D7E60408D7E6040894
:10E86000D7E60408D7E60408D7E60408D7E6040884
:10E87000D7E60408D7E60408D7E60408D7E6040874
:10E8800029EC040801250023A3F110014FF6EF72D3
:10E8900091423FF620AF2268D3601DE7002800F0C8
:10E8A0009F84012800F0B085022800F0C38503286A
:10E8B00000F0E885042800F00D86052800F0708639
:10E8C000062800F0AF86072800F0F486082800F03C
:10E8D0008087092800F09C870A2800F0F18743F61A
:10E8E0000953124A0B2818BF13466268002503EB30
:10E8F0005203B3FBF2F39BB2C6E700BFF369FFCF4D
:10E90000000C0058FFF4FF11004400400048004094
:10E91000004C0040005000400014014000780040CE
:10E92000007C00400044025870C6090800093D0000
:10E93000B74B1A68920640F15A841A68B54BC2F375
:10E94000C102D3400028D0D0012800F085840228DD
:10E9500000F0CC84032800F0C684042800F0418530
:10E96000052800F08486062800F0EB86072800F0D2
:10E970000C86082800F03D86092800F081860A28C8
:10E9800000F0EE860B28B0D126E06846FFF7E6FCE3
:10E99000626A019B002AA8D0012A00F05D84022A45
:10E9A00000F0A484032A00F09E84042A00F0198554
:10E9B000052A00F01385062A00F09D85072A00F03D
:10E9C000E485082A00F01586092A00F059860A2AEB
:10E9D00000F0C6860B2A88D11B0A86E703A8FFF73A
:10E9E00069FD626A049B002A3FF47FAFD4E705F01B
:10E9F000EDFB636A03B3012B00F01285022B00F0DC
:10EA0000EA84032B00F0E484042B00F02D85052B11
:10EA100000F02785062B00F0F585072B00F03B86DC
:10EA2000082B00F0BC86092B00F0DA860A2B00F0D8
:10EA30005D870B2B08BF000A6268002500EB5203BC
:10EA4000B3FBF2F39BB21FE705F0D8FB636A03B395
:10EA5000012B00F0DE84022B00F0C984032B00F0B0
:10EA6000C384042B00F00685052B00F00085062BDF
:10EA700000F0C285072B00F01A86082B00F09B8659
:10EA8000092B00F0C2860A2B00F017870B2B08BF5A
:10EA9000000A626800EB5203B3FBF2F39BB2F3E6A9
:10EAA0005B4B5B6D03F00703052B3FF614AE5A4A30
:10EAB000D55C24E6402D7FF40EAE002800F0938351
:10EAC000012800F0A984022800F0B984032800F08E
:10EAD000DC84042800F00185052800F05D85062807
:10EAE00000F09C85072800F0DE85082800F05F868E
:10EAF000092800F09C860A2800F014870B280CBF18
:10EB000080234FF40043F0E6414B5B6D03F00703B5
:10EB1000052B3FF6E0AD414AD55CF0E5402E7FF491
:10EB2000DAAD002900F09583012900F080840229E4
:10EB300000F09484032900F0C484042900F02185A6
:10EB4000052900F04B85062900F09685072900F07D
:10EB50001186082900F05586092900F08B860A29BC
:10EB600000F0C7860B290CBF80254FF4004582E0DA
:10EB700001250023A3F110014FF6EF7291423FF6F9
:10EB8000AAAD23F00F02C3F3420321681343CB6005
:10EB9000A2E5402D7FF49FAD002800F0608301289E
:10EBA00000F05F83022800F08284032800F0DB84F9
:10EBB000042800F00D85052800F05085062800F097
:10EBC000CC85072800F00F86082800F03886092831
:10EBD00000F09D860A2800F000870B280CBF4FF438
:10EBE00080714FF480313CE3094B5B6D03F0070308
:10EBF000052B3FF670AD0A4AD55C80E5044B5B6D92
:10EC000003F03803282B3FF666AD064AD55C76E55F
:10EC1000004402580090D003A4C60908A4C60908FD
:10EC2000A4C6090878C60908002900F06F830129E5
:10EC300000F0F983022900F00C84032900F04584D8
:10EC4000042900F09884052900F0CC84062900F0FE
:10EC50000B85072900F08B85082900F0DF8509293D
:10EC600000F0E9850A2900F0378643F60955C94BBB
:10EC70000B2918BF1D46676807EB4703AB423FF6F9
:10EC80002AADB5EB073F3FF626AD202E00F20183FB
:10EC9000012E7FF620ADB31E1E2B3FF61CAD01A248
:10ECA00052F823F073F10408D7E6040861F1040870
:10ECB000D7E60408D7E60408D7E60408F1F004080C
:10ECC000D7E60408D7E60408D7E60408D7E6040820
:10ECD000D7E60408D7E60408D7E604086FF004086E
:10ECE000D7E60408D7E60408D7E60408D7E6040800
:10ECF000D7E60408D7E60408D7E60408D7E60408F0
:10ED0000D7E60408D7E60408D7E60408D7E60408DF
:10ED1000D7E60408D7E60408D7E60408FFEF04089E
:10ED20009D4B1A68950640F1F3821B689B4DC3F317
:10ED3000C103DD4000299ED0012900F0B3830229E0
:10ED400000F0AA83032900F0A483042900F07F8443
:10ED5000052900F0B684062900F03685072900F061
:10ED60008685082900F0BF85092900F0FC850A295D
:10ED700000F0E6850B297FF47EAF2D0A7BE703A820
:10ED8000FFF798FB636A049D03B3012B00F0B9827F
:10ED9000022B00F0B182032B00F0AB82042B00F0B9
:10EDA0002E83052B00F02883062B00F09A83072B77
:10EDB00000F0F983082B00F02B84092B00F0658408
:10EDC0000A2B00F0FB840B2B00F05382002D3FF444
:10EDD00083AC50E76846FFF7C1FA636A019D002BD8
:10EDE000D3D1002D3FF478AC45E7FFF70FFC636A01
:10EDF0000546002BC9D1002D3FF46EAC3BE700283F
:10EE000000F0AA82012800F01E83022800F04D8342
:10EE1000032800F0A683042800F0D883052800F01A
:10EE20000D84062800F09284072800F0DF8408286B
:10EE300000F03785092800F049850A2800F0D085C0
:10EE400047F61223564A0B2818BF1346626800255E
:10EE500003EB5203B3FBF2F39BB28BE64E4B1A6803
:10EE6000910640F18F821A684C4BC2F3C10223FA1B
:10EE700002F200B3012800F04483022800F09B83D3
:10EE8000032800F0D483042800F05584052800F0FE
:10EE90008184062800F0DD84072800F047850828D3
:10EEA00000F04785092800F07F850A2800F0798561
:10EEB0000B2808BF120A616800254B0803EB4203C8
:10EEC000B3FBF1F39BB255E603A8FFF7F3FA626ACE
:10EED000049902B3012A00F09A82022A00F0AD825E
:10EEE000032A00F0CA82042A00F0F282052A00F008
:10EEF0004F83062A00F07983072A00F0D283082A7C
:10EF000000F03C84092A00F08F840A2A00F0028570
:10EF10000B2A08BF090A62680025530803EB410366
:10EF2000B3FBF2F39BB225E605F050F9636A03B335
:10EF3000012B00F08C82022B00F0BC82032B00F02E
:10EF40000B83042B00F03E83052B00F08383062BFC
:10EF500000F00984072B00F04F84082B00F0938405
:10EF6000092B00F0B6840A2B00F00C850B2B08BF90
:10EF7000000A616800254A0802EB4003B3FBF1F385
:10EF80009BB2F7E56846FFF7E9F9626A0199002A42
:10EF9000C1D09FE700093D00004402580090D00313
:10EFA00000127A0005F02AF9636A03B3012B00F01E
:10EFB0004C82022B00F08082032B00F0D782042BBE
:10EFC00000F00283052B00F03E83062B00F0C18386
:10EFD000072B00F00E84082B00F05284092B00F060
:10EFE0007F840A2B00F0BC840B2B08BF000A6168E9
:10EFF0004A0802EB4003B3FBF1F39BB2BAE5636A44
:10F0000003B3012B00F04A83022B00F0BD83032BD6
:10F0100000F03C84042B00F04C84052B00F09C8411
:10F02000062B00F09484072B00F08D84082B00F051
:10F03000E984092B00F005850A2B00F0FE840B2BD8
:10F0400000F0F784C54800217D0800233A464019A6
:10F0500041F1000149F064F8A0F54073C04A9342C1
:10F060003FF639AB23680025D860FFF735BBBD4BB1
:10F070001A68900640F14A821A680021BA48C2F321
:10F08000C102636AD0400BB3012B00F0C583022B91
:10F0900000F0F483032B00F00784042B00F08D8430
:10F0A000052B00F08484062B00F0DA84072B00F097
:10F0B000D484082B00F0CD84092B00F0C6840A2BE1
:10F0C00000F0B3840B2B01D1000A00214FEA012983
:10F0D00000237D083A464FEA002849EA106918EBF8
:10F0E000050049F1000149F01BF8A0F54073B5E7B0
:10F0F0006846FFF733F9636A019800210BB3012BCF
:10F1000000F05E82022B00F09782032B00F00E834A
:10F11000042B00F07483052B00F0A483062B00F071
:10F12000F183072B00F03A84082B00F03484092B7C
:10F1300000F02D840A2B00F0A4840B2B01D1000ACF
:10F14000002162680F0206020023510847EA106797
:10F15000701847F1000148F0E3FFA0F540737DE728
:10F1600003A8FFF7A7F9636A04980021002BE8D0F1
:10F17000C5E7FFF74BFA636A002105460BB3012B85
:10F1800000F08182022B00F01083032B00F08383B8
:10F19000042B00F09983052B00F0EE83062B00F082
:10F1A000E583072B00F0F183082B00F06784092B1F
:10F1B00000F060840A2B00F059840B2B01D1050A62
:10F1C000002162680F022E020023500847EA1567EB
:10F1D000301847F1000148F0A3FFA0F540733DE768
:10F1E000624BFFF782BB4FF40043FFF77EBB002862
:10F1F00000F0EB80012800F02E81022800F05E81F3
:10F20000032800F0BB81042800F0E581052800F008
:10F210002882062800F0B5820728E1D0082800F0EF
:10F22000F380092800F006810A2800F05381504B32
:10F230004D4A0B2818BF1346FFF757BB494B5B6D70
:10F2400003F00703052B3FF646AA4A4AD55CFFF7B1
:10F2500056BA4FF400450EE55B08FFF746BB4FF486
:10F2600080316268002501EB5203B3FBF2F39BB2DD
:10F2700080E42D0A002D3FF42FAAFCE4394B5B6D8E
:10F2800003F00703052B3FF626AA3B4AD55CFFF7A0
:10F2900036BA402E7FF41FAA636A03B3012B00F035
:10F2A0000C82022B00F09882032B00F0D782042BF3
:10F2B00000F02383052B00F08C83062B00F0858360
:10F2C000072B00F07D83082B00F09283092B00F0C0
:10F2D000A7830A2B00F09F830B2B00F097834FF43A
:10F2E00000000021B0E6254AA2FB03239B08FFF79C
:10F2F000FCBA224BA3FB0535AD08002D3FF4ECA969
:10F30000B9E46D08002D3FF4E7A9B4E4174DB2E469
:10F3100000296FD0012900F0C280022900F0F3809B
:10F32000032900F04A81042900F08A81052900F0B0
:10F330000582062900F036820729E7D0082972D015
:10F34000092900F086800A2900F01581084D064B36
:10F350000B2918BF1D468EE4094B77E50000093DD7
:10F36000FFFC0F00004402580090D00300093D004C
:10F3700090D00300A4C60908A4C60908ABAAAAAA8B
:10F3800000127A00002850D0012800F0B280022834
:10F3900000F00F81032800F04881042800F09681D6
:10F3A000052800F0F481062800F050820728D3D009
:10F3B000082848D0092878D00A2800F00781C54BD2
:10F3C000C54A0B2818BF134640E5C44BFFF78DBA5A
:10F3D000C34BA3FB00308008FFF72EBBC14AA2FB42
:10F3E0000323DB08FFF781BABD4BA3FB0030800885
:10F3F000FFF74FBBB94D3EE4BA4BA3FB0535ED0813
:10F40000002D3FF469A936E4B74BFFF76EBA4908FF
:10F4100081E54008FFF73DBB4FF48043FFF765BA35
:10F420004008FFF709BBB04D25E4AB4B0EE54FF4A8
:10F43000804520E4AD4BFFF758BA89086BE54FF4DF
:10F440000053FFF752BAAA4B00E54008CFE5400849
:10F450008FE5A64D0FE4A74BFFF747BA4FF40055D1
:10F4600009E4A04BA3FB0030C008FFF7E5BA9D4BB1
:10F47000A3FB0030C008FFF70CBB994BA3FB012393
:10F48000990848E59C4BFFF730BA41F25553FFF716
:10F490002CBA934BA3FB0535AD08FFF7ECBB954D9C
:10F4A000FFF7E9BB6D08FFF7E6BB8F4BCEE44FF4E7
:10F4B0008041D6E680085CE5800898E58F4BFFF731
:10F4C00014BA41F25555FFF7D6BB8B4DFFF7D3BBAE
:10F4D000C90820E57F4BFFF708BA4FF48053FFF7C8
:10F4E00004BA0C23B5FBF3F5002D3FF4F5A8FFF7A4
:10F4F000C2BB7A4BAAE47A4AA2FB0323DB08FFF7DC
:10F50000F4B95208D7E47D4DFFF7B5BB636A03B386
:10F51000012B00F08681022B00F09481032B00F078
:10F52000FC81042B00F00882052B00F05D82062B85
:10F5300000F06382072B3FF485AD082B00F0AE800E
:10F54000092B00F021810A2B00F0B3810B2B00F076
:10F55000FA816B48032177E5614BA3FB00239808F0
:10F5600007E5684B72E442F6AA217AE65C4BA3FBFE
:10F57000002398083BE5574DFFF77DBB624BFFF733
:10F58000B4B94FF48055FFF776BB1B09FFF7ADB94F
:10F590000A23B1FBF3F1BEE440F6CC43FFF7A5B973
:10F5A0005A4BFFF7A2B92D09002D3FF495A8FFF79C
:10F5B00062BB504B4AE492087DE4534DFFF75BBBBE
:10F5C0004008BEE5C008D4E4C00810E5474B3DE460
:10F5D0004FF4005145E64E4BFFF787B940F6CC4556
:10F5E000FFF749BB494DFFF746BB0C23B1FBF3F1D5
:10F5F00091E45B09FFF779B9394BA3FB0030C008F0
:10F60000FFF747BA364BA3FB0030C008FFF714BA28
:10F610006D09002D3FF460A8FFF72DBB40F6AA232B
:10F62000FFF763B93B4BFFF760B93B4B0EE42C4B44
:10F63000A3FB02239A083EE4800882E5374B05E4E9
:10F64000334DFFF718BB0A23B0FBF3F0CFE4ED080E
:10F65000FFF711BB0A23B0FBF3F08AE441F69811DF
